:020000040800F2
:10000000F0FF001055C005084153050815B7010859
:10001000F5C00508F5C00508F5C00508000000009A
:10002000000000000000000000000000455305082B
:1000300049530508000000004D530508D1A20008EF
:10004000F5C00508F5C00508F5C00508F5C00508A8
:10005000F5C00508F5C00508D1BA0008F5BA0008D2
:1000600019BB00083DBB000861BB00089DB5000836
:10007000B1B50008C5B50008D9B50008EDB5000850
:1000800001B6000815B60008F5C00508F5C005085A
:10009000F5C00508F5C00508F5C0050885BB0008D2
:1000A00065CC0008C5CB000875CC0008B5CB0008AE
:1000B000EDCB0008FDCB00080DCC0008B1AF000867
:1000C00085C40008B9AF000889C40008F5C0050858
:1000D000F5C00508B91A0508B91B0508DD1C050897
:1000E000C1BB0008F5C00508D5B5050885CC0008DA
:1000F0003DCC000895CC00082DCC000829B600089E
:10010000F5C00508F5C005081DCC0008F5C00508B8
:10011000011E0508251F0508F5C00508F5C00508DE
:100120003DB6000851B6000865B6000879B600086B
:100130008DB60008F5C00508F5C00508F5C005082E
:10014000F5C00508F5C00508F5C0050851530508B8
:10015000A1B60008B5B60008C9B6000849200508D0
:10016000C1AF00088DC40008F5C00508F5C005083A
:10017000F5C00508F5C00508F5C00508F5C0050877
:08018000F5C00508F5C00508F3
:1080000010B40C4B4FF0E02C1A68DCF8180019681B
:108010008A42F9D159688842F6D89C684FF47A713F
:1080200001FB04F31B1AB3FBF4F35DF8044B01FBF3
:1080300002307047C0190020074BD0F8E4105B688D
:10804000D0F8F0205B1A9A42B8BFC0F8F030012394
:1080500080F81C3100207047001000E0B04A00EBAF
:10806000800102EBC1012DE9F041CB685B68B3F8F8
:1080700014C01CF0010F4FEA800E40F082805FFABE
:108080008CF4A6074DD5BFF35F8F91F82840012CE3
:10809000E5B200F0F7804FEA400C198BBFF35F8F19
:1080A0000EEB000102EBC10191F82840022C00F018
:1080B00017810EEB000102EBC10191F82840032C5F
:1080C0000AD191F82A1039B10CEB0001114491F852
:1080D0008440002C40F06381998889B241F480612A
:1080E00099800CEB0001114491F986100EEB00040D
:1080F00002EBC40494F8284001348C420FD184442C
:10810000944400218CF884109CF88510002940F0DC
:10811000E080704402EBC000002380F82530BDE809
:10812000F08165076BD400EB4007174414F040045E
:108130001FFA8CF697F986504FEA400C00F0E68063
:108140001E8A0C6BF6B26655EEB2741C64B291F8DE
:10815000288087F88640E51CA845214600F0458127
:108160000EEB000502EBC50595F82850AC42BDD1D9
:108170000CEB00011144023676B281F8866031467C
:10818000B4E71C8824F400642404240C1C801C889C
:10819000A4B244F480641C8000EB4004144491F8C1
:1081A0002A50002684F886604FEA400C002D56D0F5
:1081B00094F88440002C4ED00EEB000102EBC1017C
:1081C000844491F828109444012402298CF88440B6
:1081D00004D1198889B241F4006119800EEB0001C5
:1081E00002EBC10191F8261041F0010119820EEB5A
:1081F000000302EBC30292F82830BDE8F08100EBE7
:108200004005154491F82A40012685F8856000FA5A
:1082100006FC002C7ED095F88440002C40F0828033
:108220000EEB000102EBC10191F82910002900F0CA
:10823000B98019880CEB0004144489B241F4007130
:10824000198094F88610013149B284F886101C8890
:10825000E705FCD44AE791F82710FF29ACD00EEBD4
:10826000000102EBC10191F8264004F0FE041C82DB
:1082700091F82730FF2BBAD084449444FF238CF824
:108280008630B4E791F82A1000293FF404AF00EBE0
:10829000400111444FEA400C91F88440002C3FF417
:1082A000FCAE1C8824F480642404240C1C80BFF3DE
:1082B0005F8F1C8B1C8881F88550A4B244F4007435
:1082C0001C809C8891F98610A4B244F480649C8040
:1082D0000CE7998821F440710904090C998018E78A
:1082E00091F82A1000293FF4E4AE0CEB0001114490
:1082F00091F88440002C3FF4DCAE1C8891F9861084
:1083000024F480642404240C1C8041E036062FD41D
:108310002946EBE695F88410002981D089E700BF53
:10832000C019002091F828400E6B022C1C8847D9F8
:1083300024F480642404240C1C801F8A95F9864050
:10834000FFB237550F6B198889B241F4007119805B
:10835000E4B21E8A611C49B2F6B27E54A11C9C880C
:10836000A4B249B244F4806485F886109C806EE71C
:108370006E1C41D0CC6A665D6C1CF5B21D8291F812
:10838000285064B2A54287F8864021467FF4AEAEFD
:108390009C8824F480642404240C9C80A6E691F933
:1083A0008610F5E7198889B241F4807119800CEBC9
:1083B00000011144012481F8844091F9861046E7B8
:1083C000A4B244F400741C801F8A95F98640FFB261
:1083D0003755E4B20F6B1E8A611C49B2F6B27E5467
:1083E000E11C49B285F8861031E79D8825F4806547
:1083F0002D042D0C9D80B3E687F8864091F8274028
:10840000E4B21C8291F82A4024B991F8281000297E
:108410007FF4EDAE998821F480610904090C9980FC
:10842000E5E600BF10B404698269E468416814603D
:1084300000234024C2E90234446993630C31C2E949
:108440000433C2E90633C2E90833C2E90A33C2E998
:108450000C33516094B1C269E46893634FF4803087
:10846000C2E90041C2E90233C2E90433C2E906337A
:10847000C2E90833C2E90A03C2E90C335DF8044BD0
:10848000704700BFD0E9001300221A60037D1F2B44
:1084900007D9203B202202FA03F343F01803CB60F4
:1084A0007047202202FA03F343F018038B607047F1
:1084B0001B4B016803F57D7C02E02C3363452CD017
:1084C0001A688A42F9D170B593F804E0427996456A
:1084D0000BD02C33634505D01A688A42F4D02C3374
:1084E0006345F9D14FF0FF3070BD9E468468DEF8D9
:1084F0000C50A5424FF0000208D00132032A0EF1C1
:108500000C0EE6D0DEF80C50A542F6D1DEF8105085
:10851000C668B542F1D150B270BD4FF0FF30704720
:108520005CDC0508002A4FEA014C30B503460ABF5F
:10853000E6468E468C4600F1C005002419689A680C
:1085400041EA0C0142EA0E029A60C3E900140C33BE
:10855000AB42F3D1D0F8C030C0F8C44043EA0E03B8
:10856000C0F8C030C0F8C84030BD00BF8369196989
:10857000B3F80CC00A6830B49C6822F00102246889
:108580000A60A28992B222EA0C02A281027D0068EE
:108590001F2A06D94568203A082494402C4245D029
:1085A000FEE70568082494402C42F9D1202404FAFF
:1085B00002F28260264A1278002A35D01A7E012AF9
:1085C00039D0D3F8F4200132C3F8F420EFF311814D
:1085D000502282F3128858685C6C026822EA040216
:1085E0009C6C2243C9B2026081F31188D3E90C402C
:1085F0001A6999681D6C096814605061D3E90E40CE
:10860000546090600024B3F8A800D5604C62C86242
:1086100010680124204310601C7683F8F1408A8999
:108620009B8913439BB28B8130BC7047202404FA92
:1086300002F2C260BEE7002283F8F120D3F8F8000E
:108640000A68013022F00102C3F8F8000A60EBE783
:108650000400001010B40C4C6368002B11DD0020E6
:1086600004F1080C0146DCF8A03003F1C0025960A7
:108670000C339342FBD16368013083420CF5807C5C
:10868000F1DC5DF8044B704704000010F0B5414C7C
:1086900004EB401393F8243403B9F0BD3E4B93F838
:1086A0008D5093F88E2095424FEA401C0CD002EB7F
:1086B000420E03EBCE0E9EF89060771E012F4FEA1C
:1086C000420E58D9032E51D004EB0C00A0F8081428
:1086D000EFF31182902383F3128890F80A34B0F8F4
:1086E000081443EA41030021D2B29BB280F80A1475
:1086F00082F311882178D0F820441A0982EA1322E3
:108700005A40C9B1D0F80C14D4F8A040D2431B0190
:108710009BB202F00F0201208840134304F1C00114
:108720005A0013F4004F93B202D1626802436260B0
:108730000C34A142F4D1F0BDD0F80C14D4F8A04010
:108740001B0110319BB202F00F020120884013433D
:1087500004F1C0015A0013F4004F93B202D16268D1
:10876000024362600C34A142F4D1F0BD561C06F005
:108770000306AE42A8D0964403EBCE03184490F80B
:108780009D100029A0D004EB0C03012283F80A24D9
:108790009AE700BF04000010C0190020704700BF16
:1087A000024B03EB401393F82504704704000010BC
:1087B0004368B0F8502010B41A83EFF311825023AD
:1087C00083F312884168446C0B6823EA0403C46C89
:1087D0002343D2B20B6082F31188D0E9074182684B
:1087E000036912681C605961D0E909415C60C46A80
:1087F0009960B0F86010DC600023D1625DF8044B32
:108800000376704710B4037D02681F2B09D95468A2
:10881000203B202101FA03F31C4215D15DF8044BE3
:1088200070471468202101FA03F31C42F6D00D4969
:108830004068002481F8F04001685DF8044B21F0A5
:10884000010101609360704706494068002481F887
:10885000F04001685DF8044B21F001010160D36034
:10886000704700BFC0190020122301480B807047D9
:1088700088010020042301480B8070479C010020E0
:108880001C48D0F8103AD0F8182A10B59B184FF0B1
:108890001A040C8001D1184810BD174AD0F8140AE8
:1088A00002F1100411464FF0000E4FEA137CB3F1B1
:1088B000204F34BF0CF1300C0CF1370C81F802C0A2
:1088C00081F803E002318C424FEA0313EDD102F14B
:1088D00008040021030FB0F1204F34BF3033373389
:1088E0009374D174023294424FEA0010F2D10248DC
:1088F00010BD00BF0070FF1FA0010020D0E90920BB
:10890000131A58425841704790F84F3830B53BB968
:1089100090F84D1890F84E380124DAB2914200D800
:1089200030BDB0F8565804FA03F22A43A0F856288E
:108930000133F2E70379024613F0010006D0D2E9D1
:108940000731D2685B1A013A03EA0200704710B59A
:10895000037913F0010304460ED0FFF7EBFF034643
:1089600050B1226A6369E1689B5C0132B2FBF1F0AD
:1089700001FB1022DBB22262184610BD03799B076F
:108980000AD5436A8269D154436A02690133B3FB51
:10899000F2F102FB11334362704770470171704777
:1089A0000379014613F0020007D00B69D1E90921D0
:1089B000013B521A1A40D2B2981A704782B01D4B2E
:1089C0001D49002201920193019B04330193019BF5
:1089D0001A688B6803F00C03042B02D0082B05D017
:1089E000164A174BC3F8F42002B0704748684B682A
:1089F000400203F03F0314D44A681049B1FBF3F37B
:108A0000C2F3881203FB02F20B4B5B68C3F3014312
:108A100001335B00B2FBF3F2094BC3F8F42002B060
:108A200070474968B2FBF3F2C1F3881303FB02F20B
:108A3000EAE700BF50280040003802400024F4005C
:108A4000C01900204A484B494B4BDFF830C12DE993
:108A5000F04F4FF0010A4FF002094FF004080827C9
:108A60001026202540244FF0800E30F8022B12F003
:108A7000010F03D01960A3F804A0083312F0020F0D
:108A800003D01960A3F80490083312F0040F03D048
:108A90001960A3F80480083312F0080F02D019609F
:108AA0009F80083312F0100F02D019609E800833A7
:108AB00012F0200F02D019609D80083312F0400F91
:108AC00002D019609C80083312F0800F03D0196027
:108AD000A3F804E0083312F4807F05D04FF4807BC4
:108AE0001960A3F804B0083312F4007F05D04FF4E6
:108AF000007B1960A3F804B0083312F4806F05D02E
:108B00004FF4806B1960A3F804B0083312F4006FBF
:108B100005D04FF4006B1960A3F804B0083312F4C9
:108B2000805F05D04FF4805B1960A3F804B0083370
:108B300012F4005F05D04FF4005B1960A3F804B095
:108B4000083312F4804F05D04FF4804B1960A3F81E
:108B500004B00833D20B04D04FF4004219609A805D
:108B6000083301F5806161457FF47FAFBDE8F08F88
:108B700050E0050800000240B81A0020001802402A
:108B800010B584464FEA810E102312F4004F14BF33
:108B90000E2407245200013BCCF8004092B2F4446A
:108BA000F3D100EB81128C01035142F821301220E5
:108BB00010BD00BF10B584464FEA810E0424130B8C
:108BC00003EB430318331201013CCCF8003092B29E
:108BD000F444F4D100EB01130A01845043F821401E
:108BE000062010BD704700BF704700BF034B00EB6D
:108BF000400003EBC00393F8190570470400001010
:108C0000064B93F8C825824283BF00EB400003EB7C
:108C1000C003D3F81C050020704700BF04000010FB
:108C20001D4B93F8CC25AAB3D3F8081509B1002041
:108C30000860012A2ED0D3F8201509B10020086061
:108C4000022A27D0D3F8381509B100200860032A7A
:108C500020D0D3F8501509B100200860042A19D09B
:108C6000D3F8681509B100200860052A12D0D3F89E
:108C7000801509B100200860062A0BD0D3F898159A
:108C800009B100200860072A04D0D3F8B0350BB131
:108C900000221A60704700BF040000101D4B93F8BB
:108CA000CC25AAB3D3F8081509B100200860012A21
:108CB0002ED0D3F8201509B100200860022A27D051
:108CC000D3F8381509B100200860032A20D0D3F862
:108CD000501509B100200860042A19D0D3F868158E
:108CE00009B100200860052A12D0D3F8801509B117
:108CF00000200860062A0BD0D3F8981509B100208F
:108D00000860072A04D0D3F8B0350BB100221A60EE
:108D1000704700BF04000010C24B93F83230002BA4
:108D200040F05781C04B93F8CC25002A00F05181C8
:108D300093F8181530B500294ED1D3F80815002046
:108D4000012A086047D993F83015002967D1D3F874
:108D500020150020022A08603DD993F84815002903
:108D600040F0D080D3F838150020032A086032D9AB
:108D700093F86015002940F0E880D3F850150020E2
:108D8000042A086027D993F87815002940F0FF805D
:108D9000D3F868150020052A08601CD993F89015AF
:108DA000002940F01781D3F880150020062A0860BA
:108DB00011D993F8A81500295BD1D3F89815002094
:108DC000072A086007D993F8C025002A76D1D3F87E
:108DD000B03500221A6030BDD3F80C158A0AA2F50E
:108DE0008012522A40F218814FF0FE0CEFF31180EE
:108DF000502282F312888D4C4D6A8A8A4FF02C0ED5
:108E00000EFB0C4C92B2013542F00102CCF820541A
:108E1000C0B28A8280F3118893F8CC258DE7D3F80D
:108E200024158A0AA2F58012522A40F203814FF0DB
:108E3000FE0CEFF31180502282F312887B4C4D6AB6
:108E40008A8A4FF02C0E0EFB0C4492B2013542F090
:108E50000102C4F82054C0B28A8280F3118893F8CA
:108E6000CC25D3F820150020022A08603FF675AF04
:108E7000B1E7D3F89C158A0AA2F58012522A00F2B3
:108E8000F2806B48024492F800C4EFF31180502244
:108E900082F31288654C4D6A8A8A4FF02C0E0EFBC5
:108EA0000C4492B2013542F00102C4F82054C0B221
:108EB0008A8280F3118893F8CC257EE7D3F8B41525
:108EC0008A0AA2F58012522A9BBF594812184FF005
:108ED000FE0C92F800C4EFF31180502282F3128846
:108EE000524C4D6A8A8A4FF02C0E0EFB0C4492B203
:108EF000013542F00102C4F82054C0B28A8280F3E6
:108F0000118864E7D3F83C158A0AA2F58012522A28
:108F100040F295804FF0FE0EEFF31180502282F365
:108F20001288424C4D6A8A8A4FF02C0C0CFB0E447E
:108F300092B2013542F00102C4F82054C0B28A82D4
:108F400080F3118893F8CC250CE7D3F854158A0ADE
:108F5000A2F58012522A77D94FF0FE0CEFF3118060
:108F6000502282F31288314C4D6A8A8A4FF02C0EBF
:108F70000EFB0C4492B2013542F00102C4F82054B9
:108F8000C0B28A8280F3118893F8CC25F5E6D3F835
:108F90006C158A0AA2F58012522A5AD94FF0FE0C9B
:108FA000EFF31180502282F31288204C4D6A8A8A96
:108FB0004FF02C0E0EFB0C4492B2013542F0010230
:108FC000C4F82054C0B28A8280F3118893F8CC256B
:108FD000DEE67047D3F884158A0AA2F58012522A79
:108FE0003CD94FF0FE0CEFF31180502282F312882F
:108FF0000E4C4D6A8A8A4FF02C0E0EFB0C4492B236
:10900000013542F00102C4F82054C0B28A8280F3D4
:10901000118893F8CC25C6E60548024492F800C4AE
:10902000E4E600BF8801002004000010C019002001
:109030005CDC05080D48024492F800C4F9E60B48D0
:10904000024492F800E467E70848024492F800C43A
:1090500084E70648024492F800C4A1E703480244AA
:1090600092F800C4BFE74FF0FE0C0EE75CDC050889
:1090700000EE100AB8EE400A704700BFBCEEC00A0E
:1090800010EE103A98B27047072809D8054B8C2289
:1090900002FB0033B3F8D005B0FA80F04009704706
:1090A0000020704704000010072806D8034B8C22CC
:1090B00002FB0033012283F8D22570470400001020
:1090C00070B53F4C8C2303FB004393F8DF3503B9A5
:1090D00070BD3C4B93F88DE093F88E2096450CD0F4
:1090E00002EB420C03EBCC0C9CF890506E1E012E50
:1090F0004FEA420C44D9032D3DD08C2202FB0042A2
:10910000A2F8D015EFF31181902383F31288B2F8FF
:10911000D05592F8D23543EA45030025C9B29BB237
:1091200082F8D25581F311881A09217882EA132234
:109130005A4001B1D2431B019BB294F8341AD4F8BF
:10914000305A02F00F021A438C2303FB004431BB58
:109150000121D4F85806A847D4F85416B4F8DC55C1
:109160008A8AD4F850362A438A8258601A6842F0B4
:1091700001021A6070BD551C05F003057545BCD091
:10918000944403EBCC03034493F89D100029B4D01E
:109190008C2303FB0043012283F8D225ADE7D4F8EA
:1091A000D835D4F854165B79086903F0FC031844E9
:1091B0000421A847D4F854368000988170BD00BFC0
:1091C00004000010C01900207AE700BF072808D863
:1091D000044B03EB401393F8242412B1012283F8CB
:1091E0000A24704704000010072808D8054B03EB39
:1091F0004013B3F80804B0FA80F04009704700202B
:10920000704700BF04000010054B93F8C825824248
:1092100086BF03EB4013D3F814040020704700BF4F
:1092200004000010012343770020704708B503466F
:109230008269006BD96A02449A6101B188470020B3
:1092400008BD00BF436A1B681B6A5B685B78024607
:1092500013F0010008BF5077704700BFF0B5224CF3
:10926000224A234B95B0054604F13C00CDE90002AB
:10927000049304F140000023CDE90503CDE90E334A
:109280001C4A09920B9304F1340210931393119327
:109290006B6A2F7F0A921868012302228DF80C3026
:1092A00007938DF820308DF834308DF848303B1D11
:1092B00002920E460C9351F071FC97B1330E84F874
:1092C00035303634320C330A22706370A670686A07
:1092D000694647F0ADFB6B6A186851F05FFC15B04A
:1092E000F0BD3534EEE700BF8801002020200020CB
:1092F000459200082592000810B5044694B050220B
:109300000649684654F016FA606A694647F090FBD1
:10931000636A186851F042FC14B010BDB0E0050853
:10932000C2628161704700BF2DE9F0410446406A86
:1093300000681E460F46904651F030FC237FA0691E
:10934000002B3DD0274D030E85F84530052205F151
:1093500046039870EA67020C000A58701A703B685E
:10936000C5F888300020D8F80030C5F89030012EBC
:109370002363C5F8A00028D0022E1FD1D8F80420FE
:10938000C5F89800796885F89400C5F89C101344D6
:109390001549C5F8A4200120236385F8A800C5F865
:1093A000AC10124B627F606AA3F11401002A08BF5F
:1093B000194647F03DFBE36A7BB1206BBDE8F081C5
:1093C0000B4B0422A3F14505C3E7074B85F89460D6
:1093D000C5E92630C5F8A400E3E7636A186851F0D0
:1093E000DDFBEAE7880100202D920008E80100205B
:1093F000CD010020704700BF00B583B081610192AC
:10940000049A0093C26201236A4601A9FFF78CFF08
:1094100003B05DF804FB00BF043070470D4B93F8B8
:109420006826D3F864160244D2B283F8682693F80B
:10943000682601441206C3F8641605D593F8682619
:1094400082F0800283F86826034B012283F8C4204F
:10945000704700BFC0190020880100202DE9F047A7
:10946000154FD7F86C56ED0A20D00026B14607F20A
:10947000A4687419D7F870361048D3F828A0C7F834
:109480009C9604EBD474641010234246E102D0474A
:109490000F280BDD0A4B03F1100153F8042B0132A6
:1094A00007D18B42F9D12546B542E2DCE802BDE89E
:1094B000F087661CF8E700BFC019002030200020AC
:1094C00064200020194B1968D3F8B4268A1A322A6E
:1094D00005DCD3F8C8268A1A002A0FDC704793F8F7
:1094E000B826D3F8BC1602F0010219B108688988C1
:1094F000B2B901830022C3F8C8267047D3F8BC264E
:1095000082B11068928810B444693231224218BF87
:1095100042835DF8044B08BF0283C3F8C816704746
:109520004183E7E73231C3F8C8167047C0190020FD
:10953000064AD2F8BC363BB192F8B8169A881B6836
:10954000C90754BF1A835A8300207047C0190020EE
:109550004FF40070034B1060D3F8D8360B60002036
:10956000704700BFC01900200020704701207047DD
:10957000012070470020704730B585B0684649F03B
:1095800071F80F480F4AD0F8FC10009B0E4D41F0C7
:109590008071C0F8FC10002400F1C840C2F8B05F30
:1095A000A0F5650054601168084CA0F67D60A0FB32
:1095B000030341F001019B0CA360116005B030BDB5
:1095C00000ED00E0001000E055CEACC5C019002051
:1095D0002DE9F84F01307E4C7E4D01F1FF385FFAE6
:1095E00080FB102601274FF0B5FA4FF4FA794FF0BF
:1095F000E0214FF47A7C6B68C3F30803002B40F042
:10960000C080EFF31183002B40F0BB802368886992
:1096100022689342FAD162689042F7D8A2680CFBA4
:1096200002FEAEEB000EBEFBF2FE0CFB03EE6B681F
:10963000C3F30803002B40F08680EFF31183002B67
:1096400040F081802368886922689342FAD1626879
:109650009042F7D8D4F808A00CFB0AF2121AB2FB19
:10966000FAF20CFB0323A3EB0E03B3F57A7FDED3F0
:10967000B9F10109BFD158464FF47A794FF01EFF76
:109680004FF0E021CC466B68C3F30803002B40F099
:109690008B80EFF31183002B40F08680236888696C
:1096A00022689342FAD162689042F7D8A2680CFB14
:1096B00002FEAEEB000EBEFBF2FE0CFB03EE6B688F
:1096C000C3F308030BBBEFF31183F3B92368886975
:1096D00022689342FAD162689042F7D8D4F808A081
:1096E0000CFB0AF2121AB2FBFAF20CFB0323A3EBF7
:1096F0000E03B3F57A7FE2D3B9F10109C3D1B8F112
:109700000108BFF470AFBDE8F88FEFF3118386F363
:109710001288D1F818A00A69D20344BFC4F80877A8
:10972000D1F818A02068D4F80827DBB283F3118899
:109730000244A0680CFB00F3A3EB0A03B3FBF0F3B5
:109740000CFB0233D3E7EFF3118386F31288D1F8D1
:1097500018A00A69D20344BFC4F80877D1F818A04A
:109760002068D4F80827DBB283F311880244A0688C
:109770000CFB00F3A3EB0A03B3FBF0F30CFB023387
:1097800071E7EFF3118286F3128888690B69DB03B6
:1097900044BFC4F8087788692368D4F808E7D2B2D0
:1097A00082F31188734439E7EFF3118286F312884C
:1097B00088690B69DB0344BFC4F8087788692368AC
:1097C000D4F808E7D2B282F3118873446EE700BF81
:1097D000C019002000ED00E02DE9F0411D4CDFF83C
:1097E0007C801D4F82B004F54075012602E00834EC
:1097F000A54224D094F90630002BF8D1206800F15E
:109800003F4303F57E0308EB932393F8A4345A09EE
:10981000032A03F01F0306FA03F317D0042A11D01A
:10982000022A02D17A6C13437B640023A1881A4672
:10983000CDE90036083450F047FFA542DAD102B036
:10984000BDE8F0813A6B13433B63EEE73A6C134398
:109850003B64EAE7B81A0020003802405CDC0508E7
:1098600009494B6C10B5094C43F480434B644022CA
:10987000002104F20C7053F0B5FF4FF0FF33C4F831
:109880004C37C4F84F3710BD00380240C0190020D3
:109890002DE9F0411348144D4FF41A72002153F092
:1098A000A1FF4FF00008A5F2AC4705F6880440F28E
:1098B000222655F82810002354F8332091420BD06B
:1098C00001330E2BF8D1002008F107084EF0C6FC3A
:1098D000B045EED1BDE8F08107EBC30393F8380D36
:1098E000F2E700BFB81D002008E105082DE9F843A4
:1098F000038AB0F80C801FFA88F818EA030829D008
:1099000005460E464FF00047B8FA88F327FA03F2EF
:10991000D24391B21B3B298208EA0208042B16D8D5
:10992000DFE803F0352C231A0300B36A002B37D08D
:1099300003F1FF3900231FFA89F9B362746A34B165
:1099400023682046494698476468002CF8D1B8F14E
:10995000000FD9D1BDE8F8837068696B036889B2DC
:109960009847B8F1000FCFD1F4E7B068A96B03684E
:1099700089B29847B8F1000FC6D1EBE7F068E96B00
:10998000036889B29847B8F1000FBDD1E2E73069AA
:10999000296C036889B29847B8F1000FB4D1D9E7B0
:1099A000EB6A1FFA83F9C9E770B50B4C0546072629
:1099B000013E00D170BD94F900001BF031FE031E82
:1099C00008DBEA1861789171A178E954052BDCBFB6
:1099D000E37813730434EBE700EA050810B5274B6E
:1099E00093F88D2093F88E309A4242D1244A92F80F
:1099F000F80AF8B192F8344A02F6382300EB400036
:109A0000D2F8382A03EBC000B4B140F20D3C00E0BC
:109A10001A6899689C894C600C6844F001040C60D9
:109A2000A2F848C09189183389B241F48071834209
:109A30009181EDD110BD1A68118821F080010904CF
:109A40001833090C118033F8141CD162118889B2C3
:109A500041F0800111805462B2F80CC033F8041C4C
:109A600041EA0C0189B28342918123F8044CE2D18E
:109A700010BD51F02DFB0028B8D110BDC019002039
:109A80000400001010B5044653F07CF981B2204662
:109A9000BDE81040FEF7FABD10B5044653F072F968
:109AA00081B22046BDE81040FFF70ABB38B50B4D28
:109AB00000EB400005F5A16303EBC00393ED027AD0
:109AC000D3ED037AE7EE007AC4002544B0EE670ACE
:109AD00053F058F9D5F80835186038BD0400001067
:109AE0000A4608B5054920B9054849F0EBF803488E
:109AF00008BD044849F0E6F8004808BD14210020DC
:109B0000C45A0608EC5A060810B5044C04480A4624
:109B1000214649F0D7F8204610BD00BF142100208F
:109B2000145B060810B5044C04480A46214649F067
:109B3000C9F8204610BD00BF14210020285B06088C
:109B400010B5044C04480A46214649F0BBF82046AB
:109B500010BD00BF14210020345B0608F8B5A0F644
:109B600068042379DB0725D5657994F84C3805F02E
:109B700001073D46FBB1D4F848341A68D36A5B0844
:109B8000536294F8503823B1B4F85A380133A4F82A
:109B90005A38606C85F001014EF048F8012384F8D2
:109BA0004F38002384F84D3884F84E38A4F85638DE
:109BB00084F84C38F8BD94F84F68012E04BF94F82F
:109BC0004D3884F84E382046FEF79EFE4EB90123EC
:109BD00084F84F3887EA0301606CBDE8F8404EF026
:109BE00025B8002384F84F383946F5E78069002806
:109BF00036D003681A6A127B2ABBD3E904125B6869
:109C0000496872B110B4546800220A6022609A88D0
:109C10005DF8044B22F003021204120C9A8047F004
:109C2000C1BA1A891206FCD41A89D20709D40022B3
:109C30000A609A8822F002021204120C9A8047F0FD
:109C4000B1BA9A89F0E78268002AD6D01168928862
:109C50000A83D3E904125B684968002AD2D1E0E79D
:109C6000704700BF806900B97047016830B4D1E91E
:109C700004424B6864687AB15568002222602A6009
:109C80009A8822F003021204120C9A800B6A1B7B42
:109C9000A3B930BC47F086BA1A891506FCD41A89D4
:109CA000D20714D4002222609A8822F00202120401
:109CB000120C9A800B6A1B7B002BEAD08368002B66
:109CC000E7D01A689B88138330BC47F06BBA9A8937
:109CD000E5E700BF38B590F82830012B044606D0E0
:109CE000407F08B9012038BD0023637738BD406A42
:109CF00003681A7B92B9637F002BF3D00A4D0B499E
:109D0000022305F6540246F04DFE95F85538D84327
:109D100003F0010300F001006377E7E71B6A002B03
:109D2000E9D0002038BD00BFC0190020500200203B
:109D300038B5044694F82830012B07D0637F0BB167
:109D400000236377012038BD1B6A23B1606A036872
:109D50001A7B002AF8D1637F002BF3D0074D084906
:109D6000022305F6540246F01DFE95F8553803F01F
:109D70000102DB076277E5D5DCE700BFC0190020F0
:109D8000500200202DE9F843DDF820800F461546EB
:109D90000021202204461E4653F024FDB8F1000F96
:109DA0000CD0D8F80030E3811B0C2382D8F80430A3
:109DB000B8F80A20E3821B0C62822383384651F0F4
:109DC00061FCEB0619D4431EB8B107EB000C01E0AF
:109DD000013B12D31CF801EDBEF12E0FF8D1C01AD1
:109DE000421E032AA8BF0322082B03F10109A8BFC2
:109DF00008239046B9441A4606E008280246B946A8
:109E0000A8BF08224FF000084FF0203339462360E6
:109E10006360204653F08EFC04F10800154B23814B
:109E200042464946837053F085FC611EE21D11F8DD
:109E300001CFACF16103192B9CBFACF1200C81F870
:109E400000C09142F3D104F10A0011F8013FA3F1DF
:109E50006102192A9CBF203B0B708142F5D1182367
:109E60002373330CA382E572099B6683E361BDE82B
:109E7000F88300BF202020002DE9F04FDFF84CB41C
:109E8000DBF8000085B0CBF8B406002B60D013449B
:109E90000C46174601F5FE7A99461FE0002F64D064
:109EA000DBF8E436BB4200F0C680DBF8E036BB42AC
:109EB00000F0F880DBF8E836DBF8EC16BB424BD854
:109EC000B94200F27081791A20464DF00BFC01373F
:109ED0004F4504F500740AF5007A39D0DBF8F03606
:109EE000BB42DBD8DBF80057FB1A296BDA080232D9
:109EF0008A4203F0070602D3AB6B9A420BD929467C
:109F0000104602924DF0BEFB029A0546002800F072
:109F10006A81CBF800072B79002B40F01E81D5F821
:109F20002880B8F1000F00F057812B6BD21AEB6834
:109F300006EBC20203EB422220462B464FF400718F
:109F40000137C0474F4504F500740AF5007AC5D1C2
:109F5000002005B0BDE8F08FB942B4D94FF40072CB
:109F60000021204653F03EFCB1E74FF40072394621
:109F7000204653F037FC802384F8BE310C2384F84C
:109F8000C231DBF8E016C54ADBF8D836C4F8C61192
:109F90009142C4F8CA3100F30B81C14AC14D82FB22
:109FA000010285FB01050A44C817C0EB6212C0EB31
:109FB0002530BD4D84F8C10185FB0265C2EB8216D8
:109FC0008010891B013120F03F0015440843D11750
:109FD000C1EBE5110A4484F8BF21B04A84F8C001FE
:109FE000013B934200F3F080AD4AAE4882FB03127E
:109FF00080FB03101A44D917C1EB6212C1EB203168
:10A00000A94884F8C51180FB0250C2EB8215891063
:10A010005B1B013321F03F0110441943D317C3EBFD
:10A02000E0131A4484F8C41184F8C3214AF6552376
:10A03000A4F8FE314BE74FF0FF3384F8EC3184F89D
:10A04000ED3184F8EE3184F8EF31522323706370E0
:10A050006123A37084F8E7314123E37084F8E6318B
:10A060007223002584F8E43184F8E531DBF8F83612
:10A07000C4F8E8314FF4F0722946201D53F0B2FBCA
:10A08000552384F8FE316FF05503C4F8F051C4F83D
:10A09000F451C4F8F85184F8FC5184F8FD5184F867
:10A0A000FF3114E74FF400720021204653F09AFB71
:10A0B0007E4B03CB45F6EB0323809023C4F80710B7
:10A0C000A37002220821F823C4F8030061732274EC
:10A0D0006375DBF8D8362273A27384F82C20DBF882
:10A0E000E0269B1A2362DBF8E826DBF8EC369B1AA5
:10A0F00063620023E372E3736377A377E37784F803
:10A100002D3084F82E3084F82F3084F83130684BAD
:10A11000A361684BC4F842303E232377012384F8BF
:10A120003030654A802384F8403084F846104AF67F
:10A130005521A4F8FE1103CA604BC4F84700C4F8C7
:10A140004B1003CB1388A4F84F309378C4F8520017
:10A15000C4F8561084F85130B9E64FF4007200216B
:10A16000204653F03FFB002E44D12B6C04F1200815
:10A17000002B7BD02B6B52491122CDE90066204683
:10A18000FFF700FE2B6C1A6C002A7ED01B6B4D492A
:10A19000CDE9006640461122FFF7F4FD04F14008C6
:10A1A0004FF4E0736DE0F91A20464DF09BFA8EE60D
:10A1B000FF2284F8C1214FF6FF72A4F8BF21374A6D
:10A1C000013B93427FF710AFFF2384F8C5314FF670
:10A1D000FF73A4F8C33129E741464FF400722046CB
:10A1E00053F000FB73E6384A231F43F8042F9A45C7
:10A1F000FBD16CE6D5E910253301002A43D0023BA0
:10A20000002D3FF464AE013BAD6CF9D1A0464FF494
:10A210000073002D3FF45BAECDE9027A08EB030634
:10A22000A24608E00024CDE900C4FFF7ABFDAD6C09
:10A23000BDB1B04515D02C7929682B6B404605F18E
:10A240001C0C112208F12008002CEBD16A792C6932
:10A2500042F02102CDE900C4FFF794FDAD6C002D62
:10A26000E7D15446029FDDF80CA030E6CDE9006648
:10A270003346DBF8DC1608222046FFF783FD4FF457
:10A28000F0736D6CC5E7013BBAE7CDE900660D4997
:10A29000334640461122FFF775FD7FE7FF03FB00C1
:10A2A0008320088297554541818080804C5B060859
:10A2B0003F00FF0029940E0D585B0608645B0608FA
:10A2C000445B0608485B0608DEADBEEFC0190020FF
:10A2D00010B4EFF31182102383F31288084B19682E
:10A2E0004FF0E02001311960816959600024C3F802
:10A2F00008470369D3B283F311885DF8044B7047B4
:10A30000C019002010B4EFF31181102383F31288D9
:10A310004FF0E022C9B29469136913F4803F0C4BEB
:10A320001EBF0120C3F8080794691868D3F80827EE
:10A3300081F31188996802444FF47A7000FB01F3AD
:10A340001B1B5DF8044BB3FBF1F300FB02307047BD
:10A35000C0190020234B5B68C3F3080310B4DBB9BA
:10A36000EFF31183C3B9204B4FF0E02C1A68DCF8EF
:10A37000180019688A42F9D159688842F6D89C6851
:10A380004FF47A7101FB04F3181AB0FBF4F05DF896
:10A39000044B01FB02007047EFF31181102383F39C
:10A3A00012884FF0E022C9B29469136913F4803F18
:10A3B0000D4B1EBF0120C3F8080794691868D3F835
:10A3C000082781F3118899684FF47A73024403FBDC
:10A3D00001F0001B5DF8044BB0FBF1F003FB020041
:10A3E000704700BF00ED00E0C01900202DE9F04FDC
:10A3F000037D02681F2B83B0044609D95068A3F17E
:10A4000020052021A940014207D103B0BDE8F08F0B
:10A410001068202199400142F7D04749474D4968CB
:10A42000A769C5F8FC1A8C2101FB075195F834CABD
:10A43000D1F8D8050668BCF1000F18D1D1F8500644
:10A44000B1F8DCC5016821F001010160B18989B270
:10A4500021EA0C01B1812978B9B91F2B60D9A3F188
:10A46000200120238B40D36003B0BDE8F08F00694A
:10A47000016821F001010160B18921F480710904B2
:10A48000090CB18129780029E7D04FF08C0808FB2E
:10A4900007F805EB08030193D3F850A6DFF8A0B046
:10A4A000504648F02BF9019B012283F82426D5F869
:10A4B000043B08F11809D944002B38D033889BB2EB
:10A4C00043F08003338008F174084FF0FF330BEB47
:10A4D0000801F362304648F047FB8C2303FB075723
:10A4E000494600235046C7F8F43546F007FDD7F833
:10A4F000503616225A601A6842F001021A60D7F8E4
:10A50000D825B7F8DC35126891890B439BB293814B
:10A510000949237D49682268C5F8001B1F2B9ED876
:10A52000202101FA03F3936003B0BDE8F08FFFF739
:10A5300011FFC5F8040BC1E7001000E00400001093
:10A54000D40500102DE9F843FFF704FF204F214EFA
:10A550007C6805464FF00008002C2DDD00231A46CC
:10A5600007EB0321013391F8F9109C4242EA010202
:10A57000F6D142EA08095FFA89F990467368C3F395
:10A580000803B3B9EFF311839BB9FDF739FD401B05
:10A59000B0F5FA6F02DCB8F1000FDDD1B9F1000FB0
:10A5A00004D00D4B93F85628542A09D04846BDE8EC
:10A5B000F883FFF7A7FEEAE7C1464FF00008DDE7A2
:10A5C000B3F85C280132A3F85C284846BDE8F8835C
:10A5D0000400001000ED00E0C0190020AD4B1B7816
:10A5E0000BB9012070472DE9F04FDFF8BCB2AA4942
:10A5F000DBF80020A94BA1FB02125209A3FB0213B6
:10A60000DB08A44987B003EB8303A2EB430391F873
:10A61000C825049201F60834DAB2059204EB8307E8
:10A62000002201F6E853019301F5816A9046049BEC
:10A63000984500F00D81DAF81820DAF80490D2F885
:10A64000E830D2F8EC600293FFF784FE029B03909F
:10A650004FEA890C9BF856989BF868080CF1085C47
:10A6600006F180610CEB431C3939B9F1540F0CEB46
:10A6700081110CEB801301D1ABF85E08994240F2D6
:10A680007D811A68002A00F071811A6C002A00F09E
:10A690008381D3F88020002A00F08081D3F8C02085
:10A6A00003F58073002AE9D1A3EB0C0C99424FEA21
:10A6B000AC1240F26381B11A45294FF0000628BF61
:10A6C00045213046B64603EB81111D4616460DE086
:10A6D0001A6C002A40F0EA80D3F88020002A40F06B
:10A6E0001581D3F8C02003F580732AB9994206D9A1
:10A6F0001A68002AECD04033994200F2DB803246DF
:10A700007646112E40F23E81DEF1150100F13A81CC
:10A71000634B1D46D3F8CC309A4238BF2B46039D7D
:10A7200038BFC3F8CC20DBF86C38EA1A002A18DBF3
:10A7300003F5F42303F590739D4284BF2B46053344
:10A74000CBF86C38564B564AD3F8CC30052B86BF25
:10A75000053BDBB200238BF868384FF0FF33C2F8BB
:10A76000CC3031B100FA01F1C6F114060120B0403D
:10A7700008434C4EC0F3C43306EB8303D3F8BC1D2F
:10A7800000F01F0306EB8303D3F8BC2D42EA01322D
:10A79000C0F3441106EB8101C0F3842306EB83036D
:10A7A000D1F8BC1DD3F8BC3D42EA011141EA0321B6
:10A7B00081EA112383EA131303F00F02354BD3F818
:10A7C000F03D0F2A03F1010340F0BD80B1F5803F59
:10A7D00080F0B980B9F1540F4FEA111140D02D4AE1
:10A7E000B1F5606FC2F8F03D45D0019B998194F8B6
:10A7F0005830059883420CD0BA6823689B1A2360AE
:10A800003A6B63689B1A63600023BB603B6384F808
:10A810005800236801332360BB680133BB604FF6E7
:10A82000FF73994205D16368013363603B6B013369
:10A830003B63019B08F101081433B8F1080F04F1E0
:10A840005C0407F15C0701930AF1200A7FF4EFAE84
:10A85000104A0123012082F8EC3E07B0BDE8F08FDA
:10A86000BBF858280132ABF858280A4AB1F5606F96
:10A87000C2F8F03DB9D19BF88E3003EB43030BEBEC
:10A88000C303434493F89D300D2BAED1019A80232E
:10A890009377ACE7040000101F85EB51CDCCCCCCF6
:10A8A000880100205CDC0508C01900208033994233
:10A8B0007FF625AFA3EB050C3C4A4FEAAC1C0CF12C
:10A8C000010C82FB0C52A2EBEC72012AB8BF0122F0
:10A8D00090404FF0010C9644013A0CFA02F21043FA
:10A8E0009C46DCF800209AB1DCF84020002A57D0C2
:10A8F000DCF88020002A56D0DCF8C0200CF5807CE3
:10A9000042B16145EDD81D466346EFE6C033F3E63C
:10A910000CF1400C6145F6D9ACEB03029211234BCC
:10A92000013283FB0253A3EBE273012BB8BF012377
:10A9300098409E440122013B02FA03F31843634608
:10A940001D466346D2E6B9F1540F04D1BBF858282E
:10A950000132ABF85828164AC2F8F03DD2F8EC3D67
:10A960000133C2F8EC3D4FF6FF7140E74033A3EBF3
:10A970000C0C99424FEAAC123FF69DAE10B1013873
:10A980008BF86808B9F1540F7FF453AFBBF85A380D
:10A990000133ABF85A384CE7803385E6C03383E6A1
:10A9A0000CF1800CB6E70CF1C00CB3E756555555C9
:10A9B00004000010F8B51D4B93F88D2093F88E30ED
:10A9C0009A422ED11A4F7D68002D11DD38460024A1
:10A9D00010F8086B16B1037E012B1CD002691368B6
:10A9E000013443F00103A54200F580701360F1D1FA
:10A9F000FFF7B0FCD7F8F04E002C0BDD0D4A02EB50
:10AA0000C404116893888889083203439BB2944236
:10AA10008B81F6D1F8BD002380F8F030FDF7C8FE39
:10AA2000DCE750F055FB0028CCD1F8BDC019002060
:10AA300004000010F80E00102DE9F8430546FFF75A
:10AA400089FC244E244B044610274FF0E02C4FF491
:10AA50007A7E4FF001087268C2F30802CAB9EFF3B8
:10AA60001182B2B91A68DCF8180019688A42F9D163
:10AA700059688842F6D8D3F808900EFB09F1091AF4
:10AA8000B1FBF9F10EFB0212121BAA42E3D3BDE89F
:10AA9000F883EFF3118287F31288DCF81800DCF8F2
:10AAA0001010C90344BFC3F80887DCF81800D3F8B6
:10AAB0000090D3F80817D2B282F311884944D3F832
:10AAC00008900EFB09F2121AB2FBF9F20EFB0122FA
:10AAD000DAE700BF00ED00E0C01900202DE9F047E3
:10AAE0003A4B3B4D471E10264FF0E0204FF47A7C46
:10AAF0004FF001086A68C2F30802002A52D1EFF34E
:10AB00001182002A4ED11A68846919688A42FAD1E2
:10AB100059688C42F7D899680CFB01FEAEEB040E25
:10AB2000BEFBF1FE0CFB02EE6A68C2F30802E2B95A
:10AB3000EFF31182CAB91A68846919688A42FAD196
:10AB400059688C42F7D8D3F808900CFB09F1091B1F
:10AB5000B1FBF9F10CFB0212A2EB0E02B2F57A7F07
:10AB6000E2D3013FC6D2BDE8F087EFF3118286F34E
:10AB7000128884690169C90344BFC3F808878469DE
:10AB8000D3F800A0D3F80817D2B282F31188D3F813
:10AB9000089051440CFB09F2121BB2FBF9F20CFBBA
:10ABA0000122D9E7EFF3118186F3128884690269E3
:10ABB000D20344BFC3F808878469D3F800E0D3F810
:10ABC0000827C9B281F311887244A4E7C019002094
:10ABD00000ED00E030B50C4683B00546D8B10368FF
:10ABE00003F13F4303F57E039B0A0C4A134493F899
:10ABF000A4044DF033FBC4F34112C4F30013CDE9B8
:10AC00000032C4F38103A988286804F003024FF0DE
:10AC10005BFD03B030BD4FF0FF33E6E75CDC0508B9
:10AC200000B1D7E7704700BF70B50E4C94F8C86507
:10AC3000B6B104F58164002504E00135B54204F1A4
:10AC400020040DD0237F002BF7D0E0680028F4D03B
:10AC5000217D0135FFF7BEFFB54204F12004F1D19B
:10AC6000012070BD0400001070B5002486B0CDE94D
:10AC70000144CDE903440DF1040CC0E93D44C0E9B1
:10AC80003F44C0F80441054600F5847EBCE80F004F
:10AC9000AEE80F00CEF8004095F82131059444F25B
:10ACA0003B36A5F84C610BB906B070BD1C09013CE0
:10ACB000052C03F00F032BD81A4E06EB4402B2F812
:10ACC000F40340FA03F2D20722D5012202FA03F379
:10ACD000013B2644184052F019FE96F83C2E124BC8
:10ACE000024403EBC20429462623104DE38020468C
:10ACF00041F80C5F4EF0C6FF0D49A2880868B2FA11
:10AD000082F24FF00043D34003430B6006B070BDA6
:10AD10002946064B41F80C3F002006B0BDE87040C4
:10AD20004EF0B0BF5CDC0508B81A002001B1000885
:10AD3000003C014048B182880449B2FA82F20868B6
:10AD40004FF00043D34003430B607047003C014089
:10AD500038B50409013C052C1AD80F4D05EB440207
:10AD600000F00F03B2F8F40340FA03F212F001020C
:10AD700010D0012202FA03F3013B1840254452F09F
:10AD8000C5FD95F83C3E054A034402EBC30038BDBF
:10AD9000002038BD104638BD5CDC0508B81A00201C
:10ADA00008B51AF03DFC052807D8054BD3F87038D4
:10ADB0000344187BBDE80840CAE7002008BD00BF77
:10ADC000C019002008B51D20FFF7C2FF10B190F98F
:10ADD000063053B11E20FFF7BBFF10B190F90630CB
:10ADE00003B108BD5523C38008BD5523C380F1E7D7
:10ADF000F8B5037D856902681F2B04464BD950685E
:10AE0000203B20219940084237D0D1601021994041
:10AE1000D1605168D940CE077FD4EFF3118350221F
:10AE200082F312882A6C1168C90757D4516889B215
:10AE300091B9D5E9096086424DD0AF699CBF0E46F5
:10AE40002969074494BF081A301A80B20021D760DC
:10AE5000AE6285F864105060116841F00101DBB208
:10AE6000116083F3118895F86430002B3DD1237D68
:10AE700022681F2B194614D9203B5068082199409D
:10AE8000084200D0D1605068042101FA03F318424F
:10AE900000D0D360F8BD16682020984006420DD13E
:10AEA0001946106808238B40184200D09360106840
:10AEB00004238B401842EDD09360F8BD10219940D7
:10AEC000906091601168D940C807A6D5012101FAA8
:10AED00003F39360A1E7012285F86420DBB283F3DA
:10AEE000118895F86430002BC1D095F87230002B92
:10AEF000BDD195F87100FFF72BFF2A6E938923F0DF
:10AF000008031B0401211B0C938185F87210002893
:10AF1000ADD02021FFF75EFEA9E7012101FA03F37E
:10AF2000D3607AE708B54AF01DFA1B20FFF710FF3F
:10AF300008B12923C3801C20FFF70AFF08B1292389
:10AF4000C3800A4B93F87928012A01D0012008BD5B
:10AF50000748C3F87C0800F120014C304FF00EFC8C
:10AF6000044B002083F8230008BD00BFC019002057
:10AF70005802002000ED00E043680B4A23F04073C4
:10AF800023F4807343F48073436083681A4042F073
:10AF900002028260C36A0139C9B223F4700343EA32
:10AFA0000153C362704700BFFDF7FFC0704700BF89
:10AFB0000020FDF753B800BF0120FDF74FB800BFD8
:10AFC0000220FDF74BB800BF10B1036882881A83D6
:10AFD000704700BF10B1036882885A83704700BF72
:10AFE000F0B5056890F888606B688488012285F860
:10AFF00024201A8822F040021204120C1A802A8996
:10B00000A24255D1017BAA7A8A420BD01A8822F03B
:10B0100003021204120C1A801A8892B2002944D03A
:10B020001A80A9721A882F7B92B242F040021A80CD
:10B030002B6A9A6892B34FF0000C2F4C1433E646FB
:10B0400053F8101C964401EA040221B1B2F1805F6A
:10B0500027D06A692AB353F8142C143302EA040186
:10B0600012B1B1F1805F1CD053F80C2C0CF1010C23
:10B07000002AE5D1AFB1A6B1BCF1010F0AD8BEF1EB
:10B08000070F07D80CEB8C0C4FEA8C022B6A134489
:10B090001B7B33B9BDE8F04045F05EBF0FB1002E19
:10B0A000F4D1BDE8F04046F0D5B942F00302B7E76D
:10B0B0001A88124922F0380212048B424FEA1242D7
:10B0C00017D001F580618B4213D02146B1F5807F06
:10B0D000A8BF4FF480710229B8BF022191FAA1F1F3
:10B0E000B1FA81F1013942EAC10292B21A802C818F
:10B0F00088E76108EAE700BF0000FFFF0038004072
:10B1000038B52C4AD0F8E0305268D0F8D810044650
:10B1100073B1501A83420BDC94F8D030C4F8D820B5
:10B12000012B10D0D4F8D4300133C4F8D43038BD5A
:10B13000D4F8E430C4F8D8200B44C4F8DC3094F8D8
:10B14000D030012BEED16168201D04F1E805EFF34A
:10B15000118C102383F3128863681B6A0BB3D4F835
:10B16000F0302A461BB1D3691432002BFBD10B6A95
:10B170006BB1996839B9934209D0196829B15B68F4
:10B1800099680029F7D01433F3E7C3E900055FFAA3
:10B190008CFC8CF31188D4F8D4300133C4F8D4304B
:10B1A00038BD0D625FFA8CFC8CF31188FFF718FF35
:10B1B000B8E700BF001000E02DE9F041826992F885
:10B1C000DC30012B8AB005464CD0023B012B54D811
:10B1D00092F84C31D2F89C202E4C63F07F03137010
:10B1E0008769D7F8A030D7F8108003F1010E0FCC93
:10B1F000EC46ACE80F00D7F89C30CDE9003E0FCC10
:10B20000ACE80F0094E8030007F110068CE8030097
:10B21000EFF31180102383F312883B691B6A002B24
:10B220002FD0029B6A461BB1D3691432002BFBD18D
:10B23000D8F8203073B1996839B99A420AD01968A0
:10B2400029B15B6899680029F7D01433F3E71E60D1
:10B25000C3F804D0C0B280F31188AA6911690B6ADF
:10B26000002BFCD1D2F8A0305A8852BAEA819A88D1
:10B2700052BA2A82DB885BBA6B8201200AB0BDE831
:10B28000F081C8F820D0C0B280F311883046FFF7B3
:10B29000A7FEE2E7A0EA05082DE9F04190F8DC30CE
:10B2A000D0F8A050012B8AB0044673D041D9023B9C
:10B2B000012B6BD890F84D31D0F89C205E4E63F096
:10B2C0007F031370D0F8A030D0F8108003F1010E86
:10B2D00000F110070FCEEC46ACE80F00D4F89C301C
:10B2E000CDE9003E0FCEACE80F0096E803008CE8F5
:10B2F0000300EFF31180102383F3128823691B6A84
:10B30000002B00F08F80029B6A461BB1D369143278
:10B31000002BFBD1D8F820302BB3996839B9934270
:10B3200021D01968E1B15B6899680029F7D014331E
:10B33000F3E7D0F89C304FF0FF321A605A609A6001
:10B34000DA60D0F8E0300522B3F57A7FC0F8F0205B
:10B350003BD8032380F8DC3001200AB0BDE8F0813F
:10B360001F60C3F804D0C0B280F311882269136A49
:10B37000002BFCD16B885BBAA4F8D030AB885BBAE9
:10B38000A4F8D230EB885BBAA4F8D43001200AB01C
:10B39000BDE8F08190F84C2190F84D319B1A5B107C
:10B3A0000133DBB205EB430235F813305BBAA0F88A
:10B3B000D03053885BBAA0F8D23093885BBAA0F83B
:10B3C000D43001200AB0BDE8F08103691A7B2AB3AA
:10B3D0005B691BB390F8983003B390F84C31D0F808
:10B3E0009C20C4F8A40063F07F03137090F84C1104
:10B3F00090F84D31D0F8A0201048C4F804015B1A31
:10B4000007330121C4F8FC30D4F89C3084F80011D3
:10B410000A44C4E93D3284F8DC10B7E7022384F81B
:10B42000DC30B3E7C8F820D0C0B280F311883846CA
:10B43000FFF7D6FD9AE700BFA0EA050839800008AB
:10B44000D3B2012B1DD8104B02EB420210B54FEACC
:10B45000820E0EF1080403F5137C02E01C336345F1
:10B460000DD01A788242F9D15A788A42F6D11A5907
:10B47000002AF3D00EF1040E03EB0E0010BD0020E5
:10B4800010BD0020704700BFC8EA050810B40C4C7E
:10B49000002304F5086C01E0152B0CD003EB4302EC
:10B4A00001331CF802108142F6D1144494F9820849
:10B4B0005DF8044B70474FF0FF305DF8044B704768
:10B4C000C0190020D3B2022B22D870B502EB420281
:10B4D000104C4FEA820E23460EF10C05002204E0C8
:10B4E0000132172A03F12C0310D01E68B042F7D1A5
:10B4F00093F804C08C45F3D15E59002EF0D02C2176
:10B500000EF1080301FB0233E01870BD002070BD8E
:10B51000002070475CDC0508002839D030B51D4D8F
:10B5200090F804C0002305F5086401E0152B2DD028
:10B5300003EB43020133A15C6145F7D11544046874
:10B5400095F9823890F805E0DAB2022A1ED803EBAA
:10B55000430311484FEA830C0CF10C05034600220B
:10B5600004E00132172A03F12C030FD019688C4232
:10B57000F7D119797145F4D159590029F1D02C210D
:10B580000CF1080301FB0233184430BD002030BD2C
:10B59000704700BFC01900205CDC05080348D0F8E4
:10B5A000483113B100F59C7018477047880100209E
:10B5B0000348D0F86C3113B100F5AE7018477047EE
:10B5C000880100200348D0F8903113B100F5C07015
:10B5D00018477047880100200348D0F8B43113B1F0
:10B5E00000F5D27018477047880100200348D0F852
:10B5F000D83113B100F5E470184770478801002076
:10B600000348D0F8FC3113B100F5F67018477047C5
:10B61000880100200348D0F8203213B100F50470EF
:10B6200018477047880100200348D0F8443213B10E
:10B6300000F50D7018477047880100200348D0F8C6
:10B64000683213B100F51670184770478801002062
:10B650000348D0F88C3213B100F51F7018477047BB
:10B66000880100200348D0F8B03213B100F52870EB
:10B6700018477047880100200348D0F8D43213B12E
:10B6800000F5317018477047880100200348D0F852
:10B69000F83213B100F53A7018477047880100205E
:10B6A0000348D0F81C3313B100F5437018477047B6
:10B6B000880100200348D0F8403313B100F54C70E6
:10B6C00018477047880100200348D0F8643313B14D
:10B6D00000F555701847704788010020094B0A4A49
:10B6E000013800EBC00003EB80030848D3F8383181
:10B6F000116B834214BF4FF480034FF400130B43CC
:10B700001363704788010020003802400060024047
:10B71000F0B401383B4C3C4E3C4D00EBC00C04EB0C
:10B720008C0CDCF83871AF4214BF4FF480054FF435
:10B730000015376B3D433563354DCCF85031DCF89F
:10B740003C31CCF84811AB424FEAC0013FD005F57F
:10B750008065AB423BD0A5F57A75AB4246D005F586
:10B760008065AB4242D0A5F57A75AB4240D005F575
:10B770008065AB423CD0A5F57A75AB4234D005F577
:10B780008065AB4230D0A5F57A75AB4232D005F575
:10B790008065AB422ED0A5F57A75AB422CD005F56D
:10B7A0008065AB4228D0A5F57A75AB4226D005F569
:10B7B0008065AB4222D0A5F57A75AB4220D0154DFD
:10B7C00006F532563836B34218BF002500E0124D58
:10B7D0000B1804EB8304C2F3871194F84D01C4F8ED
:10B7E0005851F0BC4EF030BA0C4DF1E70C4DEFE77C
:10B7F0000C4DEDE70C4DEBE70C4DE9E70C4DE7E7A1
:10B80000044DE5E788010020003802400060024056
:10B810001060024000800028208000100080001886
:10B820000088001000802010208000200088002068
:10B83000008020202DE9F04F934A92F8D138012B57
:10B8400085B021D0022B15D0002300938F4F4FF0ED
:10B85000000807F1780A3B78022B17D008F101089D
:10B86000B8F1030F07F128070AF1050AF3D105B073
:10B87000BDE8F08F92F8C63833B192F8C238083B71
:10B8800018BF01230093E1E70093DFE79AF9033043
:10B890007F4D0297591C15BFDBB200239B464FF02A
:10B8A000010B1E46DAB2012A00F2DB8006EB4601EC
:10B8B00089007300774C019308315FFA88F703E041
:10B8C0001C34AC4200F0CD802378002BF8D1637893
:10B8D000BB42F5D160580028F2D00EF019F8009B59
:10B8E000814623B1A0F10901072940F2BF807A1CEB
:10B8F000D2B2142148460DF0F7FF002800F0B180C5
:10B90000DDE90137334404EB830409F1FF33E068D8
:10B91000614C594203EBC30201F0070103F0070336
:10B9200058BF4B4204EB820104F59C7404EB820285
:10B93000C1F844013A61484681F84031FFF7CEFE34
:10B940009AF904305A1C00F09A80DEB23246CDE9F2
:10B9500002974F4DF3B29346012B62D806EB460196
:10B96000890073004B4C019308315FFA88F902E0BB
:10B970001C34AC4255D02378012BF9D163784B4568
:10B98000F6D160580028F3D00DF0C2FF009B0746A7
:10B990001BB1A0F10901072947D909F10102D2B26F
:10B9A000132138460DF0A0FF00283AD0019ADDF8A7
:10B9B00008903244BB4604EB82040BF1FF32514243
:10B9C000E068354C039F02EBC20501F0070102F06D
:10B9D000070258BF4A4204EB850104F59C7404EB4E
:10B9E0008505C1F844017D61584681F84021FFF783
:10B9F00075FEB9F1000F3DD0BBF1000F1BD02846FA
:10BA0000FCF740FD3869FCF73DFD3846FCF70AFDC0
:10BA100000231A4621495846FFF77AFE01233B735B
:10BA20001CE70136F3B29B4596D2DDE90297B9F1E6
:10BA3000000F1FD01A4C09F1FF33242202FB0340F0
:10BA4000002438617C61FCF71DFD3846FCF7EAFCF8
:10BA50002346144922464846FFF75AFE01233B730A
:10BA6000FCE60136F2B25A457FF61DAF029F4FF059
:10BA7000000965E700220023C7E90423EEE601235D
:10BA80001A46002663E700BFC0190020A822002044
:10BA900014ED0508C8EA050888010020ED9B0008A0
:10BAA000C0020020659C0008800AA0F58010522882
:10BAB00008D8054B034493F800340D2B02D8034AF1
:10BAC000D0567047002070475CDC0508F05B060824
:10BAD000064A136851690B4003F00103536123B117
:10BAE000034BD3F80C07036818477047003C01402C
:10BAF000C0190020064A136851690B4003F0020385
:10BB0000536123B1034BD3F81007036818477047FC
:10BB1000003C0140C0190020064A136851690B40DF
:10BB200003F00403536123B1034BD3F814070368F4
:10BB300018477047003C0140C0190020064A1368AE
:10BB400051690B4003F00803536123B1034BD3F851
:10BB50001807036818477047003C0140C0190020CF
:10BB6000064A136851690B4003F01003536123B177
:10BB7000034BD3F81C07036818477047003C01408B
:10BB8000C0190020F8B50C4B1D685A69154005F422
:10BB900078755D617DB1094F0126B5FA85F4C4F170
:10BBA0001F0407EB840306FA04F4D3F80C070368B8
:10BBB0009847A543F1D1F8BD003C0140C0190020D1
:10BBC000F8B50C4B1D685A69154005F47C455D615C
:10BBD0007DB1094F0126B5FA85F4C4F11F0407EBC6
:10BBE000840306FA04F4D3F80C0703689847A543C6
:10BBF000F1D1F8BD003C0140C0190020F0B5054668
:10BC000083B0A0B307681D4B144607F13F4202F50D
:10BC10007E0203EB92230E4693F8A4044CF01EFB25
:10BC2000A988B1FA81F3C3F11F03C3F3CC0207EB78
:10BC3000820203F00703156A4FF00F0C9B009C4033
:10BC40000CFA03F325EA03031362136A1C4314621C
:10BC5000C6F30013C6F34112CDE900323846C6F3ED
:10BC6000810306F003024EF02FFD03B0F0BD034B3D
:10BC700093F8A3044CF0F2FA2B68FFDE5CDC0508B5
:10BC800000B1BBE7704700BF2DE9F047684E06EBF7
:10BC90000013D3F87049002C76D093F878790546D4
:10BCA0004FEA001838464CF0D9FA07F01F027F0916
:10BCB0000123032F03FA02F372D0042F6BD0022F5B
:10BCC00064D006EB0803013593F87409FFF740F8D8
:10BCD000EDB2824610B11223C571837106EB0803E1
:10BCE00093F87509FFF734F8814610B11323C57135
:10BCF000837106EB080393F87609FFF729F80746E6
:10BD000010B11423C571837106EB0803504693F8F4
:10BD100077594A212A46FFF7B3FF2A4648462A2187
:10BD2000FFF7AEFF2A460A213846FFF7A9FF414B2D
:10BD30009C423AD0404B9C4242D0404B9C424AD01D
:10BD40003F4B9C4252D03F4B9C425AD03E4B9C4270
:10BD500062D0A38823F003031B041B0CA380238859
:10BD600003F4415343F4457343F003032380A38B4F
:10BD700023F400631B041B0C0722A3832282238865
:10BD80009BB243F040032380BDE8F0872F4A516AFD
:10BD90000B43536295E72D4A11690B43136190E7FA
:10BDA0002A4A116A0B4313628BE703F584335A6AFC
:10BDB00042F480525A625A6A22F480525A62C8E7A8
:10BDC00003F500331A6A42F480421A621A6A22F4B6
:10BDD00080421A62BDE703F5FE331A6A42F400425C
:10BDE0001A621A6A22F400421A62B2E703F5823339
:10BDF0005A6A42F400525A625A6A22F400525A6253
:10BE0000A7E703F568435A6A42F480125A625A6AF5
:10BE100022F480125A629CE703F564435A6A42F4A2
:10BE200000125A625A6A22F400125A6291E700BF65
:10BE3000C01900200030014000380040003C0040A4
:10BE400000340140005001400054014000380240DD
:10BE5000431C00F02C812DE9F04FDFF8488300EB04
:10BE6000800308EBC30387B0D3F80C90820005462B
:10BE70000192B9F1000F04D05C692CB194F906303D
:10BE800013B107B0BDE8F08FAB002B4408EBC30340
:10BE9000D3F818A0BAF1000F03D09AF90630002B9E
:10BEA000EFD1AB002B44B84ED9F80470DB00183347
:10BEB000F0180022691CF250C9B2C0E90122C26028
:10BEC000002C00F081811523E171A37199F82800FD
:10BED000BAF1000F00F0688116238AF807108AF87B
:10BEE00006304CF0BBF9BB882268A08823F440736D
:10BEF0001B041B0CBB80DAF800301083BAF8042056
:10BF00001A8311212046FEF765FE11215046FEF7E7
:10BF100061FE09264FF0330B2CB9C2E0BBF1010BD7
:10BF200006D04DF035FE2268A18810690142F5D097
:10BF300051834DF0D1FD2368A2881A834DF0CCFDCA
:10BF4000013EE7D1002C00F0DC80332603E0013E07
:10BF500006D04DF01DFE2268A18813691942F6D063
:10BF600051834DF0B9FDBAF1000F00F0F280DAF81C
:10BF70000030BAF804205A834DF0AEFD2368A28841
:10BF80001A834DF0A9FDDAF80030BAF804201A83BC
:10BF90004DF0A2FD2368A2881B691A4240F08880F8
:10BFA000019B2B4408EBC303997F1A7F002940F0C3
:10BFB0008B8020461221FFF721FE1221019B2B448A
:10BFC00008EBC3035A7F5046FFF718FE6F4B9F42A2
:10BFD00000F012816E4B9F4200F019816D4B9F4221
:10BFE00000F02081019B2B4408EBC3034FF47A72CD
:10BFF0001C8CBB8823F440731B041B0CBB803B8848
:10C000009BB243F001033B80BD8802A802FB04F40D
:10C0100025F03F0546F026FB04995F4B2D04A3FB5A
:10C0200001232D0C45EA9345BD803A8822F0010298
:10C030001204120C3A80594A980C9442034649DC87
:10C040006200B1FBF2F292B20133042A38BF04223B
:10C050003B84BA833B889BB243F001033B803B881F
:10C0600023F4816323F002031B041B0C4FF4804272
:10C0700043F480633B803A813B8823F080031B04B8
:10C080001B0C3B8099F82A0000214DF0DDFD99F84A
:10C090002900002107B0BDE8F04F4DF0D5BD4DF0AF
:10C0A00077FDBBF1010BFAD14DF016FD46E7704765
:10C0B000019BDAF800202B4408EBC30312699A7F36
:10C0C000002A00F0BA801A7F32212046FFF796FD41
:10C0D000322173E704EB4404B1FBF4F18AB2C1F3FB
:10C0E0000B0109B942F001022D494FF4967300FB90
:10C0F00003F3A1FB03139B09013342F400423B8489
:10C10000A7E7332401E04DF043FD013CFBD14DF0A6
:10C11000E3FCBAF1000F00F09680DAF80030BAF8CC
:10C1200004205A834DF0D8FC4DF0D6FCDAF80030EC
:10C13000BAF804201A834DF0CFFC019B2B4408EB86
:10C14000C3039A7F002A18BF32215A7F08BF1221E9
:10C1500039E74DF0C1FC2368A2881A834DF0BCFC7E
:10C160004DF0BAFC2368A2881B691A4272D1019B68
:10C170002B4408EBC303997F1A7F002979D020460E
:10C180003221FFF73BFD21E7CC190020005400408D
:10C1900000580040005C004083DE1B43A086010085
:10C1A000D34D6210C01900204CF058F8BB88A2880B
:10C1B00023F440731B041B0CBB80236811211A83DA
:10C1C0002046FEF707FDA4E699F82800BAF1000F13
:10C1D00054D016238AF806308AF807104CF03EF83F
:10C1E000BB88BAF8042023F440731B041B0CBB80EB
:10C1F000DAF800301A8388E603F5F2331A6A42F45B
:10C2000000121A621A6A22F400121A62EAE603F5B0
:10C21000F0331A6A42F480021A621A6A22F4800227
:10C220001A62DFE603F5EE331A6A42F400021A627C
:10C230001A6A22F400021A62D4E61A7F20461221FA
:10C24000FFF7DCFCB9E64DF047FC4DF045FC4DF046
:10C2500043FCBBE6019B2B4408EBC30320469A7FBB
:10C26000002A18BF32211A7F08BF1221FFF7C6FC2F
:10C27000ACE620461221FFF7C1FCA7E64BF0EEFF2B
:10C28000BB8823F440731B041B0CBB8041E600BF3A
:10C290002DE9F8430746FEF735F8DFF84C8007EB49
:10C2A0008709044608EBC90542F20F7604E0FEF761
:10C2B00029F8001BB0420BDC95F82530002BF6D195
:10C2C00008EBC90898F8240080F00100BDE8F88365
:10C2D000B8F8A039013338469BB2A8F8A039FFF767
:10C2E000B7FD0020BDE8F883C0190020B0F1FF3F82
:10C2F0006DD02DE9F04F022883B0044614DC354E92
:10C30000984600EB800306EBC305DB00D5F810A0D0
:10C310000093BAF1000F07D0894695F8251093468F
:10C3200001F0FF02019219B1002003B0BDE8F08FC7
:10C33000FDF7E8FF009B019A203307464FEA4901C9
:10C3400006F10C00C9B200EB030C85F826104FF083
:10C35000010E0C9985F827B085F8292085F82AE088
:10C36000C150CCF8041085F8288085F825E085F8C0
:10C370002420BAF8043099051DD4BAF80030DA0543
:10C3800012D442F20F7504E0FDF7BCFFC31BAB42B1
:10C3900013DCBAF800309B05F6D4BAF800309BB233
:10C3A00043F48073AAF80030BAF804309BB243F427
:10C3B0004073AAF804300120B7E7B6F8A03901337A
:10C3C0009BB22046A6F8A039FFF742FDACE700205B
:10C3D000704700BFC0190020E0B5294E00EB800374
:10C3E00006EBC30384B0DA685568AA8A92B2039256
:10C3F000039A12F4706F1CBF012283F82420039B60
:10C4000013F4E06F4FEA80070DD1AB8A074423F4A1
:10C41000706306EBC7061B041B0C0022AB8286F878
:10C42000252004B0E0BD2B8BAB8823F480631B0474
:10C430001B0CAB80039B9A05E7D42B889B05E4D4A7
:10C440002B88D9050FD52B88DA05FCD42B889BB215
:10C4500043F400732B802B889B05FCD40190FFF7DD
:10C46000F7FC0198D1E72B889BB243F400732B8033
:10C47000AB8823F440731B041B0CAB80C5E700BFE3
:10C48000C01900200020A7E70120A5E70220A3E7AC
:10C4900070B590F871301C09013C052C0FD81A4E6C
:10C4A00006EB44020546B2F8F40303F00F0340FA2A
:10C4B00003F2D20703D595F87220012A01D001209A
:10C4C00070BD9A40013A1040264451F01FFA96F888
:10C4D0003C3E0E4A034402EBC30452F83320A388C7
:10C4E00010691840ECD0EB6E002285F8722093F8AA
:10C4F000212002212046FFF781FB2A6E93899BB2FF
:10C5000043F008039381DAE75CDC0508B81A0020E1
:10C51000F8B50E4C94F8C8759FB104F5BA64C7F12C
:10C5200009070925013D0ED0A6683079FEF710FCF9
:10C53000217DF27908B1FFF761FBAF4204F18C0471
:10C54000F0D10120F8BDAB68FFDE00BF0400001091
:10C55000094BD3F8A429D3F8A81940F22A400023A4
:10C5600050604B620B889BB243F001030B80136851
:10C5700043F0010313607047C019002010B41D4B35
:10C580001D48196C1D4A41F08051012485B0196481
:10C5900004625321FF24CA205462506251625B6FCF
:10C5A000DB0017D416480423002102910290029A5E
:10C5B0001A440292029A04331C2B1160F5D10391A4
:10C5C0000390039B0393039B0E4A1A6005B05DF82A
:10C5D000044B70470A4B002201920193019B019387
:10C5E000019A084B12689A42DCD105B05DF8044B01
:10C5F000704700BF0038024000000E420028004093
:10C6000050280040316665422DE9F041046ED0F8B3
:10C610000880A38923F400531B0407461B0C90B029
:10C62000A38143793D79C3F38000190305F0010626
:10C630001B0215F002054FEA00304FEA860203F4B0
:10C64000806318BF42F0080203431A43238A9BB257
:10C6500001F4005123F440530B432382A38923F4B4
:10C66000B05323F00C031B041B0C1A43A281A38AB2
:10C6700023F440731B041B0CA38201A845F0F2FFB6
:10C680006B4B9C4205D003F580639C4201D0039B19
:10C6900000E0049BA2896749A089120403EB83038D
:10C6A0004CBF4FEA48084FEA880803EB8303B3FB0B
:10C6B000F8F3A1FB03C252094FF0640C00040CFB19
:10C6C00012334FEA021200F19A801B013233A1FBB0
:10C6D0000313C3F3431313439BB2238197F9380029
:10C6E00097F80580FEF75CFB30B10368828818F08C
:10C6F000010F14BF1A835A8318F0080FA38A78D049
:10C700009BB243F00803A382A3899BB243F4005376
:10C71000A381002E2FD0FE6B002E7DD00023CDE90B
:10C720000833CDE90C33CDE90E33049306937B6CCB
:10C730000193FB6D0293FB6805937B6903934FF4B0
:10C7400080714FF48033CDE90A1330464FF4806393
:10C75000079345F0D3FF01A9304644F0CFFB33687F
:10C7600043F001033360A38A9BB243F04003A382EA
:10C7700073689BB27B65002D33D03E6C002E46D093
:10C78000BB6C0193BB6D02933B69059340230493FB
:10C790004FF48033002530460B934FF480630793AA
:10C7A000CDE90855CDE90C55CDE90E550395069513
:10C7B0000A9545F0A3FF01A9304644F09FFB736939
:10C7C00043F080037361336843F016033360756090
:10C7D000A38A9BB243F08003A382E36843F0400343
:10C7E000E360A3899BB243F40053A38110B0BDE87A
:10C7F000F08123F008031B041B0CA38284E7DB00F9
:10C800003233A1FB0313C3F34213134364E7E3681A
:10C8100043F08003E360E0E74FF6DF732380E368D3
:10C8200043F02003E360E36843F01003E360A2E712
:10C83000001001401F85EB51BFF34F8F0549064B98
:10C84000CA6802F4E0621343CB60BFF34F8F00BFAE
:10C85000FDE700BF00ED00E00400FA0508B5002187
:10C86000032043F0C7F972B6FFF7E6FF154C08B591
:10C87000D4F8AC3994F8B209ABB91420FEF72EF90C
:10C8800000BFD4F8AC395BB11A689B88116994F881
:10C89000B2290B4012B91BB1FFF7E0FF002BFBD010
:10C8A000FCF710FEECE719689A880B69134020B179
:10C8B000002BE2D10B691340FAE7002BDDD00B69A6
:10C8C0001340FAE7C019002008B572B6FFF7B4FFAD
:10C8D00000B583B00D49002200920091009B0C33FB
:10C8E0000093009B1B68012B02D003B05DF804FB92
:10C8F00001920191019B06490C330193019B1A603F
:10C900000B6883F308884B689847FEE7502800407F
:10C910000000FF1F38B5FFF731FEFFF7D9FF0120F8
:10C9200045F0D6FF6D4A936823F003039360936844
:10C9300013F00C0FFBD113686849A0B943F0010351
:10C94000136041F2883302E0013B00F0C5800A68C1
:10C950009507F9D5624C00220823C4F8B429C4F81D
:10C96000B83902251EE043F48033136041F2883366
:10C9700002E0013B00F0B0800A689403F9D5584CFE
:10C98000584B594DB0FBF5F5B0FBF3F0B5EB400F4C
:10C9900018BF28464FF48003C4F8B439C4F8B80966
:10C9A000B5FBF0F50220C4F8BC5945F091FF03280F
:10C9B0000DD84E4B03EBC0039988DA88C4F8C4192C
:10C9C0005B88C4F8C829B3FBF5F3C4F8C039434BFE
:10C9D00047491A6C42F080521A640A6842F4404295
:10C9E0000A609A689A609A6842F400429A609A686B
:10C9F00042F4A0529A60D4F8B419D4F8B8290A4382
:10CA0000D4F8C01942EA8112D4F8C81942EA016286
:10CA1000D4F8C4194908013942EA01425A601A6837
:10CA200042F080721A601A689201FCD5314A40F2D5
:10CA300005711160996821F003019960996841F0CE
:10CA40000201A2F580629960936803F00C03082B41
:10CA5000FAD12949D823B3FBF5F39B0143F00053E6
:10CA60000120C2F884308866FBF7A8FF234D1B4BDA
:10CA7000234AEA60234A596FAA605A6B224922F07E
:10CA800080025A635A6F42F080725A671A6B42F4FE
:10CA9000CE021A635A6B5A639A6B9A631A6C0A43F2
:10CAA0001A64596C194A0A435A64FCF765FD184A1E
:10CAB000D4F8F430A2FB03239B09013BB3F1807F40
:10CAC00009D24FF0E022F02053610021072385F8BE
:10CAD00023009161136138BD014CC7E70038024063
:10CAE000C019002080841E0040420F0014ED05088C
:10CAF00000700040003C02400000474200ED00E0B2
:10CB00000005FA0500000020FFC9FE36335F07006C
:10CB1000D34D62100C4B0D49DB68DB43C3F302239A
:10CB2000C3F104030122DBB202FA03F301EB000CB0
:10CB30001B0103F0F0038CF80033430900F01F00E1
:10CB4000824041F82320704700ED00E000E100E062
:10CB500030B5154C154D85B00139002389B2A0427E
:10CB6000ADF80C30ADF806308DF80E300291D5F8E6
:10CB7000F4300FD00E4988420CD001F58041884234
:10CB800008D001F58061884204D001F580618842B7
:10CB900018BF5B08B3FBF2F301A9013BADF8043009
:10CBA00045F08AFF05B030BD00040140C0190020E7
:10CBB0000000014001490248FCF798BEB81D002062
:10CBC0000000014010B5064C064804F57E71FCF7E4
:10CBD0008DFE04F284510448BDE81040FCF786BE87
:10CBE000C0190020000001400044014002494FF0FC
:10CBF0008040FCF77BBE00BFE41D002001490248D5
:10CC0000FCF774BE101E00200004004001490248D9
:10CC1000FCF76CBE3C1E00200008004001490248A1
:10CC2000FCF764BE681E0020000C00400149024869
:10CC3000FCF75CBEEC1E00200004014010B5064C61
:10CC4000064804F22C51FCF751FE04F5C16104487A
:10CC5000BDE81040FCF74ABEC019002000040140A6
:10CC6000001C004001490248FCF740BE181F00208C
:10CC70000040014001490248FCF738BE701F002007
:10CC80000048014001490248FCF730BE9C1F0020CB
:10CC90000018004001490248FCF728BEF41F00209C
:10CCA0000020004010B50C2935D8DFE801F09134A0
:10CCB000343463343434073434343500038C5488CA
:10CCC000B2F80CE023F480731B041B0C0384038C68
:10CCD000B0F804C0818B21F073014EEA040E090400
:10CCE000148823F40073090C1B042143764C1B0C9D
:10CCF00043EA0E23A0421FFA8CFC9BB200F0948002
:10CD000004F58064A04200F08F809268A0F804C00F
:10CD10008183C263038410BD038C5488B2F80CE095
:10CD200023F480531B041B0C0384038CB0F804C051
:10CD3000818B21F4E6414EEA040E0904148823F4A1
:10CD40000053090C41EA04211B045F4C1B0C43EA0D
:10CD50000E33A0421FFA8CFC9BB289B27ED004F540
:10CD60008064A0427AD09268A0F804C081830264F3
:10CD7000038410BD038C5488B2F80CE023F0100338
:10CD80001B041B0C0384038CB0F804C0018B21F43A
:10CD9000E6414EEA040E0904148823F02003090C2E
:10CDA00041EA04211B04484C1B0C43EA0E13A04229
:10CDB0001FFA8CFC9BB289B26CD004F58064A0424F
:10CDC00068D09268A0F804C001838263038410BD18
:10CDD000038C5488B2F80CE023F001031B041B0CF5
:10CDE0000384038CB0F804C0018B21F073014EEA78
:10CDF000040E0904148823F00203090C1B042143C8
:10CE0000314C1B0C43EA0E03A0421FFA8CFC9BB270
:10CE10002CD004F58064A04228D09268A0F804C009
:10CE200001834263038410BDD489B2F810E023F477
:10CE3000006343EA0423548A2CF4405C4EEA040E57
:10CE40004CEA0E1C94884FF6FF3E03EA0E0E4EEAA3
:10CE5000042E1FFA8CFC1FFA8EF356E7148A2CF46A
:10CE6000804C4CEA841C1FFA8CFC7CE7D489B2F815
:10CE700010E023F008032343548A2CF4407C4EEA4C
:10CE8000040E948823F004034CEA0E0C1FFA8CFC69
:10CE90002343C2E7D489B2F810E023F0800343EAC9
:10CEA0000413548A2CF4406C4EEA040E4CEA8E0CA7
:10CEB00094884FF6BF7E03EA0E0E4EEA041E1FFA58
:10CEC0008CFC1FFA8EF37CE7000001402DE9F04F47
:10CED000B14BDFF8DC8293F8D2E8B04CB04D93B0A0
:10CEE0000EF1FF37FBB200930023CDE9013EC246AD
:10CEF000DFF8C0B2DBF80070BB0AA3F58013522B39
:10CF000000F20B81234493F800340D2B00F20581CD
:10CF100015F90390029B012B00F00681029B022B66
:10CF200002D1B9F1080F33D10026314648460DF041
:10CF300065FE0DF0EFFE90F9003013B1542B40F078
:10CF4000EB820436B6B2102EEFD1019B0021002BEC
:10CF500000F0A38042460CE0234493F800340D2BEC
:10CF60000ED8EB564B450ED002F58072524500F0BC
:10CF70009180906803689B0AA3F58013522BEBD92C
:10CF800000234B45F0D143799BF805009842EBD143
:10CF9000844B0BF11C0B9B45ACD1019B0133042B43
:10CFA00001930AF5807AA3D1DFF80C9299F8C8357D
:10CFB000013309F5816A04934FF0010B049B5B4533
:10CFC00065D0DAF80C30744A9AF8101092F8CC292F
:10CFD00001930291002B5AD01968D9F804009B885C
:10CFE000039101F13F4505F57E0500284FEA95259F
:10CFF000009340F3A780002303E00133834200F055
:10D000009E801C0258F80410A942F6D14444009AAC
:10D01000029B8AF81030B2FA82F6019BCAF80C30F3
:10D02000C6F11F054FF00301CAF80450CAF81840B2
:10D03000997183F807B0E16C606C6B0001220327E3
:10D040009F4002FA03F3194399F80030E164384332
:10D0500002FA05F56064276DD4F8A000A9B2002B90
:10D0600000F060823D432565039D009B2B83FBF709
:10D0700059FA20460BF1010BFBF79AFB40F2011322
:10D08000BBF1090FAAF81C300AF1200A96D113B09F
:10D09000BDE8F08F00297FF47BAF5846FBF708FA14
:10D0A000C3B2022B9BF805E000F2778200F1010C7D
:10D0B0003A4A0CEB4C0C4FEA8C0C02F57D7003E005
:10D0C0002C32904200F0698213689F42F8D11379A4
:10D0D0007345F5D152F80C30002BF1D0324842683C
:10D0E0009A424FF0000108D00131102900F12400CC
:10D0F0003FF44EAF42689A42F6D14B1CDBB22B4A4A
:10D10000013B03EBC30302EB830393F95431002B80
:10D110007FF43EAFCAF808B03FE7009B012B7FF6D3
:10D1200037AF4FF00009FFE6B9F1010F3FF4FCAE55
:10D130001C4B0BF11C0B9B457FF4DCAE2DE7042B45
:10D1400000F0FC8109EB00230102059119690691A9
:10D15000002900F016826C1C0792E4B24FF05402D2
:10D160009D6083F8042183F80541069B01305E79B8
:10D17000C9F8040018461D680896FBF799F9C3B270
:10D18000022B00F20A82471C07EB4707034B079A62
:10D19000BF000021B44617E0C01900205CDC050880
:10D1A000F05B060830EE0508C00200208801002070
:10D1B0000C00001034ED050804000010013117299F
:10D1C00003F12C0300F0E9811E68B542F6D11E7907
:10D1D0006645F3D1DE59002EF0D02C2300EB400041
:10D1E00001FB03F3BB49BC4F03EB80030B44384600
:10D1F0001969059B0A914B44C3E906614368B34230
:10D200004FF0000108D00131102900F124003FF453
:10D210003EAF4368B342F6D14B1CDBB2AF49013B92
:10D2200003EBC30301EB830393F9541100297FF44B
:10D230002EAF83F85541059CA948E11101EB24214B
:10D2400001EB011100EB810C0599CDF81CC08C2479
:10D25000091204FB01F100F54C7000EB4100059947
:10D26000099049440998C1F8F440039CCC605424C7
:10D27000C1F8F00083F854419A48C1F8A8C033239C
:10D28000C1F8AC30984B0599D3F8F430854208EBDF
:10D2900001040FD095498D420CD001F580418D429B
:10D2A00008D001F580618D4204D001F580618D4286
:10D2B00018BF5B08062A00F06181072A8C488D4A56
:10D2C0008D4918BF11468D4A18BF02460598B3FB19
:10D2D000F2F2B3FBF1F3013A09EB000192B2013B28
:10D2E000A1F8B030A1F8682000F154010023A4F89F
:10D2F0005C30284648F80130A265414445F0DCFB2B
:10D300000023ADF838302B8808999BB243F0800396
:10D310002B802B8823F001031B041B0C2B80784BE4
:10D320000D934FF0020E4FF48073CDE910E32846C1
:10D330000A230DAA0F93FFF7B5FC069B1879002866
:10D3400040F006812B889BB243F001032B80002321
:10D350007A68964203F1010300F0F780102B07F181
:10D360002407F5D14FF0FF3300205C4A6549664F32
:10D3700003EBC30302EB8303644AD3F838318B42D7
:10D3800014BF4FF480034FF40013116B0B4313636E
:10D39000089A0C2A9BBF5E4B03EB42030021B3F8B3
:10D3A000DC10059B4B449982002306E0954200F077
:10D3B000EF800133042B00F0ED8057F83320002A72
:10D3C000F4D1D9F8F02E0132C9F8F02E09EBC302DE
:10D3D000DB00C2F8F45E3B4400259A881143998033
:10D3E00090224C492346FEF793F93368059A039837
:10D3F00043F010033360079BE3660A9B636602F108
:10D40000640104234FF40032C4E923234023332270
:10D41000C4E91C3200F118024FF48067A2664FF491
:10D4200080504FF48042C4E9200241443046C4E9B0
:10D430002555A567C4F88850C4F89C50E76743F0A9
:10D440005DFD3068E0617069206270680A9B60620F
:10D45000B068A062F068C4F8AC300423C4F8D830D7
:10D46000099BE062C4F8B4300398059AC4F8C4700C
:10D470004FF44033C4F8D4308C23C4F8BC3000F1EE
:10D48000100302F1AC01C4F8B0304FF480424FF405
:10D490000063C4F8C830C4E937554144C4F8CC200F
:10D4A000C4F8B850C4F8C050C4F8D050C4F8E45020
:10D4B000304643F023FD3368236373696363736805
:10D4C000A363B368E363F3682364336843F0100332
:10D4D00033609CE55CDC0508C00200208801002068
:10D4E0009023002000040140C019002000000140EA
:10D4F000D0DD0600449508001055220040771B003F
:10D500006000010000600240F80E00100038024088
:10D5100054ED05086D850008019B0121002B7FF467
:10D5200019AD35E5C6F12F06B2403A432265039A9C
:10D53000009D55831A46FAF7F5FF9AE5184A03232A
:10D5400082F8CD3913B0BDE8F08FD8B2431E0CE796
:10D55000FDF7FEFB0B9038B1069B0221DA79FEF74E
:10D560004DFB0B9B5422DA80B5F844306FEA4343FD
:10D570006FEA53439BB2A5F84430E3E609490A4AEF
:10D58000A4E6074A022382F8CD3913B0BDE8F08F34
:10D59000DB0020E700239B88FFDE00235B68FFDEC3
:10D5A000C0190020882A1100A0BB0D000C2911D839
:10D5B000DFE801F0231010101910101011101010D6
:10D5C0000700838B23F400631B041B0C43EA022334
:10D5D0009BB283837047838B23F008031B041B0CCF
:10D5E0001A4382837047038B23F400631B041B0CD4
:10D5F00043EA02239BB203837047038B23F00803A3
:10D600001B041B0C1A430283704700BF2DE9F04F27
:10D61000DFF85CB39BF868709BB01FB900201BB0AB
:10D62000BDE8F08F00222F2138460DF0C7FB804661
:10D630000028F3D0DFF83C930568C9F8A859FDF736
:10D640006BFF0028EAD0D0E901430193C9F8A4494F
:10D65000002CE3D0BA4E0022314601E0102ADDD082
:10D660004868844201F1240102F10102F6D1D2B2EC
:10D67000DFF804A3013A02EBC2020AEB820292F93C
:10D6800054110029CAD138462F27A2F85471FDF74A
:10D690005FFBCBF86C0028B1C78098F807202A21DF
:10D6A000FEF7ACFAA74F002207F6345050F83210BC
:10D6B0008D4200F0128101320E2AF7D100204AF08B
:10D6C000CDFD2988D9F8F42021F001010904090CC5
:10D6D00029809D498D4200F0E880A1F580618D424E
:10D6E00000F0E38001F580418D4200F0DE8001F51D
:10D6F00080618D4200F0D98001F580618D429349AF
:10D7000000F00A81B1EB520F4FEA520040F2F8806C
:10D7100001220021B0FBF2F2ADF80C108C498D48CB
:10D72000120AA1FB02121109A0FB01014908ABF882
:10D730007210490000271209ABF87010284603A99F
:10D740000492ADF81470ADF80E708DF8167045F0B7
:10D75000B3F998F80630ADF81C70602206929A076B
:10D76000CDE908770A9798F8057040F1A380DB00AF
:10D7700003F008034FF00408ADF82630ADF81C8024
:10D7800006AA39462846FFF78DFA08223946FFF7E0
:10D790000DFFB5F844206FEA42426FEA524292B25E
:10D7A000A5F844202A8892B242F080022A802A8C6E
:10D7B00008FA07F39BB292B222EA03022A842A8C67
:10D7C00092B213432B842B889BB243F001032B802E
:10D7D0003246002351688C4202F1240203F1010316
:10D7E00076D0102BF6D14FF0FF3303EBC3030AEBD7
:10D7F000830A594ADAF8383158498B4214BF4FF43A
:10D8000080034FF40013116B0B4313630023726802
:10D81000944206F1240603F101035CD0102BF6D1EB
:10D8200000204F4960220023FDF772FF204644F09C
:10D8300065FF236823F001032360204644F05EFF68
:10D84000019B0B9305F134033B440C9340F22A43B4
:10D850000F934FF480631193424B0D9340230E932B
:10D860004FF480504FF480430026CDE912030BA9FA
:10D870004FF440332046CDE91666CDE91866109680
:10D880001496159343F03AFB0C2F04D8364B03EB58
:10D890004703B3F8DC60AB899BB23343AB812368A9
:10D8A00043F0100301202360B9E628498A4219D2C7
:10D8B000002131E75B0003F00203ADF824304FF0A4
:10D8C00001084FF48073ADF81A80ADF8283057E79F
:10D8D000DBB2013B89E7D8B2A3E707EBC20797F8B1
:10D8E000380DECE6214802F1B77101F55851A0FB63
:10D8F0000101890D013989B2481CB2FBF0F20BE736
:10D900001A4900F1B77202F55852A1FB0221890DA4
:10D91000013989B24A1CFDE68A4204D20120002165
:10D92000B2FBF0F2F8E6114802F1B77101F5585177
:10D93000A0FB0101890D013989B2481CF0E700BF45
:10D94000C00200205CDC050800040140006CDC0221
:10D95000598B4F01ABAAAAAA0038024000600240CE
:10D96000058800087882002054ED0508819F5E1626
:10D97000B82A0020C0190020880100202DE9F04FAE
:10D98000DFF8709299F8003089B01BB9012009B016
:10D99000BDE8F08F934B1C68FCF7DCFC99F8C835A8
:10D9A0000393002B00F012828F4BA3FB04328F4BAA
:10D9B0005209A3FB0213DB0803EB8303A2EB43032F
:10D9C000D9F8042B821A049209F6083BDAB20792BE
:10D9D0000BEB830309F5C66409F6E85202920027AF
:10D9E0009846019432E0304644F088FE8C2303FBD5
:10D9F0000793002583F824569AF805A0204651463F
:10DA00002A46FFF7D3FD019C2246FFF74BF951460A
:10DA10000822FFF7CBFD402344F83C3CA4F1480129
:10DA2000304643F06BFA04F18C030193029B1433EC
:10DA30000293336843F010033360039B01379F4226
:10DA40000BF15C0B08F15C0800F0D680049A002A08
:10DA500005DB019B53F8083C934200F3A2818C2321
:10DA6000019A03FB079352F858AC93F82436166AD0
:10DA7000DAF80040002BB6D07568A389ADB2114624
:10DA800032F8542CC5F116059BB223EA0203072D88
:10DA9000A381A8D9D9F8F03D8A6A0133C9F8F03DCD
:10DAA0000021CDE90572106896468C46012315E0E9
:10DAB000BCF1140F1EDC12F1080748BF02F1170772
:10DAC0003A110CEB271C571E01FA02F201210B44FC
:10DAD00001FA07F79D4247EA02010BD302465EF8BE
:10DAE000040F9D42A0EB0202E2D8CCF115024FF0E8
:10DAF000150CE8E7BCF1150FDDE9057266D13C4D68
:10DB0000C1F38423C1F3441005EB830305EB8000CC
:10DB1000D3F8F830D0F8F8001B0243EA001301F004
:10DB20001F0005EB8000C1F3C43105EB8101D0F883
:10DB3000F800D1F8F810034343EA013383EA1321D4
:10DB400081EA111101F00F010F293FD1C3F30F1327
:10DB50004FF6FF718B4239D0B3F5606F00F025812D
:10DB6000029A93819BF858200798824214D0D8F8E3
:10DB70000810DBF80020521ACBF80020D8F830103B
:10DB8000DBF80420521ACBF804200022C8F8082041
:10DB9000C8F830208BF85800DBF800200132CBF8B1
:10DBA0000020D8F808200132C8F808204FF6FF728C
:10DBB00093427FF418AFDBF804300133CBF8043024
:10DBC000D8F830300133C8F830300CE7D9F8EC3DE4
:10DBD0000133C9F8EC3D002F00F0D9804FF6FF73F8
:10DBE000C0E700BFC01900201F85EB51CDCCCCCCC5
:10DBF00054ED050804000010D9F8D815C9F8045BE5
:10DC0000012389F8EC3E0A68487999F8E0158907FC
:10DC100048BF0423118C83409BB289B221EA0301DF
:10DC20001184118C89B20B431384039B012B3FF4A5
:10DC3000ADAED9F864261368517999F86C26970728
:10DC400054BF012204228A40198C92B289B221EA7F
:10DC500002011984198C89B20A431A84039B022B8E
:10DC60003FF494AED9F8F0261368517999F8F82664
:10DC7000960754BF012204228A40198C92B289B2BD
:10DC800021EA02011984198C89B20A431A84039B80
:10DC9000032B3FF47BAED9F87C271368517999F8B0
:10DCA0008427950754BF012204228A40198C92B21E
:10DCB00089B221EA02011984198C89B20A431A84B3
:10DCC000039B042B3FF462AED9F8082813685179FE
:10DCD00099F81028940754BF012204228A40198C15
:10DCE00092B289B221EA02011984198C89B20A43DD
:10DCF0001A84039B052B3FF449AED9F89428136886
:10DD0000517999F89C28900754BF012204228A4037
:10DD1000198C92B289B221EA02011984198C89B254
:10DD20000A431A84039B062B3FF430AED9F820290E
:10DD30001368517999F82829920754BF01220422C7
:10DD40008A40198C92B289B221EA02011984198C95
:10DD500089B20A431A84039B082B7FF417AED9F8C3
:10DD6000AC2999F8B4191368507911F0020F18BF53
:10DD70000422198C08BF0122824092B289B221EAA2
:10DD800002011984198C89B20A431A84FEE51146EE
:10DD9000124858224FF0CEFCDAF800404FF6FF73DD
:10DDA000E0E6002009B0BDE8F08F0D4991F88E2023
:10DDB00002EB420201EBC2023A4492F89D200D2A86
:10DDC0007FF4CEAE029980228A77CBE6012389F8D0
:10DDD000EC3E039BC9F8043BD8E500BF980E001049
:10DDE000C019002037B590F85F38032B04462DD1B9
:10DDF00000231F4D8DF807309DF8073094F86028F8
:10DE00009A4201D803B030BD9DF8073005EBC3033B
:10DE100093F8783083B181F001037BB19DF807302E
:10DE200005EBC303586FFDF7CFF89DF807300133BA
:10DE3000DBB28DF80730DFE70B46EEE79DF80730E1
:10DE400005EBC303586FFDF7C5F8EEE7D0E9100303
:10DE50009B7903F00103994204D003B0BDE8304040
:10DE6000FDF7B2B803B0BDE83040FDF7B3B800BF6E
:10DE7000B82A002038B5044600790D4650B1FCF7A9
:10DE800067FF08B10323C380E2792946BDE8384023
:10DE9000FDF7F6BE38BD10B504462221FFF7EAFFB4
:10DEA0006379216802229B0802FA03F3DB439BB2E9
:10DEB0000B8263798889D3409A40024392B28A8167
:10DEC00010BD10B504460121FFF7D4FF2068617929
:10DED0008389890802229BB28A4023EA0203838154
:10DEE00010BD38B510F8133CA0F664041BBB94F8C1
:10DEF00050388BBBD4E909239A421CD05A1CA16923
:10DF0000A262CB5C21695B0043F40073A4F854382F
:10DF10000A2384F85238012384F8503894F85F3883
:10DF20008A4228BF0022012BA26201D0042B02D119
:10DF3000606CFFF7C6FF94F84C38002B6DD194F855
:10DF40004D380133DBB2092B84F84D3825D12046FA
:10DF5000BDE83840FAF7D8BC94F952586DB1B4F81E
:10DF600054184B08A4F8543801F001012046013D33
:10DF7000FFF738FF84F85258DDE7D4E909239A42C5
:10DF800084F85058D7D194F85F38012B01D0042B76
:10DF9000D1D1606CFFF77FFFCDE70A2B3DD194F81C
:10DFA0004F382BB9B4F8563843F00103A4F856386B
:10DFB0002379D9070AD5B4F85608820501D4C307D6
:10DFC00018D4B4F85C380133A4F85C38012284F822
:10DFD0004C2894F84F280023012A84F84D381CD18E
:10DFE000617984F84F38606C01F00101BDE8384078
:10DFF00049F01CBEE36AC0F3470013B1216B984798
:10E00000E4E7E3696269D054E369E2680133B3FB92
:10E01000F2F102FB1133E361D8E738BD1648174A25
:10E02000174938B5174C184D121A4FF083FBD4F826
:10E030008820164B164842F47002C4F888201A68EB
:10E04000002142F001021A6099601A6822F084727D
:10E0500022F480321A6058601A6822F480221A6012
:10E060000C4AD960521B28460B494FF063FBA56050
:10E07000BDE83840FAF7A2BC000000100400001010
:10E080007010070800ED00E000000020003802409A
:10E09000103000248801002000000008144BD3F841
:10E0A000F430B0EB930F14D2B0EBD30F13D2B0EB2C
:10E0B000131F12D2B0EB531F11D2B0EB931F10D22B
:10E0C000B0EBD31F0FD2B0EB132F0ED24FF48070F2
:10E0D00070470220704704207047082070471020C6
:10E0E000704720207047402070478020704700BF55
:10E0F000C019002011F001020ED170B590F828105F
:10E10000C568012982B0044607D0B5F1807F01D9E6
:10E110000123037702B070BD70470A4B466AD3F8FB
:10E12000B400FFF7BBFFB5F1807FB080F2D9B7250F
:10E1300021770B46304601A98DF8045042F032FC9D
:10E14000E8E700BFB82A00202DE9F0410546406A03
:10E1500094B0144600681F460E464CF01FFD0B9409
:10E16000264C0C9704F560730093254B0193022312
:10E17000002202930123CDE90922CDE90E22CDE947
:10E1800010228DF80C308DF834308DF8483006921E
:10E190002B7F8DF8202013921A4A049204F55E72A8
:10E1A00005921A1D079223B3330E84F8793304F2D3
:10E1B0007A34330CDFF850802370330A6370A67012
:10E1C000D8F8B4006A6AFFF769FF6B7F90809BB153
:10E1D0006946104642F02CFC6C6A20684CF0DEFC6C
:10E1E000D8F8BC00FFF75AFFA080384614B0BDE84D
:10E1F000F08104F27934DCE705A9EAE78801002020
:10E20000702B002045920008B82A00202DE9F04F1D
:10E21000013B9FB2B44BDFF8D8C2D3F8F4400B688F
:10E2200083B06345BDF830609DF834503AD0DFF8D4
:10E23000BCC2634536D00CF5804C634500F042818A
:10E240000CF5806C634500F03D810CF5806C6345F6
:10E2500000F038816408B4FBF2F41A88013CB3F191
:10E26000804FA4B292B200F03781DFF888C26345D4
:10E2700000F032810CF5806C634500F02D810CF5C7
:10E28000806C634500F02881DFF86CC2634500F0C4
:10E290006481DFF868C2634540F01A811A80DF624A
:10E2A0001C850DE0B4FBF2F41A8822F45C721204AF
:10E2B000120C013C1A80A4B20022DF621C851A866F
:10E2C00001229A824C798A790DB182F0010212F012
:10E2D000020C62D0D2004FF0000E02F008074FF49B
:10E2E000806201924FF0400CF346CDF800E0F24618
:10E2F00072464FF0040975460C2C35D8DFE804F05F
:10E30000B73434348B343434073434345E001C8CEA
:10E31000DFF8D8C124F480742404240C1C841C8CE1
:10E3200024F4007424042A43240C9D8844EA022423
:10E330009A8B22F073021204120C6345ADB242F0C4
:10E34000600200F0EB800CF5806C634500F0E68025
:10E350009D809A83DE631C849A8B22F0080212044B
:10E36000120C42F008029A83B3F844206FEA42424A
:10E370006FEA524292B2A3F844201A881C4692B225
:10E3800042F0010224F8342B4A794360A11800239B
:10E390000160A35003B0BDE8F08F4FF480655200D8
:10E3A000CDE9005C02F002024FF4805E4FF4804B36
:10E3B0004FF4807A6746E14601259DE715431A8CA4
:10E3C0004A4F22F480521204120C1A841A8C22F43E
:10E3D00000521204120C42EA05329D889C8B24F4F0
:10E3E000E6442404240CBB42ADB244F4C04400F023
:10E3F000AF8007F58067BB4200F0AA809D809C83B8
:10E400001E641A849A8B22F400621204120C42F4E5
:10E4100000629A83A8E71C8CDFF8D0E024F0100497
:10E420002404240C1C841C8C24F0200424042A437F
:10E43000240C9D8844EA02141A8B22F4E64212044A
:10E44000120C7345ADB242F4C04259D00EF5806E45
:10E45000734555D09D801A839E631C841A8B22F4C9
:10E4600000621204120C42F400621A837CE71C8CD6
:10E47000DFF878C024F001042404240C1C841C8CD4
:10E4800024F0020424042A43240C9D8814431A8B8C
:10E4900022F073021204120C6345ADB242F0600226
:10E4A00049D00CF5806C634545D09D801A835E632E
:10E4B0001C841A8B22F008021204120C42F008028B
:10E4C0001A8351E7B4FBF2F2541E1A88A4B292B236
:10E4D00022F4407292B2E1E622F45C7292B21A80A7
:10E4E000DF621C85ECE600BFC0190020000001407F
:10E4F00000040140000400400010004000140040EF
:10E5000024F0800444EA0714009F25F4406524F0B9
:10E5100040042F434CEA04043D469BE724F4006486
:10E5200044EA0724019F24F4806425F440553C43C9
:10E530004EEA05050CE74FF6F37C04EA0C0C25F4D3
:10E5400040754CEA070C45EA0A054CEA0904ACE7B9
:10E5500025F480454BEA050550E7ACF80020CCF8DF
:10E560002C70ACF82840ABE6274A92F8F83A7BB317
:10E57000D2F8381A884237D0012B29D0D2F8501A55
:10E58000814235D0022B23D0D2F8681A884231D08C
:10E59000032B1DD0D2F8801A88422DD0042B17D01F
:10E5A000D2F8981A884229D0052B11D0D2F8B01A87
:10E5B000884225D0062B0BD0D2F8C81A884221D029
:10E5C000072B05D0D2F8E01A814208BF07230CD0F0
:10E5D00003EB430102EBC10103F1010CC1F8380A5E
:10E5E00082F8F8CA184670470023DBB21846704715
:10E5F0000123FAE70223F8E70323F6E70423F4E70D
:10E600000523F2E70623F0E7040000100548D0F8E0
:10E61000703623B1DB6A13B100F5CE6018470248AB
:10E62000704700BFC0190020CCEE050838B51D4C5E
:10E63000D4F8C0301B8843B91B4D002384F8CF3079
:10E6400085F86836C5F8643638BDD4F8C420002A89
:10E65000F2DDD4F8C810012A488806D00123124DF3
:10E66000A4F8CC0084F8CE30E7E78A880132121A89
:10E670009A42F3D10C4DD5F8703600221B69C5F8CB
:10E680009C2605F5CE609847D5F870369B68002B20
:10E69000D3D005F5CE6098470028CED14AF024FCAF
:10E6A000CBE700BFB82A0020C01900200748D0F8E7
:10E6B0006C361BB1064B93F8CE300BB1002070477F
:10E6C000D0F8703600F5CE605B681847C01900209E
:10E6D000B82A002030B4174A174B92F868C603F1E5
:10E6E000D00505EB0C04C0E9004593F8CF3092F853
:10E6F0006806834292F8680614D8834206D3002342
:10E700001A46184630BCC1E90032704792F86806D4
:10E710001A1EC0F1800330BC0CBF01200220C1E9E9
:10E72000003270471B1A0022012030BCC1E90032C0
:10E73000704700BFC0190020B82A00200E4B0F4AB6
:10E7400093F8681692F8CF0093F86826904293F8F1
:10E7500068260CD8904238BF93F86826D3F8643600
:10E760003ABFC2F180028018002018447047D3F8E5
:10E770006436801A18447047C0190020B82A002057
:10E7800038B5194D194CD5F8C020937B012B08D012
:10E79000D4F8643603F2FF736FF30A03C4F86436E7
:10E7A00038BDD4F870365B6A63B104F5CE60984723
:10E7B000D4F870369B681BB104F5CE60984778B1E9
:10E7C000D5F8C020D4F864365288013B1344524235
:10E7D000134003F2FF736FF30A03C4F8643638BDC5
:10E7E0004AF082FBECE700BFB82A0020C0190020E5
:10E7F00070B51E4C1E4D94F8683694F8681684B0B7
:10E8000005F1D0021344029395F8CF3003928B4266
:10E8100020D894F86826934214D294F868161E46BD
:10E82000C1F18001F3B98C460122CDE9001610B97F
:10E83000BCF13F0F06D90023694602A84CF030FE18
:10E8400095F8CF3094F86806C01AB0FA80F0400905
:10E8500004B070BD94F868C6A3EB0C0C61460026AA
:10E860000122E2E701EB030C0222DEE7C0190020DF
:10E87000B82A00202DE9F043164685B0002936D08D
:10E88000441E254D254F04EB01084FF0000901E01F
:10E89000A0452CD095F8CF0014F8013F411C284426
:10E8A000C9B280F8D0300B0648BF002097F8683610
:10E8B00085F8CF104ABF0146084685F8CF909942A7
:10E8C00097F8683636BFC3F18003C01AC0183F28D6
:10E8D000DED997F868369942DAD0114B93F8C430F4
:10E8E000002BD5D00020FFF783FFA045D2D1694689
:10E8F00002A8FFF7EFFE20B1DDE9003213443F2B01
:10E9000002D805B0BDE8F0830246334602A84CF0B9
:10E91000C7FD05B0BDE8F083B82A0020C01900206B
:10E920008801002030B585B0694602A8FFF7D2FE05
:10E9300058B9094C04F5CE65D4F8703628465B68A2
:10E9400098470028F8D005B030BD0246012302A840
:10E950004CF0A6FDEDE700BFC019002070B5134DC7
:10E96000134C0023C5F86C3648F030FFC4F8C800DB
:10E97000FFF74CFED4F8C830C4F8C000A3B19A88A1
:10E980005B88D21A436802FB0333C5F86C36FAF78A
:10E9900065FD95F8683694F8CF209A42064601D076
:10E9A000FFF7C0FFC5F8646670BD00BFC019002046
:10E9B000B82A00202DE9F041104ED6F86C361546E5
:10E9C00082189A420E4A88BF1D1A92F8CF2096F8F4
:10E9D00068369A4204460F4601D0FFF7A3FFD6F8E7
:10E9E000702608480023C6F89C362B46956A2146B7
:10E9F0003A46AC46BDE8F041604700BFC019002070
:10EA0000B82A0020302000208C461346014662467A
:10EA10001846CFE72DE9F04F41F694628BB0002104
:10EA2000A3484EF0DFFE042043F052FF04460520C9
:10EA300043F04EFF50EA040340F02A819D4B0393BC
:10EA40004C2200219A489C4D4EF0CCFE00214C22D5
:10EA500097484EF0C7FE039B954AD3F8B433156030
:10EA600001241471D3611746136253624BF076F997
:10EA7000FFF774FF002108460AF05CFFFAF7EEFC8E
:10EA8000B0F1000840F3A1818C4DDFF850E28C4ECC
:10EA9000CDF808E0002407F14C0901942746A2466E
:10EAA00005F5A87B04E00AF5006AD04540F3AF8085
:10EAB000029A1368C2F8B436FAF704FD20225946C8
:10EAC0005046FFF777FF7F49122258464EF0C7FEA7
:10EAD0000028E8D1574525D001997B4B01EB410235
:10EAE00003EB820301934A1C184678490592AAEB6E
:10EAF0000703049301F0DCFB4946019B41F84C3BC2
:10EB0000049B059AC9F80C70C9E90433D9F81C3084
:10EB10000192C9E908336E4BC9F828300123C9F8BE
:10EB200008308946039BD3F8B433C9F81C305746E4
:10EB30001222A918335D91F85011994202F1010295
:10EB40000BD00024202AF4D12037B8455946384646
:10EB500053DBFFF72FFF0022EBE70134152CF1D137
:10EB6000D0195C4F20223946FFF724FF3846002396
:10EB70000A2209A9099701F0CDFC0746099800234C
:10EB800001300A2209A9099001F0C4FC07900998F4
:10EB9000002301300A2209A9099001F0BBFC06906C
:10EBA0000998002301300A2209A9099001F0B2FC5A
:10EBB0000590099809A9013000230A22099001F063
:10EBC000A9FC04900998002301300A22194601F09B
:10EBD000A1FC97B1DDE9063243EA4212049B059994
:10EBE0005B0143EAC123A7F2BC7143EA600342EA36
:10EBF000412243EA0243C9F81C30019B642B00F018
:10EC0000B28057460AF5006AD0453FF751AF019BE5
:10EC1000642B00F0A880BA451DD0019B2A4C2B49DB
:10EC20000C2202FB03445E1C3246204601F040FBEE
:10EC3000D9F81C20C9F80040AAEB0705C9E9082249
:10EC4000C9E90375224AC9F828200122C9F81450DD
:10EC50000196C9F80820019B002B03F1010100F384
:10EC600085804FEA4803B3F1805FC0F2AF80104B5C
:10EC70009C6834B91A461B791BB11368002B40F00D
:10EC8000DB80002108460BB0BDE8F04F0AF052BE11
:10EC90004FF47A72002321464DF052F90E4BA3FB3C
:10ECA00000231B0C40F2B27240F26D141AE000BF58
:10ECB000F05D00208801002084CA0608B82A0020E0
:10ECC000945B0608705B0608282C0020845B06080D
:10ECD00009EA0008082C002007452EC2C0190020B0
:10ECE0005B1A013212F0030514BF21464FF4B771CD
:10ECF0008B42F5DAA349002D00F098800391039927
:10ED0000D1F884138B42C0F23B819F4D01245B1AE2
:10ED100055F8041F994204F10104F8DD013343EA78
:10ED20004413A2F2BC7243EA4223984A039DB0FB0B
:10ED3000F2F102FB11024FF461603C24B2FBF0F1EE
:10ED400000FB11221C20C5F88803B2FBF4F004FB81
:10ED50001022521042EA401242EAC12242EA034320
:10ED6000C5F8B4336CE66423019365214C268848CA
:10ED7000DFF830A2874F06FB01F405193246002167
:10ED800028464EF02FFD3246002128464EF02AFD3F
:10ED90007F48814E40F804A004F110034FF00109B0
:10EDA000C5F808902F62AE6240F803800344021D4C
:10EDB000C3F804801834039B0199D3F8B43313517A
:10EDC000A018023143606B624BE72146704BDFF8BD
:10EDD000D8914C2606FB01F41D1932460021284625
:10EDE0004EF000FD3246002128464EF0FBFC684BF9
:10EDF000684E43F80490039A2E62684ED2F8B4032A
:10EE000004F1180104F110020127341FC8F1006356
:10EE1000BB404FF0020A85F805A0AF60A350224422
:10EE20005360705031444860686220E70C4603919B
:10EE30001D21C4F8881362E7554900220023C1E967
:10EE400010238C640A46CC6326462146D56C02F119
:10EE50004C03B5B198689E644D1EA842C2E9236672
:10EE6000DE6300F086804D1CA84274D113F8481C64
:10EE700000293FF406AF1A6443F8083C01461A46DD
:10EE8000E4E7434A0226294615E0D36B16635B018B
:10EE900018BF03F6FF73C2E9041114BF00EB13336C
:10EEA000334653631846906352F84C7FC31A1D448F
:10EEB000461C0134CFB11379701E002BE5D11369C4
:10EEC00016635BB103F6FF73576900EB13335363AB
:10EED0004FB107F6FF7700EB1730E4E75769334689
:10EEE0005363002FF5D13046DDE7DFF8C0E02C4B4F
:10EEF000CEF8044701383E24CEF8F8560EF5DA6213
:10EF0000CEF8DC363F254023C2E90445CEF8E8368A
:10EF1000CEF8F406840F8300D8B140F2FF155B19D8
:10EF200044F100045B0A43EAC45303F14004234460
:10EF300003EBC0001649CEF8F036C30D5360430210
:10EF4000C2E90B11CEF8EC46CEF8D806CEF8D03692
:10EF500097E60123E9E788427FF493AE00293FF466
:10EF600090AE106CC56B0135C563186493641A4686
:10EF70006CE700293FF485AE53F80C2C0146EDE711
:10EF80000124CBE6880100200C05002080510100FF
:10EF9000F05D00200068214C09EA0008F45D0020C3
:10EFA000C85B0608AC5B0608BC5B0608C0190020FD
:10EFB0002DE9F043DFF82881474D93B0FFF736FB8A
:10EFC00098F8683695F8CF209A4201D0FFF7AAFC4E
:10EFD000D8F86C760024C8F86446002F6DD03F4EF8
:10EFE0000AE098F8683695F8CF209A4201D0FFF7EA
:10EFF00099FC2034A7421BD922463146684601F0CD
:10F0000057F968464CF03EFB012201466846FFF77F
:10F0100031FCA3B2002BE4D1D8F8BC36002BE0D0F1
:10F020009A881B6859690A4214BF5A831A83D8E721
:10F03000FFF7A6FB98F8683695F8CF209A4201D0E2
:10F04000FFF770FC0023DFF89490C8F864361E4682
:10F050001C4602E02034A74229D92246494609A885
:10F0600001F026F92122002168464EF0BBFB202248
:10F0700069462046FFF79EFC2022054609A96846FE
:10F080004EF0EDFB08B9202D00D00136A3B2002BC5
:10F09000E0D1D8F8BC36002BDCD01A689B885169C7
:10F0A00020340B4214BF53831383A742D5D8B6FA3A
:10F0B00086F0400913B0BDE8F083FFF761FB98F8D4
:10F0C000683695F8CF209A4201D0FFF72BFC002339
:10F0D000C8F864360120EDE7B82A0020D05B0608A6
:10F0E000C019002000B585B0194A00230193019290
:10F0F000019A0C320192019A0321116072B6154AED
:10F10000D2F82016D2F8242651EA020412D11A4667
:10F110000F48002402940290029910310291029942
:10F120000A6003940390039A14320392039A1360C3
:10F13000FDF7CAFB084B1B684EF6602404FB00F089
:10F140005B1842F10002C31842EBE072E0E700BF37
:10F1500050280040B82A0020C019002000B501EB5B
:10F16000020E714516D001390EF1FF3E41F2210C1D
:10F1700011F8013F082280EA032003B2002B4FEA76
:10F180004000B6BF8CEA430380B298B2013AF4D192
:10F190008E45EDD15DF804FB704700BFD0ED007ADD
:10F1A000D0ED016A30EE677AE6EE877AB0EE670A54
:10F1B000C0ED007A704700BFD0ED017AD0ED026A51
:10F1C00030EE677A90ED000AE6EE877A37EEC07A85
:10F1D000C0ED017AA6EE870A80ED000A704700BFF5
:10F1E00090ED017AD0ED036AD0ED027A30EE470A55
:10F1F000A6EE807A90ED000A80ED017A37EE676A1C
:10F20000E6EE867A37EEC07AC0ED027AA6EE870A7D
:10F2100080ED000A704700BFD0ED056AD0ED017A9D
:10F2200090ED066AD0ED025A90ED035AC0ED066AE1
:10F23000B0EE407A26EEA70AD0ED007A80ED057A8E
:10F24000A7EE870AD0ED077AA5EE860A90ED086A48
:10F25000D0ED045AC0ED087AA5EE670AA5EEC60AFD
:10F2600080ED070A704700BFF0EE406AD0ED007AEB
:10F2700090ED050A90ED067A90ED016AD0ED035A03
:10F28000A7EEA60AA6EE267AD0ED047A90ED026AE1
:10F2900067EEC07AA5EEC07AE6EE267A80ED057AB2
:10F2A000C0ED067A704700BF2DE9F047DDF820A0D9
:10F2B00055460F4615F8011B002B064614460CBF99
:10F2C0004FF020094FF0300939B3002A2BDD2B46CF
:10F2D00000E09CB113F8012BA046013C002AF8D1B4
:10F2E000A8F1020854B1444649463046B847013CAB
:10F2F000FAD29AF8001008F1010459B13046B84723
:10F300002B4615F8011B0029F8D1A4EB0A041819A3
:10F31000BDE8F0872046BDE8F087002A02F1FF38FB
:10F32000E1DC0846F4E70024E8E700BF03685A1C64
:10F3300002601970704700BF10B500F1004402462A
:10F34000013C04E0B3EB0E0015D1A24214D012F838
:10F35000013BA3F14100192811F8010BA0F1410C68
:10F3600098BF2033BCF1190F00F1200EEAD91B1A07
:10F3700004D10028E9D110BD002010BD184610BDF1
:10F38000884210B54FF001043ED301FB04F4B0FBFA
:10F39000F4FC8C45F9D2CCB122BB08E0A14203F8C1
:10F3A00001EBB4FBF1F211D8B0FBF2FC1446BCF156
:10F3B000090F0CF1570E0CF1300204FB1C00EDDCC0
:10F3C000A14203F8012BB4FBF1F2EDD900221A702F
:10F3D00010BDA14203F801EBB4FBF1F2F6D8B0FB8B
:10F3E000F2FC1446BCF1090F0CF1370E0CF130029F
:10F3F00004FB1C00EDDCA14203F8012BB4FBF1F28D
:10F40000EDD900221A7010BD8446002AEAD1CEE759
:10F41000002870B503DA2D2301F8013B404209288A
:10F4200086464FF0010307DD03EB83035B00B0FB6F
:10F43000F3F2092AF8D8E3B10F4CA4FB0320BEFB7A
:10F44000F3F2092A02F1570602F130054FEAD00023
:10F4500007DD092B01F8016B03FB12EE09D9034606
:10F46000EBE7092B01F8015B03FB12EE01D9034620
:10F47000E3E700230B7070BDCDCCCCCC0378202B00
:10F48000024600F10100F9D0092BF7D02D2B28D02E
:10F490002B2B03BF5378B7EE000A0246B7EE000AE3
:10F4A000A3F13001C8B209289FED567A10D8F2EEC8
:10F4B000046A07EE901AF8EEE77A12F8013FE7EED9
:10F4C000267AA3F13001C8B20928B0EE677AF0D9E4
:10F4D0002E2B5ED003F0DF03452B07D020EE070A6A
:10F4E00070475378BFEE000A0246D9E710B451784E
:10F4F0002D2978D02B296AD0A1F13003092B02F1F4
:10F5000001026BD80024002303EB830301EB4303C8
:10F5100012F8011FA1F130000928A3F13003F3D93B
:10F52000B3F59A7F1A4628BF4FF49A72072B66D913
:10F53000DFED356A1346F7EE007A083B072B67EEDE
:10F54000A67AFAD802F00702DAB1F2EE046A012ACA
:10F5500067EEA67A15D0022A67EEA67A11D0032AA2
:10F5600067EEA67A0DD0042A67EEA67A09D0052A9E
:10F5700067EEA67A05D067EEA67A062A18BF67EE70
:10F58000A67A6CB387EE277A5DF8044B20EE070A63
:10F5900070475378A3F13001C8B2092802F1010283
:10F5A00098D8F2EE046AF0EE665A07EE901AF8EE7A
:10F5B000E77A12F8013F87EEA66AA3F13001C8B2DC
:10F5C000092866EEA56A37EE067AEED982E79178C9
:10F5D000A1F13003092B02F1020293D9F7EE007A70
:10F5E00027EE277AD0E79178A1F13003092B02F1B9
:10F5F000020288BFF7EE007AC4D8012483E7F7EE51
:10F60000007AA1E70000000020BCBE4CF0B50679EE
:10F6100006F0E003402B03D145794FF0FF3406E0BC
:10F62000602B4FF00105F8D1447905FA04F400236A
:10F63000012006F00706AB4200D1F0BD052E0FD821
:10F64000DFE806F00308101D242448B1C85CD75C2D
:10F6500078400FE020B1C856D756C71B7842784192
:10F660000133E8E70028FBD031F8130032F81370BB
:10F67000784080B220420CBF01200020F0E7002833
:10F68000EED031F9130032F91370E6E70028E7D025
:10F6900051F8230052F82370DAE7F8B50C4E3378AE
:10F6A00005468BB9F8BD25B12388C3F30B039D42F2
:10F6B00004D0D4E90201A2884EF03CF81C34BC42CC
:10F6C000F1D300233370EDE7024C034FF7E700BF9F
:10F6D0002093002050ED060810F60608037903F089
:10F6E0001803102B1CD003D833B9B0F80B007047A7
:10F6F000182BFAD000207047104BB0F80B0093F98C
:10F700000030591C06BF0E4B1B78DBB203EB4302E3
:10F7100003EB820303EBC30300EB430080B27047AB
:10F72000064BB0F80B0093F901305A1C06BF044B8E
:10F730005B78DBB200EB4310F0E700BFFC05002074
:10F74000E0300020032870B516D80C4BC60003EB40
:10F75000C000C943057A427A01F0010181EA05043B
:10F76000A24209D042682AB190881268A94214BF07
:10F770001083508333445C7270BD00BF209300201F
:10F780000379062B0FD1C9B20D2998BF074BC26868
:10F7900094BF5956002101238B40134214BF0846E1
:10F7A0004FF0FF307047481C704700BFF05B060801
:10F7B000092900D001B9704701394A0002F0080256
:10F7C000930001F00301A3EB9203C1EB0111C3EB22
:10F7D0000313C1EB011100229B00890002608180AC
:10F7E00043807047B5EEC00ADFED347AF1EE10FACF
:10F7F000CCBF30EE270A30EE670ADFED317A20EE1B
:10F80000270A30B5FDEEC07A87B017EE904A05465C
:10F8100084EAE470002303A9A0EBE470CDE900338F
:10F82000029346F0E1FB002CB4BF2D23202303A854
:10F830008DF800304BF026FF012829D0022833D064
:10F8400003281DD003A968464DF0D4FF68464BF04D
:10F8500019FFC41EE4B22246694628464DF06AFFED
:10F8600000232B5528464BF00DFF2E232B5401303F
:10F870000DEB040128444DF0EAFF284607B030BDE7
:10F88000302303A968468DF801304DF0B3FFDDE762
:10F8900043F23002302303A96846ADF801208DF809
:10F8A00003304DF0A7FFD1E743F2300303A96846C8
:10F8B000ADF801304DF09EFFC8E700BF6F12033A6C
:10F8C00000007A4409F08ABE38B5054658B14C1E8E
:10F8D00014F8011F284619B9BDE8384009F092BE56
:10F8E00009F07CFEF4E738BD70B50546B0F80900B4
:10F8F00042F04AFE054B1E7804462846FFF7EEFE0E
:10F9000016B1E368184470BDA368FBE7209300209C
:10F9100038B505460C46FFF7E7FF2A7902F00703E2
:10F9200002F0E002602A29D1052B0CD8DFE803F0B1
:10F93000030B0F0B1B1B6A7901239340DBB2027888
:10F9400014B11343037038BD22EA0303FAE76A795E
:10F95000012393409BB2028814B113430380F2E762
:10F9600022EA0303FAE76B7901229A40036814B193
:10F9700013430360E7E723EA0203FAE7052BE2D823
:10F98000DFE803F00303050507070470DBE70480E5
:10F99000D9E70460D7E708B520214DF03AFF0346C8
:10F9A000184623B10278202A03F10103F8D008BDDC
:10F9B00008B5CB0701D4FCF787FF08BD2DE9F3415B
:10F9C000124D134F002305F8243F044600EB810637
:10F9D000B44203D10F4802B0BDE8F0813946284651
:10F9E0004DF008FF214668464DF031FF4FF000080A
:10F9F000202168464DF00DFF28B9694628464DF094
:10FA0000F9FE0434E4E780F80080F1E72093002059
:10FA100050D70608449300202DE9FF47914604463D
:10FA20008A461E46FFF7ACFE421CBDF83070DDF87A
:10FA3000348005461FD0B9F1FF3F1FD0CDE9000942
:10FA4000144A236831463846C0474A4620795FFA4F
:10FA50008AF1FBF7F5FC024600B10288D3B20393AA
:10FA6000C2F30323120BCDE90052029323680A4A22
:10FA700031463846C04704B0BDE8F0877B06FAD46B
:10FA80000C902368054A31463846C44604B0BDE8A8
:10FA9000F047604762CB06086FCB060893CB060899
:10FAA0002DE9F043154685B06A1C8946BDF83060E3
:10FAB0000D9F194625D04FEA101800F00F0408F1E9
:10FAC0004008CDE90045164A43463046B847A8B13C
:10FAD00099F80510D9F800002A46FBF7F3FC68B145
:10FAE000038802780392C3F303221B0BCDE9004382
:10FAF000029243460B4A00213046B84705B0BDE8A4
:10FB0000F0837306FAD40309074A00F00F000C9043
:10FB100040333046BC4605B0BDE8F043604700BF07
:10FB2000A2CB0608B4CB0608DDCB06082DE9F043CE
:10FB300087B00709DDF8388091461E46403700F04F
:10FB40000F0439B30AF0F8FFC379174ACDE900432F
:10FB500005463B4649463046C047C0B12868FBF7DA
:10FB6000A3FFAA796B79114912F0020F4FEA9303B0
:10FB70000F4A18BF0A46E97900940133CDE9032101
:10FB8000CDE901030B4A3B4600213046C04707B090
:10FB9000BDE8F083084A0E943B4649463046C446C9
:10FBA00007B0BDE8F0436047F1CB0608E8CF060890
:10FBB0007AE1060803CC060825CC0608484008234D
:10FBC00041B240000029C0B2B8BF5040013BF7D15C
:10FBD000704700BF30B505688D42044618D901F161
:10FBE000FF3E681E00231EF801CF082183EA0C03A4
:10FBF0004FFA83FC5B00BCF1000FDBB2B8BF53408F
:10FC00000139F5D17045EED16A1C22602B7030BDF0
:10FC100000236A1C22602B7030BD00BF10B52DED93
:10FC2000028B08EE101AB8EE488ADFED7E7ADFED1F
:10FC30007E0A28EE008A044628EE278AB0EE480A9B
:10FC40004DF06EF89FED797AB4EEC70AF1EE10FA36
:10FC5000F0EE407A40F3BD809FED736ADFED746A89
:10FC6000B0EE677AB4EEE67AF1EE10FA77EEC67A85
:10FC7000F6DC9FED707AF4EEC77AF1EE10FA40F3FD
:10FC8000C5809FED6A7A77EE677A27EEA76ADFED87
:10FC90006A5ADFED6A6A9FED6A7A9FED660ADFEDC8
:10FCA000620AE6EE256A67EE865AA6EE267A38EEF6
:10FCB000000AE5EE877AB0EE678A4DF031F8DFEDA5
:10FCC0005B7AB4EEE70AF1EE10FA5BDDDFED566A1F
:10FCD0009FED577AF0EE407AF4EEC77AF1EE10FA23
:10FCE00030EE660AF6DCDFED537AB4EEE70AF1EEA9
:10FCF00010FA62DDDFED4D7A37EEC00AF7EE007ADA
:10FD0000DFED504ADFED4C5A9FED4C7AC4ED097A95
:10FD1000B0EE675AA8EE245A0023A36160EE006A91
:10FD200087EE856A63612362E361A6EEA57A9FEDA3
:10FD3000445AA6EE875A20EE264AF0EE675AA4EE01
:10FD4000050AE8EE645ABDEC028BB6EE007AF8EED6
:10FD5000006A77EEC07A26EE077A66EE266A27EE0C
:10FD6000277A66EE806A67EE867A25EE866A84EDEB
:10FD7000007AC4ED017A84ED027AC4ED036A84ED61
:10FD8000046A10BDDFED307AB4EEE70AF1EE10FA46
:10FD9000A9D5DFED256A9FED2D7AF0EE407AF4EEDD
:10FDA000C77AF1EE10FA30EE260AF6D4DFED217AAA
:10FDB000B4EEE70AF1EE10FA9CDCDFED257AB4EE42
:10FDC000E70AF1EE10FA44BFDFED1F7A37EEC00A02
:10FDD00094E79FED1D7AB4EEC70AF1EE10FA7FF5B5
:10FDE00048AF9FED116ADFED196AB0EE677AB4EEA5
:10FDF000E67AF1EE10FA77EE867AF6D49FED0D7A78
:10FE0000F4EEC77AF1EE10FA3FF73BAF9FED107AB0
:10FE1000F4EEC77AF1EE10FA44BF9FED0B7A77EE5D
:10FE2000677A32E727D4D236DB0FC940DB0F49406F
:10FE3000E4CB1641DB0FC93F92E741B99730083C4C
:10FE400015A82ABEF304353FDB0F49C0E4CB16C129
:10FE5000DB0FC9BF08B5DFED2D0A4CF061FFDFED08
:10FE60002C7AB4EEE70AF1EE10FA28DDDFED276A0E
:10FE70009FED287AF0EE407AF4EEC77AF1EE10FAB0
:10FE800030EE660AF6DCDFED247AB4EEE70AF1EE36
:10FE900010FA2FDDDFED1E7A37EEC00A20EE007A71
:10FEA0009FED1E6ADFED1E6ADFED1E7AE7EE066A41
:10FEB00020EE076AE6EE877AA6EE270A08BDDFED98
:10FEC0001A7AB4EEE70AF1EE10FADCD5DFED0F6A2C
:10FED0009FED167AF0EE407AF4EEC77AF1EE10FA62
:10FEE00030EE260AF6D4DFED0C7AB4EEE70AF1EE36
:10FEF00010FACFDCDFED0E7AB4EEE70AF1EE10FA7D
:10FF000044BFDFED097A37EEC00AC7E7DB0FC9400F
:10FF1000DB0F4940E4CB1641DB0FC93F92E741B903
:10FF20009730083C15A82ABEDB0F49C0E4CB16C1A8
:10FF3000DB0FC9BFB0EEC07AF0EEE06AF4EEC76A3C
:10FF4000F1EE10FAB4BFF0EE475AF0EE665AF5EE55
:10FF5000405AF1EE10FAF0EE407A44D0F4EEC76A5F
:10FF6000F1EE10FA8CBFB0EE475AB0EE665A85EE4D
:10FF7000256A9FED1E2A9FED1E3A9FED1E4ADFED7A
:10FF80001E4ADFED1E2ADFED1E3A9FED1E5AA6EE39
:10FF9000423AE6EE223AA6EE034AF7EE005AE6EEC1
:10FFA000044AE6EE235AA6EE245A85EE250AF4EE1C
:10FFB000C76AF1EE10FA48BF9FED137AF5EEC00A5A
:10FFC00048BF37EE400AF1EE10FA48BF9FED0F7AB6
:10FFD000F5EEC07A48BF37EE400AF1EE10FA48BF9E
:10FFE000B1EE400A70479FED070AE0E739094E3D40
:10FFF000E3B59E3E88FA163E45FE7F3F99FB243FBF
:020000040801F1
:1000000069A2163EA7DFA834DB0FC93FDB0F4940CA
:100010002DE9F04F144689B08846217801320392C9
:10002000002900F01681002507461E46A94609E072
:100030003846C047039C01352178631C039300298F
:1000400000F08F802529F3D16078A31C3028CDE9FA
:10005000033923D0A0F13003DBB2092B4FF0000AA3
:1000600026D96C282AD078287FD8572878D9A0F1AB
:100070005803202B79D8DFE803F0BD7878787878BA
:10008000787878787882AF787878787878787878AF
:10009000AA787878789E788A7878BD00A078E31C72
:1000A0000393A0F13003DBB2092B4FF0010AD8D83B
:1000B00004AA03A947F064FB6C28D4D1039C2278DE
:1000C0000134782A0394B7D8572A40F28E80A2F1DF
:1000D0005803202BB0D801A151F823F013020108D6
:1000E0003900010839000108390001083900010808
:1000F00039000108390001083900010839000108F8
:100100003900010839000108810101082F020108A6
:1001100039000108390001083900010839000108D7
:1001200039000108390001083900010839000108C7
:1001300039000108D101010839000108390001081E
:100140003900010839000108B90101083900010826
:100150003F020108390001083900010813020108B3
:1001600028B9284609B0BDE8F08F039C64E725282C
:10017000FBD1039C25213846C04701355CE7039C31
:1001800056F8041B3846C9B2C047013554E70DF193
:10019000140B56F8040B039C5B4600220A21FFF760
:1001A000EFF8049ACDF800B0534641463846FFF7C1
:1001B0007BF8054440E7039C56F8043B0093049AFF
:1001C000002341463846FFF76FF8054434E7039CA7
:1001D00056F8043B1D602FE70DF1140B56F8040B85
:1001E000039C5946FFF714F9DBE7002AB9D0252A0A
:1001F000C0D021E7A0F15802B2FA82F20DF1140B3F
:1002000056F8040B52095B461021FFF7B9F8039C1E
:10021000C7E7A2F158020DF1140BB2FA82F256F8B8
:10022000040B52095B461021FFF7AAF8B9E70DF15C
:10023000140B56F8040B5946FFF7EAF8B1E70DF135
:10024000140B56F8040B5B4600220A21FFF798F8BE
:10025000A7E70D4685E7F8B5104C0746A06C0D469C
:100260001646A0B10E49FFF72FFBA06C3946FFF7E9
:100270002BFB0C49A06CFFF727FB0B49A06C334606
:100280002A46FFF7C5FE0949A06CFFF71DFB94F84D
:100290004C3013B1012384F84D30F8BD2093002079
:1002A00037CC06087BE60608C5F8000844CC0608EB
:1002B0000EB400B584B005AB019053F8042B064989
:1002C000039301A8FFF7A4FE019B00221A7004B05B
:1002D0005DF804EB03B070472DF30008F7B5114E3D
:1002E00007463046002300F84E3F0C460E4B0F49A0
:1002F000002F18BF194615464DF07CFA0C4F04EB41
:1003000045054E36AC4202D10A4803B0F0BD39462D
:1003100034F8022B6846FFF7CBFF694630464DF0B4
:1003200069FAEFE72093002048CC060851CC060874
:100330005ACC06086E930020F7B50C4E0C4F0023E4
:1003400006F87F3F044600EB4105AC4202D1094864
:1003500003B0F0BD394634F8022B6846FFF7A8FF1A
:10036000694630464DF046FAEFE700BF2093002083
:1003700095CF06089F930020F8B5084F4E1E0546FE
:1003800001F11F0416F8012F28463946FFF790FFA8
:10039000A64205F10205F5D1F8BD00BF5FCC060805
:1003A0000246531C084605D1034B1A681B790A60A4
:1003B0000B71704701497BE79DCB060896CF060875
:1003C00010B5013114460AF0B7FB28B9054B1A687D
:1003D0001B792260237110BDC27903492046BDE814
:1003E000104065E79DCB0608FECB060803685A1C43
:1003F000026019700368090A5A1C0260197070477C
:1004000010B402681346511C016013F8021B03600C
:10041000D31C5478036093781B0443EA0423141D0F
:100420000460D0785DF8044B0B4343EA00607047EA
:10043000A0F13003092B07D920F0200041381928FA
:100440008CBF0020012070470120704730380928F8
:100450008CBF002001207047413819288CBF002034
:1004600001207047613819288CBF00200120704797
:10047000202805D0093804288CBF002001207047AF
:1004800001207047A0F14103192B98BF203070471D
:10049000A0F16103192B98BF2038704702B310B543
:1004A0008446841803E0981A15D1A44514D01CF88A
:1004B000013BA3F14100192811F8010BA0F1410EF5
:1004C00098BF2033BEF1190F00F12002EBD91B1A9F
:1004D00004D10028E9D110BD002010BD184610BD80
:1004E0001046704770B5044608460D464BF0CAF8F2
:1004F000064602E014F8013F43B132462946204641
:10050000FFF7CCFF0028F5D1204670BD1C462046E1
:1005100070BD00BF2DE9F043064686469EF800C038
:10052000BCF1200F7446ACF109050EF1010EF5D0B7
:10053000042DF3D9BCF12B0F64D0BCF12D0F26D1C3
:100540000127102A94F801C004F1010423D04FF0D0
:10055000FF35B5FBF2F502FB05FE6FEA0E0E5FFA02
:100560008EFE9046002014F801CBBCF1390F4CF000
:100570002009ACF1300C29D85FFA8CFC944528DABC
:10058000A84226461ED81BD000FB08C0EBE7102A65
:100590004FF00007DBD1BCF1300F0AD16078A0F139
:1005A0004105192D98BF2030661C78280CBF0234F5
:1005B00034466FF070454FF00F0E4FF01008D1E742
:1005C000F445E1D94FF0FF301F40CCE7B9F1600F9F
:1005D0000AD801B10E6067B923B16FF000439842A9
:1005E00028BF1846BDE8F083A9F157095FFA89FCD6
:1005F000C4E723B1B0F1004F28BF4FF000404042A4
:10060000BDE8F08300279CE773B50E461049054608
:10061000FEF792FE18B93070012002B070BD2C7840
:10062000602C8CBF613C413C082C0FD80135012364
:100630000A2201A92846FFF76DFF019BAB4205D0B6
:100640000F2803D8013440EA0410E4E70020E4E76F
:100650009DCB060801230A2200215BE770B50D46F9
:100660001446FFF798F90646A0B1FFF7F3FF40F6EE
:1006700034039842A8BF1846B0F5617FB8BF4FF465
:100680006170A0F561731922B3FBF2F32B7023782C
:10069000013323703046FFF77EF90646A0B1FFF71D
:1006A000D9FF40F634039842A8BF1846B0F5617FE1
:1006B000B8BF4FF46170A0F561731922B3FBF2F378
:1006C0006B70237801332370304670BD2DE9F04103
:1006D00016461F460446394630464FF47A720023C8
:1006E0004BF02EFC3C4D3D4B054483FB05602844FC
:1006F000E917C1EB601183FB01030B44384EC817A7
:10070000C0EB631086FB003CC317364EC3EBAC0353
:1007100086FB03764FEAE37ECEEBE61EC1EB0116C5
:10072000A5EB860CC0EB0015A1EB8501617103EB15
:100730004301A0EBC10040F2B55101FB1E33B3F5FC
:10074000896F84F806C020714FEA8E0633DA40F2D2
:10075000DA218B4237DCB3F5B77FB4BF4FF0000E20
:100760004FF0010E204F0EEB4E0107EBC101754615
:10077000C88A4FEA4E0808EB0E0C07EBCC0C0CF1C4
:10078000160C0B2101E03CF8020D984210DD0139F6
:10079000F9D1F044012137F83800A170013306F592
:1007A000FA6E1B1A7544E37022812580BDE8F08142
:1007B0000131C9B2F1E703250B4F40F29650AE4626
:1007C0004FF00608D7E70225074F40F22940AE4612
:1007D0004FF00408CFE700BF80BC92C789888888A3
:1007E000ABAAAA2A73B06D163CF805080C4B10B5DD
:1007F000D3E9004354EA030209D1014640F2011350
:100800000020C1F8023088710880088110BD054AB7
:100810001268121943F10003FFF758FF012010BDC1
:10082000D8300020C01900202DE9F0410446944240
:100830001546084609D2B4FBF2F6154B05FB1644E3
:100840001B5D00F8013BBDE8F081B4FBF2F6964277
:10085000B6FBF2F70CD20E4B05FB176705FB1644EF
:10086000DA5D00F8012B1B5D00F8013BBDE8F0816B
:10087000BA42B7FBF2F807D9054B05FB187813F815
:10088000082000F8012BE7E74046FFF7CDFFF3E72C
:10089000005C060870B5884CB4F8D434B4F8D82499
:1008A000B4F8DC14B4F8DE04B3F57A7F88BF4FF4F3
:1008B0007A7382B088BFA4F8D434B4F8D634B3F5D0
:1008C0007A7F84BF4FF47A73A4F8D634B4F8DA345C
:1008D000B2F57A7F84BF4FF47A72A4F8D824B3F5C6
:1008E0007A7F84BF0023A4F8DA34B1F57A7F50D937
:1008F0004FF47A718842A4F8DC145CD89A429CBF09
:100900000023A4F8D83481429CBF0023A4F8DC342F
:10091000B4F8EC34B4F8EA24684D9A4284BF00235A
:10092000A4F8EA34664B1B8803B36979654E012944
:10093000B27848D9062A55D93179002940F09680F5
:100940009FED617A61490A7807EE903A06EE902AA7
:10095000F8EEE77AB8EEE66AB379C6EE276A002BBE
:100960007CD1B4EEE67AF1EE10FA49DC6A78032A1B
:100970001DD8574B03EB42132A78C4F8F434032AEA
:100980000ED8544BEA2102FB0133534A136002B0E4
:1009900070BDB0F57A7F84BF0020A4F8DE04ADE717
:1009A00000224C4B2A704C4A136002B070BD0022EA
:1009B000474B6A70E0E700219A42A4F8DE14A7D8FA
:1009C000A4F8D814A4E7B1790029B3D0072A61D0DC
:1009D000B3F57A6FAED93D4908780228B8BF022036
:1009E0000870A7E73D4901EB820191ED187A317952
:1009F0000029A7D0531F032BB8D9002AB6D03BE05B
:100A000027EE277AFCEEC77ACDED017A9DF8043007
:100A100007EE903AF8EEE77AB4EEE77AF1EE10FAE4
:100A2000C4BF0133DBB29BB3102BA8BF1023DBB2D2
:100A3000934238BF13460B7098E73279002A95D15C
:100A400022499FED277A0A7807EE903A06EE902A1F
:100A5000F8EEE77AB8EEE66AC6EE276A37EE077A6E
:100A6000B4EEE67AF1EE10FA80DDC9E7053A032A22
:100A70007FF67CAF9FED147AB7EE000A80EE070A8E
:100A80004CF080F93388834228BF034633806DE7FA
:100A90000123CCE70622B3F57A6FB270CDD90B49AA
:100AA00030790A78022AB8BF02220A7000287FF43F
:100AB0005DAF9FED0B7A46E720930020E0300020E9
:100AC00028130010802200206F12033830320020DB
:100AD000C893002048940020383200203CF80508D4
:100AE00017B7D1382DE9F04F8F4B83B01B78A3F1A6
:100AF0001702022A00AF00F2C3828C4E8C4C94F88D
:100B000000357B6004F5B06804F22C594FF0000A00
:100B1000D9F8005015F0010B40F07C8299F90430AF
:100B2000142B11D028464CF0F1FEAA0340F1648248
:100B3000012809D0082807DCBBF1000F00F06F8204
:100B40007C4B1D4240F05B827B497C4841F032FD8A
:100B50000023022084F8843514F078FC94F888355A
:100B6000774A022B156800F00683002800F05283B4
:100B7000DFF8E491734B94F8E1C5C7F804C003F5BE
:100B80006A7B4FF47A7A4FF0000E4FF0640833F826
:100B9000082CB2F57A7FB3F8462088BF23F808AC5A
:100BA000B2F57A7F33F8062C88BFA3F846A0B2F5D9
:100BB0007A7F33F8042C88BF23F806AC33F8061C80
:100BC000B2F57A7F84BF002223F804EC9142B3F897
:100BD0005A10B3F85C2098BF23F806EC914293F8C2
:100BE0006B2088BFA3F85AE0013A632A93F86C207F
:100BF00088BF83F86B800132D2B2092A88BF83F89C
:100C00006CE003F16501002213F8320011F801CF06
:100C10000132844538BF81F800E0032AF4D17A68B4
:100C2000012A18BF83F886E0EA339B45AFD1DFF88D
:100C30002CA19AF80230042B00F0CB8243B9BAF809
:100C40000030B3F5F07F84BF4FF4F073AAF80030A2
:100C5000FFF720FE3C4894F8F415FEF7A9FD94F840
:100C600013161030FEF7A4FDB4F82226B4F820368F
:100C70001343B4F8242613431BB213B10123A4F881
:100C80002636324B2B40002B00F0D182E80700F1D2
:100C90008C82690400F113822A0740F15A822C4A9F
:100CA000274B15401D60D9F800301340C9F80030BB
:100CB00015F4004300F03282002384F8073584F8ED
:100CC0001735E80440F1348294F83336DFF8848035
:100CD000022B04BF012384F8333608F1780B434616
:100CE00002E006339B450CD01A780A2AF9D199788C
:100CF000DA78914202D35A79002AF2D00A2022F0FF
:100D000019FC00234FF4806084F8843514F09EFBB6
:100D1000002800F073820F4979600D46687958B356
:100D2000297831B343461EE0643100203CF80508C1
:100D300020930020BC0202004C9800209CEF060883
:100D4000B836002052940020249900200960000247
:100D5000FE9FFFFD589900200C31002080220020CA
:100D600006339B4508D01A788242F9D15A79002A75
:100D7000F6D0084622F0DEFB0635AB45CED19AF818
:100D800002807968B8F1080F00F0E88194F8E13545
:100D9000D9F80000AB4DA3F10103B3FA83F35B096B
:100DA00084F8B03694F8E235A3F10103B3FA83F383
:100DB0005B0984F8B63694F8D134032B84BF002342
:100DC00084F8D134A04BC0F3C03293F80EC084F83D
:100DD000B3262B689D4A134002402B60C9F80020BF
:100DE000BCF1000F00F0E381994DAB88002B40F07F
:100DF000D281984A1368B3F5000F24BF0023136013
:100E0000936823F4007323F0020313B140F202232A
:100E100093601379013B042B84BF01231371A8F164
:100E200005088D4BB8F1030F93F8009040F26381F1
:100E30000025B9F1000F27D0DFF83C827D603E60CD
:100E400045464E46894606E0A8F10608A8EB0A0387
:100E50009E4240F23681A84615F8010F0028F3D0D3
:100E600009F092FE0028EFD083799B07ECD57D68CE
:100E70003E68494601223DB19AF8113053B99AF8BB
:100E80000530012B00D02AB19AF8063013B10023A7
:100E90008AF80630714BDA8802F00F00042803D874
:100EA000C2F30312022A02D94FF42062DA801A89AF
:100EB00002F00F00042803D8C2F30312022A02D959
:100EC00040F601221A8194F8C90694F8D52694F8C0
:100ED000C836904205D9002284F8C92653B1A4F837
:100EE000CC2694F8D4269A4204D2002384F8C8363B
:100EF000A4F8CC3694F8BE3794F8CA26DFF87CC143
:100F00009A4284BF002384F8CA360CF1800A6346F3
:100F100013F8032D02EB4202324492F8549192F8F6
:100F2000558192F856E113F8015F9879DA784D45CA
:100F3000A8BF4D464045A8BF40467245A8BF72466F
:100F400063451D709871DA70EDD103F1200CD44522
:100F5000DDD1D4F82425002A00F0308100250120BD
:100F60000B782B2B07D14B78043300FA03F3134291
:100F70001CBF9A43012506318B45F1D10DB1C4F850
:100F80002425374D6E4605F108082B4602E04345FF
:100F900000F09C8013F8012F072AF8D9002305F8E8
:100FA000013F0133082BFAD1B4F8DA25B4F8D8356B
:100FB0009A42B54602D32B4BC4F8D8352A4B2B4D59
:100FC000FF2284F8F02703F1540013F9082C142AA7
:100FD00005D053F80C1C35EA010100F0F7800C3302
:100FE0009842F2D1224B5A79022A01D100225A7139
:100FF0000C37BD46BDE8F08F01283FF79BAD09F1E6
:101000000C09C8457FF484AD0AF1FF32022A7FF64D
:101010009FAD99E50AF1010A5FFA8AFA82E56B064B
:101020007FF592AD15F4057F07D07A68A2F10F0322
:10103000012BE4D9531E062BE1D90E4BAB43DED076
:1010400082E500BFB8360020E0300020BCD455183F
:10105000EC31002040320020D011001090350020EB
:1010600092220020AE014A0158980020010002009F
:10107000342200204000020087220020CD9300206F
:101080006F4A12F8331081B9DB001A446D4E527862
:10109000002A3FF433AD334493F87C30002B7FF4C7
:1010A0002DAD694A1823137028E502EBC301DB005C
:1010B00049680029E9D1644817210170E5E7634ACE
:1010C000EEE57D683E6849460022D4E688B0E946F0
:1010D0002022FF2148464CF085FB5D4A04E0424552
:1010E00049F823303FF460AF12F8013F59F823105C
:1010F0000131F4D052E700238AF804300125B9F118
:10110000000F7FF499AE9AF81130002B7FF4C2AE35
:101110009AF80530012B7FF4BDAEB5E694F80725AB
:10112000002A3FF4CEADE80484F817353FF5CCAD86
:1011300029067FF5C9AD444B1A78182A04D8454BC7
:10114000D340DA073FF5C0ADDFF81C8108F1780B1A
:10115000D7E5AB047FF5ACAD3F4AA1E59AF8063080
:10116000002B3FF413AE9AF81130012B04BF022379
:101170008AF811300AE600283FF4FAAC90F904909E
:101180004FF0FF0A01E080F808A0484611F02AFC61
:101190000028F8D1ECE42878796009F0F5FC79684A
:1011A00000287FF426AEA88023E62C4A78E52C4858
:1011B000034302432B60C9F8002015E62B20796019
:1011C00022F0B8F9D4F824257968C7E684F8F02726
:1011D00008E7244B25F480551D60D9F8003023F42E
:1011E0008053C9F80030BAF82030B3F57A7FBFF4E5
:1011F0002FAD4FF47A73AAF8203029E5194A136805
:1012000023F000631360D9F8003023F00063C9F8BD
:10121000003080E5134BDFF8549025F080051D6009
:10122000D9F8003023F08003C9F80030A2E4D9F8DF
:10123000003043F0080345F00805C9F800302EE5FA
:1012400058F005083CF8050864310020F6DFFFFD82
:101250009222002000410001F6BFFFFDF79FFFFD35
:1012600000040500B8360020589900200C310020F9
:101270002DE9F04FDFF8EC816F4ED8F80C30DFF835
:10128000E89103F2DC534E4583B0C8F80C3080F08F
:10129000CF8001230193694BDFF8D0B106F11C0523
:1012A0009F1C664B5988002900F0AD807A185A457A
:1012B00080F0A9803C4608E0118814460A440029C1
:1012C00000F0A1805A4580F09E80052940F29B8065
:1012D00035F81C3C6188C3F30B039942ECD1637968
:1012E0009B07E9D155F8141C238894F804A00093B7
:1012F000304641F05FF935F81C1CBAEB113F00F0A5
:1013000088800023019335F8181C55F8140C55F803
:10131000044CC1F30B0145F06DFD1C364E452060B9
:1013200005F11C05BDD3464A464B474F474C126852
:101330001A60FFF7D7FB3878454D7A78454EEA2199
:1013400004F5947300FB01332B6004F1A80303EB55
:101350004213C4F8F43421F06DFB4FF0FF332868DA
:1013600073602AF097FE22F02DF904F5C76304F5A7
:10137000D66102E00633994255D01A78002AF9D195
:101380009D78D878854202D358790028F2D094F815
:101390003036327203EB830303EB83039B00642B31
:1013A000B4F83426B8BF6423C8F80430642303FBC0
:1013B00002F2642AB8BF64220023C8E90223C8F8F5
:1013C0002020254AA8F82430C8E90433C8E90633A8
:1013D00088F82630214B93622EF016FCB4F8F407FF
:1013E00094F8F61722F0EAFF39F086FD17F0B0FE08
:1013F0001B4A01981268C8F80C20012388F8253090
:1014000003B0BDE8F08F55F8141C304641F0D2F817
:1014100077E7009BA11D9A1F304641F001F9002893
:101420007FF471AF6DE7FA7B003A18BF0122AEE797
:101430000123019377E700BF50ED06080040000844
:10144000B83600200C310020E0300020209300202E
:1014500038320020FC0500201C17001040990020A5
:10146000C01900205032002010F606080080000845
:101470000121194A10B5032800EB0104034611703D
:10148000E4B218D9FF2825D0144A002341F20241C2
:1014900000E034B10233402B22F8021B04F1FF3488
:1014A000F7D10F4A1344FF2183F8F817BDE8104025
:1014B0000E200AF06DBB0B480B49EA2203FB020029
:1014C0000A4A0B7010602AF0E5FD26F0AFF926F00D
:1014D00091FAD9E70023E4E758170010189B002081
:1014E0002093002048940020E03000203832002073
:1014F000054BD3F83C28012142F4001283F8391837
:10150000C3F83C28704700BF20930020F8B5164D63
:101510006B78BE2B26D1022229464FF6FF70FDF7CD
:101520001DFE124FAC1C22884AB1A618BE4219D229
:10153000052A17D92146FDF711FE3446F3E7214667
:101540000222FDF70BFE0222A118FDF707FE06346A
:10155000074B641BA3F8404841F60F53C31A584287
:101560005841F8BD0020FCE700400008008000085A
:10157000209300202DE9F0410768C7F30D040646CB
:1015800088460CB3D8F8005041F04EF9092840F0D5
:101590008680454C236923F440732361236943F417
:1015A00000732361236943F0010323613D6041F02F
:1015B0003BF92369092823F0010323616FD13368C4
:1015C0000433336000206CE0384B394A93422BD30C
:1015D00002F58042934226D302F5804293424CD3D7
:1015E000344A93424BD902F58032934249D902F5ED
:1015F0000032934247D902F50032934245D902F5B1
:101600000032934243D902F50032934241D902F5A8
:10161000802293423FD9B3F1016F3ED3052048F0B9
:101620001DF947F08FFA082441F0FEF8092821D16E
:101630001D4D2B6923F440732B612B6943F4007318
:101640002B612B6923F0F8032B612B691C4344F0B9
:1016500002042C612B6943F480332B6141F0E4F8E0
:101660002B6923F002032B612B69092823F0F8036F
:101670002B6187D04FF0FF3013E01024D4E71824FB
:10168000D2E72024D0E72824CEE73024CCE7382442
:10169000CAE74024C8E74824C6E75824C4E76FF0E7
:1016A0000200BDE8F08100BF003C0240004000089D
:1016B00000400008FFFF00082DE9F041594E337843
:1016C000B12B8AB073D1FFF721FF80F00104E4B29F
:1016D000554B564DB3F86331554FADF8043004F017
:1016E0000104BD4265D3002C00F099800023CDE9B0
:1016F000073309934F4B05969B1B06934E4B1A6974
:10170000002A04DA4D4A5A6002F188325A600122F6
:101710008DF82520F322DA6001A9022205A84FF0F6
:1017200000088DF8248049F055FD022201A94FF6EA
:10173000FF70FDF713FD3D4D0446BD4247D3022225
:1017400002A905A80025ADF8085049F043FD022282
:1017500002A92046FDF702FD40BAC043ADF80C00D7
:10176000022205A803A949F035FD089878B107AB16
:10177000C0F10402294618444CF034F89DF92400C5
:1017800018B907A905A8FFF7F5FE8DF824009DF804
:10179000253023B1284A136943F0004313619DF9B2
:1017A0002400B0FA80F040090AB0BDE8F0810124BD
:1017B0008EE7A988AB69A868D3F80080C1F30B0154
:1017C00045F018FB1C35804518BF012489E7AE8819
:1017D0008DF81180C6F30B06B31DADF80C302B88C5
:1017E000C3F30B02ADF80E201B0B062203A905A8BC
:1017F0008DF8103049F0EEFC062203A92046FDF7D3
:10180000ADFCA9680446324605A849F0E3FCA96886
:1018100020463246FDF7A2FC1C3504468DE7012028
:10182000C2E700BF004000083CF8050850ED06087C
:1018300010F6060800800008003C024023016745BE
:10184000F8B5184D184E194FFFF74CF9EB68012207
:1018500003F2DC53EB6086F842280324FFF72CFFE9
:1018600058B13B78B12B08D1FFF750FE013C0BD0AB
:1018700060B9FFF721FF0028F3D1013CEED105202C
:1018800047F0ECFF47F05EF90028F8D0084A1168ED
:10189000E9600122002385F8252086F8423886F881
:1018A0004338F8BD5032002020930020004000084B
:1018B000C019002008B50B490B4A01230B70937324
:1018C000FFF7BEFFFFF7D4FC084B41F20241FF22B5
:1018D000A3F8F81783F8FA27BDE808400E200AF0AD
:1018E00057B900BF58170010E030002020930020A7
:1018F00090F89230DFED6B6A6B4A07EE903A90F801
:10190000963005EE103A90F8943004EE903A90F844
:10191000953005EE903A90F89830F8EEE77AB8EE08
:10192000C55A04EE103A67EEA67A25EE265AF8EE6E
:10193000E44AF8EEE55AB8EEC44A25EE275A64EEBA
:10194000A64A65EEA65A24EE264AF0B5B7EE007A0E
:1019500090F8917064EE854A65EEA75A24EE274A06
:1019600000F16F06014602F11A050024B0EE476A45
:10197000B0EE473A137807EE903AF8EEE77A67EE62
:10198000857A67EE867AFDEEE77A17EE903AFA2BC3
:10199000A8BFFA2323EAE3730B72537807EE903A59
:1019A000F8EEE77A67EEA47A67EE867AFDEEE77ADC
:1019B00017EE903AFA2BA8BFFA2323EAE3734B728F
:1019C000937803EE903AF8EEE33A63EEA57A67EE89
:1019D000877AFDEEE77A17EE903AFA2BA8BFFA2342
:1019E00023EAE3738B72938807EE903AF8EEE77A76
:1019F00067EE847A67EE867AFDEEE77A17EE903A24
:101A0000B3F57A7FA8BF4FF47A7323EAE3738B812F
:101A10002B68D5ED007A002BF8EEE77A3FDD90F8E1
:101A2000973002EE903AF8EEE22AB0EE436AA2EE68
:101A3000E66A63EE863A83EEA76AA2EEA66A0134EE
:101A400065EEA77A67EE877A67EE867AFDEEE77A2B
:101A500017EE903AFA2BA8BFFA2323EAE373BC42AD
:101A600006F8013F00DDF0BD012C13D190F8933052
:101A700007EE103A90F89B3006EE103AB8EEC77AAF
:101A8000B8EEC66A27EE267A26EE266A04350832B4
:101A900008316FE7B7EE007AB0EE476AF6E7B7EEC7
:101AA000006ACCE70AD7233CA2F9050890F89930E0
:101AB0006BB3B0F864308BB190F89A2002EB8203DC
:101AC0006421C3EB0313B3FBF1F3A0F86430962356
:101AD00012FB03F3B3FBF1F3A0F8663043884BB17C
:101AE00090F89A3003EB8303C3EB03136422B3FB38
:101AF000F2F34380B0F850304BB190F89A30962210
:101B000013FB02F36422B3FBF2F3A0F850307047EA
:101B100090F821304BB3438B83B190F82230FA22F6
:101B200013FB02F203EB8303B3F57A7FA8BF4FF4F4
:101B30007A7364218383B2FBF1F24283838843B1D9
:101B400090F82230FA2213FB02F36422B3FBF2F383
:101B50008380C3884BB190F8223003EB8303B3F545
:101B60007A7FA8BF4FF47A73C380704770B50B4C6F
:101B7000002504F56A7694F8913013B12046FFF7FA
:101B8000B7FE2046FFF792FF01353046FFF7C0FF52
:101B9000042D04F1EA04EED170BD00BF489400208A
:101BA00010B5064C4FF48072002104F644004BF04F
:101BB00019FE0023C4F8443910BD00BF2093002053
:101BC000034BD3F8480908B107F01CBD704700BFAC
:101BD0002093002008B50B4605490246D1F8480974
:101BE00028B10449FEF714FABDE80840E8E708BD4B
:101BF00020930020C5F80008024B0146D3F848099D
:101C0000FDF762BE209300200048F5E778E1060862
:101C10000CB4C30607B500D561B9049805A90191B4
:101C2000FFF7D8FFFFF7F0FF012003B05DF804EBEA
:101C300002B070470020F8E70FB407B504A951F8C7
:101C4000040B0191FFF7C6FFFFF7DEFF03B05DF85D
:101C500004EB04B070470349034801F521610EC944
:101C6000EAE700BF0070FF1F64CC060870B5134C94
:101C7000134D144E002294F8F33403F0010302B123
:101C800070BD002BFCD001212846FFF7D5FF752041
:101C90002EF056FA01463046FFF7CEFF1A202EF0FE
:101CA0004FFA01460848FFF7C7FF1B202EF048FAFD
:101CB00001460648FFF7C0FF0122DCE72093002021
:101CC00078CC060884CC060897CC0608AACC06086F
:101CD00008B5FFF791FFBDE8084095E72DE9F0430F
:101CE00085B0FCF793FC02698389018802928268BF
:101CF00001924288009242681B4EDFF88080DFF834
:101D000080901A4F04461A48FFF796FF002515B930
:101D10001848FFF7DDFFD8F800309D4213DA33781A
:101D2000052B96BF09EB83030022D3F88C21B388DF
:101D300000937388294638460135FFF77DFF062D4D
:101D400006F10606E3D145F041FD428883886468C8
:101D50009B1A03FB0444FCF7F1FC024606482146AB
:101D600005B0BDE8F04367E76C9C002027CD06086E
:101D7000BDCC06081BCD060836CD06087C2B0020FE
:101D80003CF8050810B504460348FFF735FF204628
:101D9000BDE810409CE700BF53CD060808B50346D8
:101DA00010460AB9002008BDDB0601D50029FAD08B
:101DB000FFF7E8FFF6E72DE9F04F0A468DB0002166
:101DC0008346FFF7EBFF714CDFF8CC91039004F1F1
:101DD000800A0025A37A99F80060AB4200F3938053
:101DE00010345445F5D140F2162040F0CDFBD0E937
:101DF00002450DF1180A002E4FF015024FF00001B8
:101E0000504604BF254634464BF0ECFC00272E78A4
:101E1000002E3ED069780591304608F08DFE95F988
:101E20000290049009F1010253425341002C00F04A
:101E3000A98005990022A05CB04240F09F80224416
:101E400092F90280C14540F0978052788A4208BFDB
:101E5000012301220AF8072003F0010383F00101A6
:101E6000039A05935846FFF799FF059B039044B1E9
:101E7000474A0499CDE900B230464246FDF710FECC
:101E8000059B444A0499CDE900B230464A46FDF725
:101E900007FE0137152F05F10305B8D184B3DFF82C
:101EA000F080DFF8F090564604F13F0716F801ABDA
:101EB000BAF1000F21D12078F8B194F90230013342
:101EC0001BD0617808F038FE039A05460121584678
:101ED000FFF764FF94F902200390534620782946C7
:101EE000CDE900B8FDF7DCFD20785346CDE900B917
:101EF0004FF0FF322946FDF7D3FD0334BC42D5D164
:101F00000DB0BDE8F08FE08840F03EFBD0E9023133
:101F1000627A207A002E08BF194605FB002208BF0E
:101F200033468F562BB39E56039A0493B74214BF81
:101F30000121002158460CBF4FF001084FF0000866
:101F4000FFF72CFF049B039043B1114B3246CDE9C0
:101F500000B3294643462046FDF75EFD0D4B29465A
:101F6000CDE900B33A4643462046FDF755FD01351D
:101F700030E74FF0FF36D7E700236AE703323F2A06
:101F80007FF459AF4FF0FF3868E700BF0806002024
:101F900015210108111C01082093002010B50846E6
:101FA0000749FDF7C9F9002815BF01240024054899
:101FB0000548FFF7E7FE2046BDE8104007F004B9EA
:101FC00058CD060861CD060888CD06082DE9F04FEA
:101FD00007468BB040F216200C4640F0D5FA224658
:101FE000054600213846FFF7D9FE424BD5E90245A8
:101FF0001B78002B08BF254606464FF015024FF010
:10200000000104A808BF1C464BF0ECFB05F13F03A0
:10201000039395F80090B9F1000F31D095F801A025
:10202000002C65D0224600231178494558D1283329
:102030006B4492F80180012203F8182CD0453246F7
:1020400014BF0121002138460CBF4FF0010B4FF0A7
:10205000000BFFF7A3FE064654B1B8F1000F07D0FE
:10206000254B00935A463B4641464846FDF75EFDE8
:10207000224B00935A463B4651464846FDF756FDD3
:10208000039B03359D42C4D13CB3DFF86C90DFF86D
:102090006CA0651C0DF11008403418F8013BCBB959
:1020A00015F8013CB3B116B13046FFF76BFE297845
:1020B00015F8010CCDF800903B460022FDF736FDE7
:1020C000002215F8010CCDF800A03B461146FDF7A3
:1020D0002DFD00260335A542DFD10BB0BDE8F08F02
:1020E0000133152B02F103029ED14FF00008A5E742
:1020F000A046A3E72093002015210108111C010828
:10210000034B0146D3F8480908B107F067BA704796
:10211000209300200CB407B510F020000BD079B943
:102120002320FFF7EDFF049805A90191FFF752FD69
:10213000FFF76AFD012003B05DF804EB02B07047C1
:102140000020F8E72DE9F04F914687B00C461A467B
:1021500000218046FFF722FE4D4606460027B9F1D2
:10216000000F66D02946062220464BF0BFFB002810
:10217000324614BF0121002140460CBF4FF0010A36
:102180004FF0000AFFF70AFE0646287816F0A8FF6F
:102190008346F8B1687916F0A3FFAB78EA789BF82C
:1021A00005E095F801B04FF461714FF0190C1CFB7C
:1021B00003131CFB0212297900B14079CDE9041008
:1021C000CDE90232CDE900EB1B4A3B465146404681
:1021D000FFF7A0FF207816F083FF8346F8B16079FF
:1021E00016F07EFFA378E2789BF805E094F801B042
:1021F0004FF461714FF0190C1CFB03131CFB02120E
:10220000217900B14079CDE90410CDE90232CDE960
:1022100000EB094A3B4651464046FFF7F9FC0137BF
:10222000142F04F1060405F1060598D107B0BDE8A6
:10223000F08FCA46CEE700BFA4CD06082DE9F04FC7
:10224000904689B01A460C4600218146FFF7A6FD4C
:102250003B4EDFF8F0B008F15403074645460793BC
:1022600094F9040010F0BEFB00285DD0B8F1000F17
:1022700063D029460C2220464BF038FB00283A4612
:1022800014BF0121002148460CBF4FF0010A4FF056
:10229000000AFFF783FD074695F9040043F08EFE20
:1022A000EA7906EB82020346D2F8A42104922A7A44
:1022B00006EB82025146D2F8A4210392AA7906EBDA
:1022C00082024846D2F8A42102926A7906EB820281
:1022D000D2F8A42101922A6800925A46FFF71AFF09
:1022E00094F9040043F06AFEE27906EB82020346A9
:1022F000D2F8A4210492227A06EB82025146D2F847
:10230000A4210392A27906EB82024846D2F8A421C6
:102310000292627906EB8202D2F8A421019222682D
:1023200000925A46FFF774FC079B0C35AB4204F150
:102330000C0495D109B0BDE8F08FC246D0E700BFCC
:102340003CF80508BDCD06082DE9F04F90468BB04E
:102350000C461A4600210746FFF720FD4546099026
:1023600000264FF0190A4FF46179B8F1000F4BD0F5
:1023700029460A2220464BF0B9FA0028099A14BFD0
:102380000121002138460CBF4FF0010B4FF0000B2C
:10239000FFF704FD2A890692EA8805922A790492B9
:1023A000EA780392AA7809901AFB029202926A785C
:1023B0001AFB029201922A7800923346134A594638
:1023C0003846FFF7A7FE22890692E2880592227915
:1023D0000492E2780392A2781AFB02920292627847
:1023E0001AFB0292019214F80A2B00923346074A14
:1023F000594638460136FFF70BFC1E2E05F10A053B
:10240000B3D10BB0BDE8F08FC346DCE7DACD0608E8
:102410002DE9F04F2DED088BDFF828A195B080460F
:1024200091461E460C461546002794ED008AB5EEEF
:10243000408AF1EE10FA7DD0D4ED019A94ED029A23
:10244000D4ED038AB9F1000F49D0D5ED00BA95ED6E
:1024500001BAD5ED02AA95ED03AAB4EE6B8AF1EEAE
:1024600010FA6CD1F4EE4B9AF1EE10FA67D1B4EE9B
:102470006A9AF1EE10FA62D1F4EE4A8AF1EE10FA9D
:102480000CBF0121002132468B46404681F00101FC
:10249000FFF784FCB0EE6B0A064611A8FDF7A2F91F
:1024A000B0EE4B0A07900EA8FDF79CF9B0EE6A0A51
:1024B00006900BA8FDF796F9B0EE4A0A059008A819
:1024C000FDF790F90599069A079B039002910192F6
:1024D000009352463B4659464046FFF71BFEB0EE7E
:1024E000480A11A8FDF77EF9B0EE690A83460EA8E6
:1024F000FDF778F9B0EE490A06900BA8FDF772F9DE
:10250000B0EE680A059008A8FDF76CF9069B059ADD
:102510000390CDE900B302923B465246002140466B
:102520000137FFF775FB082F04F1100405F11005C2
:102530007FF47BAF15B0BDEC088BBDE8F08F0021B8
:10254000A1E700BFFDCD06082DE9F74F92460C46E6
:102550001A4600218146FFF721FCDFF870B0804663
:1025600056460025BAF1000F2ED0314604222046EF
:102570004BF0BCF90028424614BF01210021484617
:102580000CBF01270027FFF709FC738801933AF875
:102590002530009380462B465A4639464846FFF779
:1025A000B9FD6388019334F8043B00935A462B46E7
:1025B000394648460135FFF72BFB042D06F104068A
:1025C000D0D103B0BDE8F08F5746EAE711CE060838
:1025D0002DE9F04F89468FB0174600211A4606466E
:1025E000FFF7DCFBDFF874A0054600240DF1240B97
:1025F00059F82480CDF80880594602A843F08CFC95
:1026000057B357F82430039398452A4614BF012145
:10261000002130460CBF4FF001084FF00008FFF7D3
:10262000BDFB04A9054603A843F076FC04A900916C
:102630002346524641463046FFF76CFD2346CDF80F
:1026400000B05246414630460134FFF7E1FA202CF3
:10265000CED10FB0BDE8F08FB846EFE722CE060826
:102660002DE9F04F924685B00C461A46002181466E
:10267000FFF794FBDFF874B0804655460026BAF1A8
:10268000000F31D02946042220464BF02FF90028B4
:10269000424614BF0121002148460CBF01270027F4
:1026A000FFF77CFBEB780293AB7801932B880093C8
:1026B000804633465A4639464846FFF72BFDE378B5
:1026C0000293A378019334F8043B00935A463346AF
:1026D000394648460136FFF79BFA102E05F10405EE
:1026E000CDD105B0BDE8F08F5746E8E72CCE0608FF
:1026F0002DE9F04F85B0144602911A460021054697
:10270000FFF74CFB4FF000080646062303FB08F7D3
:10271000C0374FF00009029B13F807B0002C7ED0A1
:10272000E35D03939B45324614BF012100212846F7
:102730000CBF4FF0010A4FF0000AFFF72FFB039B7D
:10274000394ACDE900930646434651462846FFF7ED
:10275000E1FCCDE9009B344A43465146284609F145
:102760000109FFF755FAB9F1060F07F10107D2D1B8
:1027700008F10108B8F1060FC7D1E427029BA7F1C1
:10278000E40913F807A0002C4BD014F807B0DA4581
:10279000324614BF0121002128460CBF4FF001082A
:1027A0004FF00008FFF7FAFACDE9009B06461E4AF3
:1027B000062341462846FFF7ADFCCDE9009A1A4AA8
:1027C0000623414628460137FFF722FAEF2FD5D1DD
:1027D000029B93F8EF70B4B194F8EF80474532460E
:1027E00014BF0121002128460CBF01240024FFF75B
:1027F000D5FA002300930C4ACDF804800723214624
:102800002846FFF787FC00230093074A0197072318
:1028100021462846FFF7FCF905B0BDE8F08FA24637
:1028200097E7A046C9E700BF3ECE06082DE9F04F66
:102830000E46154689B01A4600210446FFF7AEFA47
:10284000B04681462F464FF0000B002D7CD0394614
:102850000C2240464BF04AF800284A4614BF01219A
:10286000002120460CBF4FF0010A4FF0000AFFF78D
:1028700095FA97F90B20049297F90A200392B7F979
:1028800008200292B7F906200192B7F904200092BD
:102890008146384A5B4651462046FFF73BFC98F993
:1028A0000B20049298F90A200392B8F908200292AA
:1028B000B8F906200192B8F9042000925B462D4A2F
:1028C000514620460BF1010BFFF7A2F9BBF1080FAF
:1028D00008F10C0807F10C07B7D1DFF89C804FF026
:1028E000000B0C2303FB0BF985B3002755F80900F7
:1028F00056F80920012303FA07FA42403AEA020295
:1029000014BF1946002110EA0A0F07D000975B4652
:10291000424620460791FFF7FDFB079956F809202C
:102920001AEA020F05D000975B4642462046FFF7A1
:102930006FF901370E2FD9D10BF1010BBBF1080F45
:10294000CFD109B0BDE8F08FAA46A8E72F4656F8C8
:102950000910012303FA07F20A4206D000975B46EA
:10296000424601212046FFF753F901370E2FEED1E1
:10297000E2E700BF52CE06086ACE06082DE9F04F06
:1029800089468DB0164600211A460746FFF706FA1B
:10299000DFF8DCA005460024C4EBC40309EB030206
:1029A00059F8030091889279089040F30748ADF8F0
:1029B00024108DF82620B8F1000F54D0002E55D0E9
:1029C000F218F058918893790A90ADF82C100722EC
:1029D0000AA908A88DF82E304AF088FF00282A4658
:1029E00014BF0121002138460CBF4FF0010B4FF0FE
:1029F000000BFFF7D3F99DF82E3006939DF92D308B
:102A000005939DF92C3004939DF82B3003939DF989
:102A10002A3002939DF8293001939DF828300093C5
:102A200005462346524659463846FFF773FB9DF844
:102A3000263006939DF9253005939DF924300493A3
:102A40009DF82330CDE902839DF8213001939DF854
:102A50002030009352462346594638460134FFF74A
:102A6000D7F8102C98D10DB0BDE8F08FB346DEE753
:102A70007FCE06082DE9F04F924689B00C461A46E3
:102A800000210746FFF78AF9002607905546B3460E
:102A90004FF019094FF46178BAF1000F28D0294698
:102AA000062220464AF022FF0028079A14BF01217F
:102AB000002138460CBF4FF0010B4FF0000BFFF721
:102AC0006DF96A79079019FB028205922A7919FB40
:102AD00002820492EA780392AA7802926A780192BA
:102AE0002A7800923346124A59463846FFF712FBBD
:102AF000627919FB02820592227919FB0282049203
:102B0000E2780392A27802926278019214F8062B7E
:102B100000923346064A594638460136FFF778F8A0
:102B20000A2E05F10605B7D109B0BDE8F08F00BF48
:102B30009CCE06082DE9F04F0F468BB014460021BD
:102B40001A460646FFF72AF90546002C00F0DD80FC
:102B500022783B789A4218BF0121024608BF002123
:102B600030460CBF4FF001084FF00008FFF716F990
:102B700023789E4A054641463046FFF7CBFA3B781C
:102B80009A4A41463046FFF743F8002C00F0BF80D8
:102B900062787B789A4218BF01212A4608BF00213B
:102BA00030460CBF4FF001084FF00008FFF7F6F871
:102BB00063788F4A054641463046FFF7ABFA7B788B
:102BC0008B4A41463046FFF723F807F1C9030593C6
:102BD000A31C0693822307F1020A04F1CA0B079390
:102BE0004FF000093B784B4500F39380002C00F038
:102BF000F68097F8EA3094F8EA209A4218BF01214B
:102C00002A4608BF002130460CBF4FF001084FF0A4
:102C10000008FFF7C3F894F8EA30764A05464146C3
:102C20003046FFF777FA97F8EA30724A4146304665
:102C3000FEF7EEFF002C00F0D48004F1EA0307F168
:102C4000EA0204F1FA014FF0010833F802CF32F83A
:102C5000020F844518BF4FF000089942F5D188F063
:102C600001012A46C9B23046FFF798F80821054607
:102C700004F1EC00FDF760FB5F4A03464146304635
:102C8000FFF748FA97F8EA1007F1EC00FDF754FB5C
:102C9000594A034641463046FEF7BAFF002C00F081
:102CA000A2804FF0FC094FF0010807EB090104EB8B
:102CB0000900FCF741FB09F10409002818BF4FF097
:102CC0000008B9F58E7FF0D188F001012A46C9B21B
:102CD0003046FFF763F8082104F1FC00FCF76EFEB4
:102CE000464A034641463046FFF714FA97F8EA1081
:102CF00007F1FC00FCF762FE404A034641463046BD
:102D00000BB0BDE8F04FFEF783BFA04637E7A04603
:102D100055E7079BFB180993002C5ED0079B099889
:102D2000E31819460893FCF707FB059B5A789BF8B4
:102D300000309A42069A06BFB0FA80F84FEA581857
:102D40004FF00008AAF10203023A0AF10E0133F82B
:102D500002CF32F8020F844518BF4FF000088B42B3
:102D6000F5D188F001012A46C9B23046FFF716F8BE
:102D70006278069905469BF81800FDF7AFFA0290B5
:102D80009BF800300193089B00931D4A09F1010351
:102D900041463046FFF7BEF9059B7A78587E51468A
:102DA000FDF79CFA059A029012F8013F019309F190
:102DB0000109099B05920093114A4B464146304652
:102DC000FEF726FF069B10330693079B09330AF193
:102DD000100A0BF1010B079304E7A046DCE7A046BD
:102DE00021E7A0464EE7A04680E700BFB5CE060823
:102DF000C7CE0608F5CE06080DCF060824CF060874
:102E0000DCCE06082DE9F04F89B00F469046002130
:102E1000139A03930646FEF7C1FF87EA08086FEA94
:102E20000803DFF8849006930446002528460FF037
:102E300069FD129B184230D0069BDFF870B003404A
:102E400014BF4FF0010A4FF0000A049310EA070381
:102E50000CBF4A465A462846059307920FF064FD78
:102E6000039B079A0090804651463046FFF752F97F
:102E7000049BB3FA83F1224649093046FEF78EFFE0
:102E8000059A039BCDF800800446002A0CBF5A46E1
:102E90004A4651463046FEF7BBFE0135172DC5D1D7
:102EA00009B0BDE8F08F00BF3BCF06080BCE060887
:102EB0002DE9F04F0A4689B000210546FEF76EFF66
:102EC000384C059094F9000006F0FEFD81466088BC
:102ED0003FF05AFB344BD0F808B01F7817B15F466B
:102EE000D0F80CB0A379012B38BF0123069300263C
:102EF0002279637906FB02331BF80380002F3BD055
:102F0000FB5C059A0793434514BF01210021284625
:102F10000CBF4FF0010A4FF0000AFEF73FFF079B7E
:102F20000590013653B303F00F021B094033CDE97E
:102F3000006302924B461D4A51462846FFF7EAF8C5
:102F4000B8F1000F24D008F00F034FEA18180293CD
:102F500008F14003CDE90063144A4B465146284628
:102F6000FEF756FE069BB342C2DC114B0834A34267
:102F7000A8D109B0BDE8F08F3B46C2E7002FDFD0F3
:102F80000C4A00964B4651462846FFF7C3F8D7E750
:102F90006B06E7D4074A00964B4651462846FEF793
:102FA00037FEDFE720FA05082093002042CF06080D
:102FB00020FB050858CF06080FB407B504A951F83F
:102FC000040B0191FEF706FE03B05DF804EB04B0BC
:102FD00070472DE9F041037903F0E002402A4DD01B
:102FE00009D83ABB03F00703052B1ED8DFE803F02E
:102FF000181D181D0910602A47D0802A41D0BDE84D
:10300000F081D0F805102348BDE8F041FEF714BE6A
:10301000D0F8052051422048BDE8F041FEF70CBE33
:10302000B0F80720B0F80510F5E7B0F90720B0F9BF
:103030000510F0E74679194D194805EBC605FEF76E
:10304000DBFD95F8E87200240123A74203D8BDE810
:10305000F041FEF7D9BDD5F8E46256F824204FEAD6
:1030600084084AB113B90F48FEF7C6FD56F8081098
:103070000D48FFF7A1FF00230134E6E741790B4833
:10308000C2E7827941790A48C6E7BDE8F0410948BC
:10309000FEF7D2BD6CCF060882CF06083CF80508C3
:1030A00099CF060830D1060838E60608AACF0608E8
:1030B000BBCF0608D2CF0608194B1B682DE9F0419B
:1030C00063B31848184FDFF86880FEF701FEFEF77B
:1030D00077FDFBF7ABFA0025FBF7E8FA044648B1A9
:1030E000132008F055FDFEF78FFDBDE8F0410F48B5
:1030F000FEF7EEBD3B78012BF2D04046FFF75CFFB8
:10310000792D05F1010602D1FEF77EFD2646FEF778
:1031100057FD6420F7F7E2FC3546DDE7BDE8F081B6
:103120002C200020EACF0608862B002004D00608B9
:1031300002E706082DE9F047B64BB7491A68B748C9
:10314000B74BB2FBF3F296B0FFF736FFB54BDFF8A3
:103150009CC30FCBDCF808700AAD85E80F00390777
:1031600048BFDCF80440B04B05934FEA970EAF4BD5
:10317000069348BFC4F3805416AB1EF0020F18BF6D
:1031800003EB8404C7F3810603EB860618BF54F8EB
:10319000442CA74C08BFA74A56F8301CA648A74D98
:1031A000A74FFFF709FFB4F870294FF47A73B2FB09
:1031B000F3F103FB11220A20B4F9723992B2B2FB87
:1031C000F0F2A048FEF738FD9F4AA049A048FFF75B
:1031D000F3FEFEF719FD9F4B9F4A997B9F4BA0483A
:1031E00005EB8101D31AD1F8B414B4F84028FEF7E6
:1031F00023FDFEF709FD9B48FEF7FEFC94F87419C9
:103200009948FFF7D9FE9948FEF7F6FC984B94F8D9
:1032100075191A88974892B2FFF7CEFEFEF7F4FCB4
:1032200095499648FFF7C8FE4FF000084646DFF87C
:10323000C09294F8EF3403F00103B8F1000F00F0EE
:103240005B81002E40F08C818D48FEF741FD8D4F53
:10325000D4F87C89DFF89C92012607F1180A012333
:10326000B34013EA080F15D019F8062057F8263096
:103270005AF8261053F822208348FFF79DFE012EAE
:1032800006D1824B93F8211011B18148FFF794FECB
:10329000FEF7BAFC0136062EE1D17E48FEF7ACFC03
:1032A0007D4B1B681B0640F18F8194F89C39032BE2
:1032B0008CBF7A487A48FEF79FFC94F88835022B39
:1032C00040F051817748FEF797FC94F89C39042B25
:1032D00000F271817448FEF78FFC94F8AC39002B32
:1032E00000F0708105EBC303D3F850156F48FFF76A
:1032F00063FEFEF789FC6E4B6E481E686E4B1B78B2
:1033000005EB8303D3F88415FFF756FE26B1327A16
:10331000717A6A48FFF750FEFEF776FCFBF776F904
:10332000016921B182686648120DFEF785FCFEF73F
:103330006BFC644B644819684FF47A73B1FBF3F18A
:10334000FFF73AFE07A8FDF751FA38B107A90EA812
:1033500048F05EF85D480EA9FFF72EFEFEF754FC1C
:10336000D4F8388AB8F1000F00F0328107EE908A65
:10337000DFED576AB8EEE77AC6EE877AFDEEE77AB8
:1033800017EE903A534F17F8080C30B1524A039396
:1033900092ED250A49F0F6FC039BD4F8B8695EB1BA
:1033A00007EE906ADFED4A6AF8EEE77A86EEA77AD2
:1033B000FDEEC77A17EE906A344AB2F870106429AD
:1033C000A8BF6421CDE9000642464448444EFEF7BA
:1033D00033FC37F8042C43486423B2FBF3F103FBBE
:1033E00011227B7B05EB830592B2D5F898350093CB
:1033F0003B7BFEF721FC3C48FEF7FEFBD4F83C4843
:103400000125002C40F0E680FEF7FEFB16B0BDE87B
:10341000F08700BFB41A002012D006081CD006089E
:1034200040420F00E0FC05082ED0060833D0060805
:10343000209300207AE1060838D006083CF80508F9
:103440002813001040D00608F0FF0010000800000C
:1034500062D00608E030002000800008004000082C
:1034600074D006088BD006089DD00608A5D00608A3
:1034700060230020A7D00608BBD00608C0D00608ED
:10348000DFD0060858FD050853DE0608581700105F
:10349000E4D00608E8D006080C310020EED006087B
:1034A000FAD006080AD106080BE806084ED106082D
:1034B000083600206AD106080436002073D10608B9
:1034C0007DD10608C019002098D10608B2D106089F
:1034D0000024744918A40020FC050020C5D106086A
:1034E0005AD106080BD2060830D20608003802402E
:1034F00030D1060888060020002B3FF4A2AE16B19A
:103500004846FEF779FB3B480121FFF755FD94F84B
:103510007839394805EB8303D3F8BC14FFF74CFD29
:1035200097F8CE33DA0702D53448FFF745FD97F810
:103530001831032B09D03248FFF73EFD97F81831B8
:10354000012B02D12F48FFF737FDFB6C5B7B012677
:10355000B342B0467FF66DAE2B48FFF72DFD66E611
:10356000FEF752FB73E6022011F090FF064608B901
:103570002648A8E690F9040042F020FD074637F0FF
:10358000A5FC05EB80003946D0F8A4212048FFF7C0
:1035900013FD94F88B35012B04D11E48FEF72CFB4C
:1035A0001D4890E6B3791D4805EB8303D3F8A411B9
:1035B000FFF702FDF4E794F88A350BB918488AE65C
:1035C000184888E6184991E61848FEF715FB90E67A
:1035D0004346D7E694FAA4F0B0FA80F005FA00F07A
:1035E00024EA000408F0BAFA01463046FFF7E4FC8A
:1035F00007E700BFC5D006085AD106082CD6060832
:10360000CAD00608D2D00608D7D0060810D10608BE
:103610001AD106082AD106082FD10608D6CD0608E9
:1036200033D1060843D106080AD006085ED1060841
:103630002DE9F04FDFF86C8198F8033099B0002B3A
:1036400000F092804E484F4EDFF85CB1DFF85C919D
:10365000DFF85CA1FEF73CFB00252F460BA9E8B282
:1036600015F0F4FF9DF83430002B53D0139C54B167
:1036700007EE904A9FED440AF8EE677A80EE270A3B
:1036800049F080FB04460B9A29465846FFF794FC04
:10369000109A002A6AD002FB04F04FF47A73B0FB50
:1036A000F3F30993DDF848C0BCF1000F60D00CFBC8
:1036B00004F142F21073B1FBF3F198F80330082DD6
:1036C00018BF7F18002B55D01798079015980690B3
:1036D000169805900A2311984FF47A7EB0FBFEFEEF
:1036E0000998CDF810E0B1FBF3FE03FB1E11CDE904
:1036F00002E10999B1FBF3F103FB1100CDE90010E0
:10370000BCFBF3F321465046FEF796FA0023C6E9C8
:103710000D33B36201351D2D06F140069ED198F898
:103720000330F3B1194C1A48D4E904124FF47A73F8
:10373000D208B1FBF3F3A169FEF77EFA0A2215481D
:1037400097FBF2F102FB1172FEF776FA124B1B782F
:10375000432B04D1D4E907211048FEF76DFA00236A
:10376000A36119B0BDE8F08F0D486CE7099299E7A5
:103770006146A2E721464846FEF75EFAC6E700BF6B
:1037800046D20608D09C00208096184B18A4002032
:10379000EDD206080DD306081622002031D3060804
:1037A000A4D20608E0300020AED20608DAD506081A
:1037B000BDD2060810B586B0104B0493104B03938E
:1037C000104B0293104B0193104B1149114A009377
:1037D0000446114B1148FFF7EFFBFEF715FA1049AD
:1037E0001048FEF729FA3CB10F4A1049104806B0BC
:1037F000BDE81040FEF720BA06B010BD9BD3060806
:10380000A0D30608ABD30608B4D30608C0D3060875
:1038100065D306085BD30608E730002070D306089E
:10382000CAD30608D2D30608E3D30608F2D30608A3
:10383000F7D306080120BDE770B52348FEF7DCF991
:10384000224B13F8083C002B38D0214B93ED250A6E
:1038500049F098FA01461F48FEF7EEF91E4C1F4842
:10386000FEF7CAF91E4B94F819051E4A00280CBF32
:1038700010461846FEF72CFA94F8193513B31A4C73
:103880001A48B4F806111A4E1A4DFFF795FB94F832
:10389000040100280CBF30462846FEF719FAB4F898
:1038A00008111548FFF788FB94F8050100280CBFA4
:1038B00030462846BDE87040FEF70ABA0F48FEF7CA
:1038C00007FACBE770BD00BF34D4060818A4002067
:1038D000FC0500204ED40608209300205DD4060885
:1038E000E7CF0608D7EC0608581700106ED4060874
:1038F0002DD4060824D4060895D4060853D4060807
:1039000038B50B4D05EBC0050C4695F9E40106F002
:10391000DBF801460748FFF74FFB95F8EA3133B172
:10392000611C0548BDE83840C9B2FFF745BB38BD4A
:103930003CF8050838E6060895CF06082DE9F04F53
:103940006B4B1B7887B0002B00F0CB80694D6A4829
:10395000A968FEF771F969686848FEF76DF9684B68
:103960006848D3E90031C91A674B1A68B1FBF2F213
:10397000FEF762F9FEF748F96448FEF7A9F96448D2
:10398000FEF7A6F94FF00008624B1B785FFA88F447
:10399000A34222D8FEF738F95F4D604E002455F857
:1039A000041F30460134FFF707FB162CF7D1FEF752
:1039B0002BF95B4D594E01242B4669681B68304634
:1039C000C91A0134FFF7F8FA162C05F10405F3D1F2
:1039D00007B0BDE8F04FFEF717B9524B142603EBC2
:1039E000840306FB045693ED450AB6F80E9049F0A1
:1039F000C9F996F81EA01AF0010F0CBF2D22522211
:103A00001AF0020F0CBF2D2354231AF0040F0CBF21
:103A10004FF02D0C4FF0560C1AF0080F0CBF4FF062
:103A20002D0E4FF0430E81B21AF0800F4FF03C0B79
:103A3000B1FBFBF105914FF064010CBF4FF02D0A73
:103A40004FF0530A80B201FB09F1671CCDE902A1D6
:103A50000490CDE900CE34483946FFF7ADFAB37F84
:103A6000DB073AD55C23314A6343D118D05891ED36
:103A7000010A70B1DFED2E7AB8EE400A20EE270A77
:103A800007EE900AF8EE677A80EE270A49F07AF995
:103A900000B2642290FBF2F102FB11022548FFF70D
:103AA0008BFA142101FB075701FB0454F988628A41
:103AB0000491218B0391E18A0291A18B0191A18A4A
:103AC000009102F0030319214B431B48218A9208FD
:103AD000FEF7B2F808F1010856E71848FEF78CF82F
:103AE000DFE7174807B0BDE8F04FFEF7F1B800BFB9
:103AF00004000010EC0D0010B5D40608C5D406086B
:103B0000000B0010DCD40608C819002009D50608EF
:103B100065D50608D0110010940E001015D60608C1
:103B2000980E001058170010C1D506080C0B001095
:103B300000401C46DED50608F3D50608EAD506087F
:103B400019D606080EB403B503AA52F8041B019255
:103B5000FCF781FB064BD3F848291AB90549986C44
:103B6000FBF7B2FE02B05DF804EB03B0704700BF94
:103B70002093002078E106082DE9F04798460B795C
:103B800003F0E005402D81460F46164632D1644DC4
:103B9000DFF8A881DFF8B091002416E03B7903F04C
:103BA0000703013B042B04D8DFE803F014171A1DA8
:103BB0002100315D5A48FFF7FFF97B79013BA342B1
:103BC00002DD4846FEF718F801347B79A342E5DCB4
:103BD000BDE8F08731572846EDE736F81410FAE7CC
:103BE00036F91410F7E756F824104046E3E756F884
:103BF0002410F0E703F00703052B57D8DFE803F0A4
:103C0000031F27292C3E3478602D55D02CD8002D49
:103C100075D1B7F80550B7F8076041482146FFF75E
:103C2000CBF9AC4239DBB44237DCB8F1000FCFD06E
:103C3000324629463B48BDE8F047FFF7BDB996F943
:103C40000040602D38D00FD8002D58D151E0348875
:103C5000DAE7B6F90040F4E7D6F800A0202D544684
:103C60004DD034D9602D27D0802DB1D132782E4B54
:103C70002E48002A14BF3146194635E0202D3468FD
:103C80003DD0EFD821462648FFF796F9D7F8051022
:103C9000A14202DB4B42A34221DDFDF7B5FF3A68AA
:103CA000234923464846BDE8F0474BE7202D25D061
:103CB0001ED9602DD8D100247B7944FA03F3DB07A9
:103CC000BDE8F0474CBF1B481B48FFF775B951468C
:103CD0001A48FFF771F9D7F805108A45DDD8B8F111
:103CE000000F3FF475AF1648BDE8F047FFF764B921
:103CF0000024B7F90550B7F907608EE700247A79F8
:103D0000104B03EBC20393F8E822A242C5DDD3F8BF
:103D1000E43253F82400BDE8F047FDF76DBF00BF63
:103D200096CF060895CE0608DBE7060838E60608B3
:103D30003BD60608E7CF0608D7EC06087FCF060873
:103D400035D606083CF80508A5D006082DE9F04F41
:103D5000164685B0CDE901011A4600213046FEF72E
:103D60001DF8314C009006F010034FF00009A246F8
:103D70000393FDF725FF2379029A03F0180393427A
:103D800003D0002A44D1182B42D14FF00D0B0BFB6E
:103D900009A3B3F809003EF0F7FB80462046FBF785
:103DA0009DFCD8E902210746024401442046FBF766
:103DB0002DFC80F00101009A0546C9B23046FDF79E
:103DC000EDFF039B009003B115BB0BFB09FBB30692
:103DD0005AF80BB00ED56DB914485946FFF7ECF8F8
:103DE000D8F8082001982B463A442146FFF7C4FE34
:103DF000FDF70AFF0E485946FFF7DEF8D8F80C2009
:103E0000019800233A442146FFF7B6FEFDF7FCFE79
:103E100009F1010940F25D23994504F10D04A8D18F
:103E200005B0BDE8F08F00BF1C07060855D6060890
:103E300056D6060870B50546084616460C46FBF7EA
:103E400053FD3346024621462846BDE8704093E6BE
:103E50000EB403B503AA52F8041B0192FCF7FBF958
:103E6000044B0549986CFBF72FFD02B05DF804EB9D
:103E700003B070472093002078E106080049E7E787
:103E800060D6060838B50C46054615492046FBF7AE
:103E900053FA30B9FDF76AFE1248BDE83840FDF725
:103EA00017BF11492046FBF747FAA0B90F4B83F81B
:103EB000B90183F8C10183F8A30283F8AB0283F848
:103EC0008D0383F8950383F8770483F87F0483F8E0
:103ED000F1040748E1E72846BDE83840CEE700BFD7
:103EE0006FD6060875D6060890D6060820930020DF
:103EF00098D606080049ABE7B4D60608F8B50646DA
:103F000008460C46FCF7A6FB20210546204649F052
:103F100080FC044618B93046BDE8F840EAE7124F85
:103F2000124E3B7832789A4204F1010401D0FAF73C
:103F3000F9FC0F4B20461D6047F0A4FB012201460F
:103F40002046FAF797FC3B7832789A4201D0FAF78C
:103F5000E9FC204647F096FB2A460146BDE8F840BA
:103F60000448FDF769BE00BF28200020872B0020F1
:103F700024200020CBD606082DE9F041064688B063
:103F800008460D46FCF766FB20210446284649F00A
:103F900040FC20B9304608B0BDE8F041AAE7FCF784
:103FA00059FB2246054601460F48FDF745FE85B1FF
:103FB000202D2A46694628BF20222046FAF7FAFC1F
:103FC000E84606460027B74208DBAD1B3444002E06
:103FD000EDD1FDF719FE08B0BDE8F08118F8010B2E
:103FE000FEF78EF80137EEE7E1D606082DE9FF4728
:103FF000074608460D4647F045FB082845D105F120
:10400000FF3801AE073531464246B14612F8010F7E
:10401000FCF73EFAAA4201F8010BF7D10023DFF8C2
:104020007CA08DF80C30A84517D11B49484628F0D4
:1040300059FF19481949082310F8012B11F8014BB1
:1040400010326A44013B02F80C4CF5D114488DF84B
:104050000C3001A9FDF7F0FD14E018F8010FFCF792
:1040600017FA06F8010B04460146504649F0D1FB09
:1040700028B12146304649F0CCFB0028D3D0384641
:10408000FFF7FCFE04B0BDE8F0870028D1D0384629
:1040900004B0BDE8F0472DE718980020046B06082F
:1040A000F9D6060807B5009313460A460249FFF7FA
:1040B000CFFE03B05DF804FB00D706082DE9F04FF2
:1040C000DFF8A4828BB006460D46284647F0DAFAA0
:1040D000034638B99649024601200BB0BDE8F04FBF
:1040E000FEF74CBC934905222846FCF7D7F9044655
:1040F000C8B9914D0146702205F1240049F072FBC8
:10410000C5F89440C5F8A040C5F8AC40C5F8B84023
:10411000C5F8C440C5F8D040C5F8DC40C5F8E84053
:104120000BB0BDE8F08F042241462846FCF7B6F9F3
:10413000044628BB2846FBF72EFC81460028EFD01A
:1041400047F0A0FADFF824B282465BF8047B37B967
:104150007A492A4630460BB0BDE8F04F78E6524621
:1041600039464846FCF79AF940B9204628F0BAF893
:104170007348744D3946FDF75FFDA6E70134E4E767
:10418000714907222846FCF789F9074600287AD1A9
:104190002021284649F03DFB044670BB6B486C4D1E
:1041A000FEF70AFF214628460134FEF705FF0E2CD4
:1041B000F8D1FDF729FDDFF8B891664FDFF8B4813B
:1041C000002529464846FEF7F7FE0C26DFF8A8A191
:1041D0006E430024F25960480123A34013420CBFF0
:1041E000414651460134FEF7E7FE0E2CF2D101356F
:1041F000FDF70AFD082DE4D192E75849574D01AA71
:1042000049F0D3FA02AC002848D0022F11D1029A0B
:10421000072A07D8039C0D2C04D80378722B13D0DF
:104220006E2B25D04E49082300223046FFF73AFF77
:1042300076E7FCF70FFA01AA44F8040B29460020A0
:10424000013749F0B2FADEE73B490C2303FB0211C8
:104250000123D1F89410A3400B4337490C2000FBF5
:1042600002123949C2F894303046FFF727FF57E76A
:10427000314B0C2000FB02330121D3F89430A140D4
:1042800023EA0103E9E728463449344F01AA49F0FB
:104290008CFA02AD002480B1082C03D13046FFF720
:1042A00029FE3DE7FCF7D6F901AA45F8040B39468B
:1042B0000020013449F079FAEDE7082CEED1029B99
:1042C0000F2B30D8DDF80CE0BEF1070F2BD8DDF84E
:1042D00010C0BCF10D0F26D8059F07F16402C82A53
:1042E00021D8069DFF2D1ED8079864281BD8089951
:1042F000642918D8884216DA099C032C13D8C3EB1A
:10430000C3020D4B134483F8291083F824E00D49B0
:1043100083F825C083F8267083F8275083F8280097
:1043200083F82A40A0E70F493046FFF791FDF7E6F2
:104330003CA4002019D7060818A4002024D706089A
:1043400035D706087AE106083FD7060839E6060899
:1043500047D70608ACA400204CD7060850D706085B
:1043600052D7060858D706081FD70608E8FD0508E3
:1043700096CF060811E606087DCE060810B504465D
:104380000748FDF7A5FCFAF713FE20B1BDE8104081
:104390000448FDF79DBC20460349BDE8104057E5A1
:1043A0006ED7060878D7060880D706082DE9F04FA3
:1043B0008FB0044602AA0846B14949F0F6F905460D
:1043C00040B903460246AF494120FEF7B3FB0FB0A8
:1043D000BDE8F08FAC49FAF7AFFF064628BBA84905
:1043E00002AA49F0E2F9FCF735F90828054606D992
:1043F000A649082332462046FFF754FEE7E7A44CBF
:1044000094F8D43683420CDC84F8D456DFE7314686
:10441000384635F02FFF013694F8D436B342F6DC37
:10442000F2E7064604F2D467F6E79A492846FAF717
:1044300083FF0646E0B9924902AA49F0B6F9FCF7B3
:1044400009F90828054603D9934908233246D2E7DB
:104450008F4C94F8D536834202DC84F8D556B6E703
:1044600030462946013641F07BFC082EF8D1F4E7AE
:104470008A492846FAF760FF064600BB804902AA2F
:1044800049F093F90028A2D0FCF7E4F80828054683
:1044900003D9834908233246ADE77D4C94F8BE37F3
:1044A000834209DD014604F2D46035F027FF294636
:1044B00004F2D46035F030FF84F8BE5787E77949BD
:1044C0002846FAF739FF064618BB714BDFF8B09162
:1044D00093F8BE7706AD01461022284649F082F9CE
:1044E000A846BE4202AA80F20A814946002049F04D
:1044F0005CF910B96C493A460AE1FCF7ABF80136B1
:1045000028F8020BEDE795E80F00684C84E80F00EF
:104510005DE767492846FAF70FFF0646C0BB5C4BCC
:10452000DFF85C9193F8BE7706ADBE4202AA80F236
:10453000F3804946002049F038F9014610B95D4939
:104540003A46E5E00322284649F09BF9AA464FF097
:104550000008284647F096F8404502D80136043551
:10456000E3E79AF80000FBF793FF08F101080AF867
:10457000010BEEE7504DB6000446B4423FF427AFBE
:1045800006AB19192819032235F05EFE0434F4E74E
:104590004A492846FAF7D0FE0746002840F0AC808A
:1045A000DFF8EC80364998F8D46602AA49F0FDF8A5
:1045B00000283FF40CAFFCF74DF8451E01D4AE4285
:1045C00003DC3F493346012215E72D4902AA0020AA
:1045D00049F0EBF8014600283FF4F9AE0026082226
:1045E00003A88DF8146049F04CF90DF10C0903A8EB
:1045F00047F048F8B0421BD8214902AA002049F0F0
:10460000D4F800283FF4E3AE037898F8D5A60193D8
:104610000026B14656451A4902AA4FF0000080F222
:10462000858049F0C2F8834650B9264952466FE06A
:1046300099F80000FBF72CFF013609F8010BD6E7CB
:10464000A6B99BF80030303B092B0FD91E49FAF769
:1046500073FE38B11D495846FAF76EFE70B11C4919
:104660005A4655E04FF001094FF0FF365846FBF728
:10467000F1FF002830DA17495A4649E0B146F3E71E
:1046800050D70608F499002087D706088DD706086A
:104690002093002098D70608A1D70608AFD70608B0
:1046A000BBD70608CDD70608BCD80608E09A00207C
:1046B000F7D70608DCD80608F09A002021D80608AB
:1046C00026D80608FCD8060849CC060832D80608C1
:1046D00039D806086ED806080EAB03EB4603013640
:1046E00023F8200C96E72049524611E033F8022BBC
:1046F00024F8022F013730E01C492A4608E01C4903
:10470000002049F052F800283FF4FDAE19493A461E
:104710002046FFF79DFB5AE61549002049F045F871
:1047200000283FF427AF14493A46F1E749F03DF835
:104730000028D8D1114C05EBC50082302044082256
:1047400003A935F081FD0198FBF7A2FE08EB0503F4
:1047500004EB051483F89E0706ABBE42C6DC454455
:1047600085F8B69733E600BF83D80608A6D80608B2
:1047700050D70608D9D7060803D80608F4990020B0
:104780002DE9F041144B1B6888B00446F3B11A6858
:1047900004A9D56A18466A46A847064688B1DFF8D4
:1047A000448004AC6D46002735F8022B34F8021B18
:1047B00040460137FDF740FABE42F5DC08B0BDE8DF
:1047C000F08106492046FFF743FBF7E7044908B0AC
:1047D000BDE8F041FFF73CBB883200203BD906081A
:1047E00053D9060821D9060870B5054608460C4677
:1047F00046F048FF024670B10E2804D10948214610
:1048000049F02DF838B12846064B074A0749BDE85C
:104810007040FFF71DBBBDE8704002490448FDF73A
:104820000BBA00BFE3D306085AD9060865D90608B3
:104830008FD9060870B5054608460C4646F022FF9B
:10484000024670B1042804D10948214649F007F80E
:1048500038B12846064B074A0749BDE87040FFF7C4
:10486000F7BABDE8704002490448FDF7E5B900BF5A
:10487000F2D306089DD9060865D90608ADD9060801
:104880002DE9F04307469BB008460C4646F0FAFE79
:1048900020220646002101A848F0A4FF36B3402E8E
:1048A00008D03B494023324638461BB0BDE8F043B0
:1048B000FFF7CEBA01AD04F140084FF00009022223
:1048C0002146684648F0DDFF0023102209A968460A
:1048D0008DF80290FBF71EFE099B0DF10202934238
:1048E00023D10234A04505F8010BE8D109AC4122DF
:1048F0000021204648F076FF264D002E3BD095F84B
:10490000F460D6B1202205F1F50101A848F0EEFFD0
:1049100098B105F1F5012046FBF72EFD1E4A1F490F
:1049200023463846FFF794FA04E01A781C493846C3
:10493000FFF78EFA1BB0BDE8F0831A4B1B78D3B992
:10494000CEB9194E01AB1A4603CAA242306071605B
:10495000134606F10806F6D101232046124985F8D0
:104960001531FBF709FD1148FDF70CFA10482146F7
:10497000FDF762F9DEE795F815311BB995F8F430CB
:10498000002BF3D008492046FBF7F6FCEEE700BF0A
:10499000C0D9060818A40020FED9060865D9060863
:1049A000E2D90608209300200DA5002008DA0608A9
:1049B00017DA06082DE9F74F834608460C4646F0FD
:1049C00061FEDFF818810646D8F8007028B102466B
:1049D00033492046FBF762FD80B93946314841F042
:1049E00071FA3149314821EA070141F06BFA304947
:1049F000304803B0BDE8F04F41F064BA23782D2B66
:104A00002D4B03BF013406F1FF364FF0010A4FF082
:104A1000000A4FF000094FF0FF3553F8041B51B165
:104A2000324620460193FBF739FD019B00280ABF5F
:104A30004D460021012109F1010991B9B9F11D0F7C
:104A4000EBD11E492246584603B0BDE8F04FFFF7B0
:104A5000FFB93B43C8F8003019491A4B12E01A4914
:104A600013E0114A0123AB401A40002AF7D007EAAD
:104A70000302BAF1000FECD027EA0303C8F80030B4
:104A80001249134B002A18BF1946124B124803EB68
:104A90008503D3F81C2603B0BDE8F04FFDF7CCB872
:104AA000A9D206084FDA0608BCD4551859DA060808
:104AB000432BAAE765DA060858FE050824D706083E
:104AC00047DA060840DA060824DA060830DA06086B
:104AD00037DA06083CF805080BCE0608B836002081
:104AE0002DE9F74F019008460E461746984646F0C6
:104AF000C9FD0446E8B93F483F4DFEF75DFA204640
:104B00000DF000FF3B68184206D020460DF00CFF68
:104B100001462846FEF750FA0134172CEFD13B68C6
:104B200013B93648FDF768F803B0BDE8F04FFDF75C
:104B30006BB8024632493046FBF7B0FC0546A8B9CF
:104B40003048FDF759F82C462F4D20460DF0DAFE7F
:104B500010EA080F06D020460DF0E6FE0146284672
:104B6000FEF72AFA0134182CEFD1DDE733782D2B2C
:104B700003BF013604F1FF34012500254FF0000981
:104B800048F4000B48460DF0CFFE2246824601460F
:104B90003046FBF783FC00BB48460DF0B3FE1BEA32
:104BA000000F1AD08DB1B9F1170F1CBF3B6840EA56
:104BB00003081648C7F80080FDF71EF81248514652
:104BC00003B0BDE8F04FFDF737B8B9F1170F1CBFC0
:104BD0003D6885433D600E48EEE709F10109B9F1F2
:104BE000180FCFD10B490198324603B0BDE8F04F02
:104BF000FFF72EB973DA060859D106087DDA0608E0
:104C0000A9D2060884DA06085AD1060837DA060857
:104C100047DA060824D70608014A40F202235FE774
:104C200048320020014B024A5AE700BFFFFF7F00D5
:104C30004032002010B50446012028F0C3F928B9FD
:104C400020460549BDE81040FFF702B9BDE8104015
:104C50000248FCF7F1BF00BF8FDA06089EDA0608AB
:104C6000074B10B50446D3F8180136F0A7F828B959
:104C700020460449BDE81040FFF7EAB810BD00BF68
:104C800018A40020A9DA060870B50546084616469D
:104C9000FBF7E0FC0D4B041E1A780EDB944205DA9C
:104CA0000B482146FCF7C8FF204670BD2EB1FF2CF3
:104CB00003D10848FCF7C0FFF6E70749013A284648
:104CC000FFF7C6F84FF0FF34EEE700BFD011001039
:104CD000BFDA0608D0DA0608E3DA06082DE9F04F55
:104CE000074691B08248834D0E46FCF7A5FF8249E6
:104CF000C5F81CD1002385F820310622012309784C
:104D00003046402485F8214104F036FC0A20F5F7AE
:104D1000E5FE95F820310C2BDAB240F2E4809DF8E4
:104D20000C60FE2E2CD0FF2E15BF0F24152400255D
:104D30000125944240F0D780611EC9B268463BF01D
:104D4000D7FA04F140030DEB030414F8413C83420D
:104D500040F0C4806A1E012A9DF80D3012D903F07C
:104D60001F0761375C096548FCF746FF022D39D003
:104D7000013C042C34D8DFE804F00B2D2F33310034
:104D80000225D6E79DF80E709DF80F401E46EAE713
:104D90005B48DFF8C491DFF8C4A1DFF8C4B1FCF7C9
:104DA00097FF5848FCF728FF6C464FF0000814F8AE
:104DB000011B484608F10108FEF7FEF8B8F10C0F98
:104DC00016D00AFB08F3B3F1553FF0D85846FCF76C
:104DD00013FFECE74C48DCE74C48DAE74C48D8E7EF
:104DE0004C48D6E700238DF83F300DF11F00D0E787
:104DF000FCF70AFF022D3AD06422B6FBF2F102FB67
:104E000011623B464448D2B2C9B2FCF715FF85F0A7
:104E100001035B42DBB2012B59D8404A404B9DF85D
:104E200010104048404E00290CBF11461946FCF7AF
:104E300003FF9DF811103D4B3D4800290CBF314642
:104E40001946FCF7F9FE022D41D19DF81240394870
:104E5000FCF7D2FE8CB1FF2C1FD00A23B4FBF3F178
:104E600003FB11423448D2B2FCF7E6FE08E03348B7
:104E70003A463146FCF7E0FECFE73046FCF728FF24
:104E80009DF813402E48FCF7B7FE44B1FF2C21D00B
:104E90002C482146FCF7D0FE04E02B48EEE72248E0
:104EA000FCF716FF204E214FDFF89C800DF1130513
:104EB000002415F8013F7BB1FF2B14BF3A46424650
:104EC000214622480134FCF7B7FE042CF1D111B081
:104ED000BDE8F08F1C48E3E73246F1E71C4938464D
:104EE000FEF7B6FFF3E71B48FCF7F2FEEFE700BF63
:104EF00029DB060818A40020D01100103ADB0608B0
:104F000045DB06086BDB06084CDB060854DB0608AD
:104F10005CDB06080AD006087DDB060812DB060803
:104F200009DB0608B4DB060819DB06084AE50608B3
:104F3000CBDB0608D2DB0608E6DB060899DB0608B1
:104F4000EEDB060896CF06081DDB0608FEDB06082A
:104F500009DC060819DC06085FCC0608ABAAAAAA79
:104F6000DBE706082DE9F843DFF8A49007460C4676
:104F7000204646F087FB064658B91D4B1D481A7857
:104F80001D4B03EB8203D3F8A815BDE8F843FCF7EB
:104F900053BE024649462046FBF780FA60B1DFF86F
:104FA0006480002558F8041BB1B9224638461349DD
:104FB000BDE8F843FEF74CBF1148124C124DFCF708
:104FC0001BFE54F8041B19B12846FDF7F5FFF8E75E
:104FD000BDE8F843FCF718BE32462046FBF75EFA00
:104FE00001350028DED1024B084C1D70C0E700BF20
:104FF0006431002022DC06083CF8050824D70608A6
:1050000084DA0608E8FD05085AD106087AE10608A0
:10501000A9D2060838B50D4604461A490522284685
:10502000FBF73CFA68B9184B93F84C2022B90121E0
:1050300083F84C1083F84D20BDE838401348FCF746
:1050400047BE134903222846FBF728FAA0B90E4DA4
:1050500095F84C3063B195F84D304BB10D49204671
:10506000FEF7F6FE002385F84C3085F84D3038BD4C
:105070000948FCF72DFEF5E720460849BDE8384011
:10508000FEF7E6BEA1E40608209300202CDC06080B
:10509000F3E5060842DC060879DC06088DDC060824
:1050A00070B5184C94F84C3005467BB194F84D30EF
:1050B00063B11549FEF7CCFE28461449FEF7C8FE39
:1050C000002084F84C0084F84D0070BD104B93F81C
:1050D0001521AAB193F8F42092B903F1F50203F572
:1050E000927503F21516106851682C4603C40832F5
:1050F000B2422546F7D1012283F85F2106F0ECFA8F
:105100000120E2E72093002042DC06089CDC060830
:1051100018A400202DE9F04F80468BB008460D46BC
:1051200046F0B0FA0246B0B3A3492846FBF7B6F9F9
:10513000044680BBFCF768FDA048A14DA14EA24FDC
:10514000DFF8C482FCF7C4FD142040F01DFEE1101E
:10515000304604F007020131FDF72EFF95F81D904F
:1051600095F91C00B9F1000F0ED004F0ADFC4A46D1
:1051700001464046FCF760FD0134102C05F1240582
:10518000E5D10BB0BDE8F08F04F09EFC0146384637
:10519000FCF752FDF0E728468C4905AA48F005FBCC
:1051A000054620B901464120FCF705FEE9E788499C
:1051B000FAF7C2F820B987494046FEF749FEE0E712
:1051C000854E0827002431682846FAF7B5F80028EC
:1051D00008BF3446013F06F11006F4D154B97F49A7
:1051E0002846FAF7A9F828B17D492A464046FEF735
:1051F0002FFEC6E7002075498DF8130005AA48F078
:10520000D4FA0646002C4DD0002849D0FBF722FAEC
:10521000031E42DB2279062A3AD1E268012101FA13
:1052200003F0104239D0DBB247F6FE7040FA03F2C9
:10523000D20732D599400139084048F067FB05464E
:10524000E0883DF0A1F96749D0E9022309780029F7
:1052500018BF1A46217A637A05FB0133002712F939
:105260000390039702EB030A584905AA002048F06F
:105270009CFA834600283ED15B49012394B39AF9F6
:1052800000202046CDE900312946FAF7C5FB78E732
:105290005D1E13B1A37A9D42D2DB54493246A5E785
:1052A000534EFAE768B10DF11301FBF7ADF928B1E0
:1052B0009DF813502846F5F74BFD20B94D4932466D
:1052C00094E74B4EFAE72846F6F7E0F88146284681
:1052D00005F01EFC0390284605F056FCA246074642
:1052E0002546C1E7CDE900319DF813004A4639460D
:1052F000FAF7D6FB45E73649FAF71EF8064658BBDB
:10530000ACB13D4FEDB2207972B22946F6F798F86C
:1053100000283FF436AF0288037800933146C2F389
:1053200003233846120BFCF787FC0136EBE7324CBF
:105330007979386872B2F6F7C5F800283FF421AFE2
:105340000288037800933146C2F303232046120BF0
:10535000FCF772FC0136EBE728495846F9F7ECFFF9
:10536000002853D05846FBF775F9064642B29CB167
:105370002079E9B2F6F764F8002849D12946204699
:10538000FAF7FEF926681E49CDF800B0034632460A
:105390004046FEF75DFDF4E679793868F6F792F855
:1053A000B0BB9DF813301749CDF800B01A09403250
:1053B00003F00F03ECE700BFBADC0608BFDC060809
:1053C000C0020020D5DC06085AD1060850D70608CE
:1053D000A9D20608E6DC0608080600201CE006083C
:1053E000FADC060820930020111C010809DD0608DC
:1053F0007AE1060819DD06082BDD06087FDA0608C3
:105400004CDD06086FDD060844DE06084FF0FF3667
:1054100006AF39463046FAF7C3FF08A94846FAF7FF
:10542000BFFF4E451CD076B274B18AF800602946A1
:105430002046FAF7A5F9266800970246134808ABFC
:105440003146FCF7F9FB9CE69DF81320039B1048BE
:105450009E701109009708AB02F00F024031F0E78F
:105460005CB129462046FAF78BF9266802460948BE
:1054700008AB3146FCF7E0FB83E69DF813200648B5
:10548000110908AB02F00F024031F3E797DD06087F
:10549000BADD0608E2DD0608FDDD06082DE9F04F5D
:1054A00007468DB008460D4646F0ECF8044630B984
:1054B000014601200DB0BDE8F04FFCF787BD024664
:1054C000A5492846FAF7EAFF30B9A44938460DB095
:1054D000BDE8F04FFEF7BCBCA14922462846FAF7CA
:1054E000DDFF002854D1FCF78FFB9E48DFF8B4A203
:1054F000DFF8B4B2FCF7ECFB172040F045FC0E27B8
:105500001AF9018BB8F1000F36D041465846FDF725
:1055100053FD00252E46B10089B2404605F06EFBD2
:10552000814605F0F7FB90F9003004460136CBB117
:105530000DB9FCF769FB99F80630657894F900001D
:10554000894A8A4C03F00203002B18BF1446B5B1F8
:1055500004F0BAFA00950346224685483146FCF726
:105560006BFB0125042ED6D115B98248FCF7B0FBA0
:10557000013F17F0FF07C3D10DB0BDE8F08F04F075
:10558000A3FA2246034631467B48FCF755FBE8E781
:10559000002476498DF81B4007AA284648F005F9F3
:1055A00018B93846FEF76AFCE6E70DF11B01FBF778
:1055B0002BF881460028F4D09DF81B502846F5F7BB
:1055C000C7FB20B96D493846FEF742FCD4E7DFF847
:1055D000DC8123464FF0FF3403EB430218F802202E
:1055E00095420BD0002C02DA002A08BF1C4601337A
:1055F000152BF1D1002C16DA6149E4E71C465B4912
:1056000007AA002048F0D1F80646002800F096804E
:105610005149F9F791FE30BB5A4FDFF84C81DFF862
:105620009091044616E04FF00009E8E7306896F8DC
:1056300007A0F6F739FAB179737911F0020F0CBFB0
:10564000394641469B08024600910133514648467F
:10565000FCF7F2FA01342146284605F06DFA0646B9
:105660000028E3D188E7484902223046FAF716FFBE
:105670004FEA151A0AF1400A05F00F0B002845D130
:105680000390B01CFAF7E6FF0399024604912846FE
:1056900001310592039105F04FFADDE90313059AF4
:1056A00038B93A4900965B4652463846FEF7D0FB79
:1056B00062E7C0799042E9D11F466300B9F1000F5B
:1056C00031D01A1942445678013E7A1C234414BF43
:1056D0002946002108EB030208F803107B1C5370D5
:1056E0000AACFF239370394622462846FAF768FE33
:1056F00008AA31462846FAF763FEB74216D1244875
:1057000008AB5A465146FCF797FA35E7214930462F
:10571000F9F712FE20B1204900965B465246C4E7D5
:105720004FF0FF37C9E74FF0FF36CEE71B48009434
:1057300008AB5A465146FCF77FFA1DE704EB4404D8
:10574000174B0093A044024698F801100123284605
:10575000FAF7ECF910E700BFA9D20608E6DC060864
:10576000BADC060819DE0608E8CF060850D7060896
:1057700039DE06085ADE06084BDE060860DE06083B
:1057800077DE06087AE10608A0DE0608A3DE060832
:10579000F5DE06087FDA0608CFDE060813DF060806
:1057A000111C0108F05B060832DE060840220020CA
:1057B0008BDE06082DE9F04F89B0074605AA08469A
:1057C0009C4947F0F2FF054630B901464120FDF7FC
:1057D0006FFB09B0BDE8F08F9749F9F7ADFD0446BE
:1057E00000283CD19548964D964EDFF89882FCF7FC
:1057F0006FFA142040F0C8FA95F9060004F064F935
:105800002968AA8801F13F4101F57E01B2FA82F2CE
:10581000890A03464131C2F11F023046FDF7CCFB35
:10582000E97911B14046FDF7C7FB0134FCF7ECF90B
:10583000602C05F10805DFD17E4905AA002047F05C
:10584000B4FF8149F9F778FD0028C2D138467A497A
:10585000FFF724FE78493846FFF75CFCB9E7DFF82C
:10586000FC91002419F9340004F02EF98046014619
:105870002846F9F761FD40B10134202CF2D173497B
:105880002A463846FEF7E4FAA3E76A4905AA47F034
:105890008CFF064690B3FAF7DDFE05466C4B03EB32
:1058A000C4034FEAC40A93F8EA314BBB002D29DC4C
:1058B00009EB0A03588893F8049093F805A03CF08C
:1058C00063FEEBB2D0F808B0009303FB09AA002EE8
:1058D00000F09A803378002B00F0968006A93046BD
:1058E000FAF792FE002800F08C809DF8185005BB56
:1058F0000BF80A505748FCF7EBF96AE70546CDE785
:10590000002D05DD012B1A4638BF0122954208DD26
:10591000012B514938BF012301223846FEF7C2FB53
:1059200057E7444905AA002047F03FFF013D0646DE
:10593000BEE72846F5F70CFA814600285DD02B0912
:10594000403302930BF80A5005F00F03434F0393C3
:105950004FF00008BB79012B38BF012301930026CB
:10596000788897F804B097F805A03CF00DFE06FB88
:105970000BA38268D15CA94222D1444504D100998D
:10598000B1421DD00021D154DDE9021234485FFA42
:1059900086FB5FFA88FAFDF70FFB59465046FDF784
:1059A000AFFF444509D12F48FDF706FB5046594645
:1059B000FDF7A6FF2C48FDF7FFFA2C48FCF788F905
:1059C000019B0136B342CBDC08F10108B8F1200F8E
:1059D00007F10807BED1D9F80010B9F8042024480F
:1059E00001F13F4101F57E01B2FA82F2890AC2F16A
:1059F0001F024131FCF720F9EBE63846FEF73EFA8C
:105A0000E7E61C4932463CE71BF80A30013573B122
:105A10001A09194903F00F03403206A8FAF748FCA7
:105A200006AB16482A464146FCF706F9D1E6144B68
:105A3000F7E700BF50D70608BADC060839DF0608CA
:105A4000B81A002077DF060882DF060886DF06081E
:105A50003CF80508A8DF0608A2DF060820FA0508BA
:105A6000BADF060801D00608DEDF060802E70608EE
:105A7000E8DF060804E0060851CF060820E0060823
:105A80009DCB060895CF060820B10078B0FA80F0CB
:105A900040097047012070472DE9F74F81460846BD
:105AA000FFF7F2FF0E46054670B1002401A920461B
:105AB00040F09AFA013401464846FFF7EDFF122CF8
:105AC000F4D103B0BDE8F08F0846FAF7C3FDC4B2C5
:105AD000112C71D8701C3D4D3D4EF9F75CFF05EB64
:105AE0004408670098F860A18346B8B9AAF102019A
:105AF0004B424B413D4495F86021B25C002B54D0A1
:105B000095F86131192040F2EE2100FB0313314872
:105B1000214603B0BDE8F04FFCF78EB8017830465F
:105B200047F077FE78B1032C94BF002201222A4966
:105B300002EB4202831B0A4452FA83F393F890A6C5
:105B4000BAF1030F05D1484603B0BDE8F04FFEF7A8
:105B500095B95846F9F71FFFF0B1BAF1020FF2D12B
:105B6000FAF778FD40F6CA0380B29842A8BF1846FB
:105B700040F2EE239842B8BF1846A0F2EE20192357
:105B8000B0FBF3F088F86101AAF1020253425341DD
:105B9000EA1982F860A1ADE7BAF1020FF4D14846E4
:105BA00003B0BDE8F04FFEF7A5B90C48214603B09D
:105BB000BDE8F04FFCF740B8094911232A46484692
:105BC00003B0BDE8F04FFEF76DBA00BF18A4002087
:105BD000146D060834E006083CF8050844E00608A1
:105BE00051E006082DE9F041054686B00846FFF76A
:105BF0004BFF0F46064640B100235C491A46012080
:105C000006B0BDE8F041FCF79DBA0846FAF722FD60
:105C10001328044600F3A18006254543781C8DF81F
:105C20001760F9F7B8FE524E074660B1FAF712FD59
:105C3000C0B213F071FA30B17319027983F83826C3
:105C400001238DF817303846F9F7A5FE074668B1ED
:105C5000FAF700FD0D2809D8062303FB046383F837
:105C600039069DF8173001338DF81730DFF8FC80C6
:105C7000A91C0DF1170241443846FAF7EFFCF9F779
:105C80008AFE074668B1FAF7E5FC012809D89DF8B5
:105C90001730062202FB0462013382F83C068DF8BD
:105CA00017303846F9F777FE80B1FAF7D3FCC0B267
:105CB00013F032FA50B19DF817300179062202FB39
:105CC0000462013382F83D168DF817309DF81720D5
:105CD000042A4FF006032FD103FB04630022A3F82C
:105CE0003C26062505FB04651DF06CFC95F838067E
:105CF00013F0F6F995F83B1695F83A7619234FF418
:105D00006172804695F83D0613FB012613FB0727B9
:105D100013F0E6F9437998F80520039395F83C369B
:105D20000097CDE90163134895F839362146FBF712
:105D300083FF06B0BDE8F081052A05D103FB0463AB
:105D4000002283F83D26CCE7062ACAD008EB0502DC
:105D5000002348F805309380C3E7074913233246F0
:105D6000284606B0BDE8F041FEF79CB958990020DE
:105D700020930020A4CD0608A2DF06082DE9F047F5
:105D800080468CB00846FFF77FFE054640B10023F1
:105D900059491A4601200CB0BDE8F047FCF74EBA4D
:105DA000CDE909000B90079107A8544947F0D0FCB2
:105DB00006463FF0FDFF431C04460ED12B460A2247
:105DC00008A93046FAF7A6FB089B1B782BB9C4B28A
:105DD000132C96BF333444B264B220460CF0B2FDAB
:105DE000054628B94046FEF749F80CB0BDE8F087F3
:105DF00042498DF8284007A847F0AAFCB0B3002319
:105E00000A221946FAF786FB02260990DFF8EC9081
:105E1000DFF8F0A00027494607A847F099FCF8B141
:105E2000FAF718FC364A002352F8041B88421FD1A7
:105E3000DBB20AEB8302D2F8A421904210D1022FE8
:105E400020D0032F23D05A1E012FD2B215D00B2AF7
:105E500003D88DF829300136F6B20137042FDAD194
:105E6000052E1AD84046FEF745F8BEE70126CDE7D5
:105E70000133102BD8D10023DBE7052AEDD88DF8AC
:105E80002A30E8E7092BE8D88DF82C30E3E79A1E92
:105E90000D2AE2D88DF82B30DDE709AB03CB286063
:105EA00018686960A860204640F088F8154A9DF897
:105EB0002B1002EB81010346D1F8A41104919DF847
:105EC0002C1002EB8101D1F8A41103919DF82A1046
:105ED00002EB8101D1F8A41102919DF8291002EB87
:105EE00081020021D2F8A4210192099A0092084669
:105EF000054AFBF78DFE78E74C98002050D706083E
:105F0000E0F905083CF80508BDCD06082DE9F04F7D
:105F10000346A1B00846FFF7B7FD054628B118466D
:105F200021B0BDE8F04FFDF7E5BFDFF8C4920B905C
:105F3000FF238DF82830D9F81831ADF83000CDE9BD
:105F4000050093F838200D908DF838200F90ADF8AB
:105F500040001193099107464FF0FF38934909A873
:105F600047F0F6FB044618BB914F01460AAC0B0103
:105F700090481A57002310F9016BB24240F0D280CA
:105F800010464E1C40F01AF8314602463846FBF7E0
:105F900053FE022E4FF00101E9D19DF938A09DF981
:105FA0002830534540F0C5808348FBF745FE4DE05F
:105FB0002378002BD2D0032FD4BF00260126062F32
:105FC00000F2A980DFE807F0044750910447500031
:105FD000042F10D079492046FAF784FA58B14FF4CB
:105FE00080600FF053FA002800F0B58190F90400AA
:105FF000012306930AE072492046F9F79DF970B92A
:10600000D9F8183193F93800042F22D0119B11933D
:1060100020AB03EB061606F8580C01379EE7204626
:106020003FF0C6FE0028EFDA01230A2212A920461B
:10603000FAF770FA40B2002803DB129B1B78002BA2
:10604000E2D060482246711CFBF7F6FD21B0BDE8A6
:10605000F08F0023DBE72046FAF7FCFA20AB03EBD6
:10606000061646F8540CD8E757492046FAF73AFA8C
:106070005649B0F1000A204618BF4FF0010AFAF75E
:1060800031FA08B14AF0020A3301DFF868C1079318
:1060900020AB03EB0616BCE80F0006F850AC12AEBE
:1060A0000FC6BCE80F000FC6BCE80F000FC69CE887
:1060B000030086E8030000260DF1480AB346DAF82B
:1060C0000010204647F0FCFB10B19AF804301E4344
:1060D0000BF1010BBBF1070F0AF1080AEFD1079B87
:1060E00080336B4403F84F6C97E739492046F9F742
:1060F00023F9A0B137492046F9F71EF900288CD0C2
:106100002046FAF7A7FA0328804686D90146324886
:10611000FBF792FD9AE731482246082194E70123D4
:1061200005937AE70133072B7FF425AF2C48013123
:106130008AE70B9B1BB9AAF1140255425541002373
:106140005F1CE368002B62D194F900B058460CF054
:1061500049FCD4F8049018B10668002E40F08B80FA
:10616000B9F1000F237A14BF4E464FF461466660C2
:1061700023B91C48FBF760FD03232372627A2AB11E
:10618000194807923946FBF757FD079A0292237A7E
:10619000CDE9006300231A46194658460FF0F8F976
:1061A000E06048BB11483946B2E700BF50D7060847
:1061B000D5E0060851F00508F2E0060874E006088C
:1061C0007FE0060883E006089EE0060877E50608FB
:1061D00019D706087FDA0608A1E00608B9E0060824
:1061E000E0E006080BE1060826E1060841E10608A2
:1061F00018A40020D4FE05085849594A5948B9F155
:10620000000F18BF0A4633463946FCF7D5FE022F69
:1062100004F110044FF0010392D1119E0D9F4DB176
:106220005148FBF755FD33681B6A1BB14F493A468D
:1062300030469847059B002B50D04D49474BBAF14B
:10624000140F18BF19464B48FBF7F6FCBAF1140FB0
:1062500009D1059B002B43D03368DB691BB146494C
:10626000002230469847069B002B43D1002231463E
:1062700038463FF0B5FDE660B9F1000F2CD0494635
:10628000304601F071FE3D4AB3683D483946FBF7A0
:10629000D3FC94F80890B9F1000F0CD032799145F5
:1062A00009D038484B463946FBF7C6FC33684946A7
:1062B0009B6930469847637A23B1727932483946F0
:1062C000FBF7BAFCF36A002BA1D030483946FBF744
:1062D000B3FC0023F3629AE7204AD5E71F49B2E7EF
:1062E000B8F1000FBFDB3368DB69002BBBD0284956
:1062F0004246B6E703F0A2FB0520F4F7EFFBDFF818
:106300009490DFF894A000254FF0030B9AF800302A
:10631000AB42ABD919F8014FC4B1204604F034FCAC
:10632000804698B12046F4F713FDEBB2044610B155
:1063300080F806B0C37120460121F4F771FC98F88B
:106340000630DB07204603D5F4F744FE0135DDE7D0
:10635000F4F73AFEFAE74FF0FF3049E67AE1060833
:1063600059E006085DE1060813E20608697F0108A6
:1063700067E006083CE20608B1F9000862E006089A
:106380007BE10608A0E10608C3E10608FAE1060879
:1063900045F7000887220020D01100102DE9F043B6
:1063A00080468BB00846FFF76FFB0F46044640B1AE
:1063B00000235E491A4601200BB0BDE8F043FBF70D
:1063C000C3BF0846FAF746F91D28054600F3A58025
:1063D0000A264643781C8DF82740F9F7DCFA10B1FD
:1063E00001238DF82730F9F7D6FA514C074668B1EA
:1063F000FAF730F90D2809D80A2303FB054383F87F
:1064000084019DF8273001338DF82730DFF81C9187
:10641000711C0DF1270249443846FAF71FF9F9F7C4
:10642000BAFA074668B1FAF715F9232809D89DF892
:1064300027300A2202FB0542013382F887018DF8DA
:1064400027303846F9F7A7FA074668B1FAF702F994
:106450000D2809D89DF827300A2202FB0542013396
:1064600082F888018DF827309DF82730062B0CD054
:1064700009EB06020023404649F8063053601381B9
:106480000BB0BDE8F043FDF735BD0A2606FB054617
:1064900000233846A6F88A31A6F88C31F9F77BFA42
:1064A000074618B1FAF7D6F8A6F88A013846F9F780
:1064B00072FA30B1FAF7CEF80A2303FB0543A3F8CA
:1064C0008C011C4B4FF0FF325A600A2303FB05423C
:1064D0004FF46170B2F88C310693B2F88A310593AB
:1064E00092F88831049392F88731039392F88611D9
:1064F000192313FB0101029192F8851113FB01038B
:10650000019392F88431009300210B4A2B460846F0
:10651000FBF77EFB0BB0BDE8F08308491D23224644
:1065200040460BB0BDE8F043FDF7BCBD9CA5002084
:1065300018A40020FC050020DACD0608A2DF06081A
:106540002DE9F14FDFF894B106460D462846FFF7D6
:106550009BFA074640B1002359491A46012001B071
:10656000BDE8F04FFBF754BF564905222846F9F71E
:1065700095FF60B9524B00221A601A611A621A63C1
:106580001A641A651A661A6701B0BDE8F08F042212
:1065900059462846F9F782FF04462846002C42D186
:1065A000F9F7F9F907460028EED045F06BF8DFF867
:1065B00030A15FFA80F85AF8049BB9F1000F07D1B7
:1065C00041492A46304601B0BDE8F04FFDF740BCD6
:1065D000424649463846F9F761FF013484460028AF
:1065E000E9D1374A0346154600210133082B42F80A
:1065F000101BFAD1354B03EBC40257682FB934484E
:10660000344D4946FBF718FBA0E713F834E0F44596
:10661000F5DA07EB0C130FCB05EB0C1484E80F0035
:106620000CF1010CF3E7FAF715F8072804463DD8FA
:106630002846F9F7B0F9074658B3F8F71FFF204B83
:1066400003EB041383ED000A01253846F9F7A3F99B
:10665000074638B1F8F712FF194B03EB041383ED2B
:10666000010A01353846F9F796F9074638B1F8F7C7
:1066700005FF134B03EB041383ED020A0135384683
:10668000F9F789F938B9304601B0BDE8F04FFDF7A8
:1066900031BC0546D9E7F8F7F1FE094B032D03EBB2
:1066A000041383ED030A3FF456AFECE70A490723CE
:1066B0003A46304601B0BDE8F04FFDF7F3BC00BFED
:1066C0006C31002019D7060824D7060858F00508B1
:1066D00035D706087AE10608A2DF06081FD70608A4
:1066E000E8FD05082DE9F34105460846FFF7CCF91A
:1066F0000C46074640B1002333491A46012002B038
:10670000BDE8F041FBF720BF30492046F8F714FE02
:1067100070B92D4B04224FF47A704FF4FA61013AAC
:106720001880598003F10403F9D102B0BDE8F0816B
:106730002046F9F78FFF0328064641D82046F9F78F
:106740002AF9074698B1F9F785FF4FF0010804468A
:106750003846F9F720F920B1F9F77CFFB8F1000FBE
:1067600009D1284602B0BDE8F041FDF7C3BB40F2B5
:10677000EE248046ECE7A4F2EE2240F2DC539A428B
:1067800003D8A0F2EE229A420AD9114940F6CA0370
:1067900040F2EE22284602B0BDE8F041FDF782BC8F
:1067A0000C4B0D4A03EB86030021A3F8B042A3F87B
:1067B000B202CDE9004033460846FBF729FAB4E7B8
:1067C000064903233A46E5E7C8A6002019D706087C
:1067D0005FE2060818A4002011CE060851E0060862
:1067E000F0B5074689B00846FFF74EF90E46054654
:1067F00040B100231A491A46012009B0BDE8F04013
:10680000FBF7E6BE0846F9F725FF1F2804461DD80A
:106810003046F9F7C0F80146204634F0B7FC78B1AD
:106820000F4803AE314600EB84003FF075FB0D4A84
:106830000096234629462846FBF7EAF909B0F0BD41
:10684000384609B0BDE8F040FDF718BB06491F23E4
:106850002A46384609B0BDE8F040FDF723BC00BF2A
:10686000D8A6002022CE0608A2DF0608F0B507460B
:1068700085B00846FFF708F90E46054640B10023EB
:106880001D491A46012005B0BDE8F040FBF7E8BEFF
:106890000846F9F7DFFE0F28044623DC3046F9F7F7
:1068A0007AF80146204634F057FDA8B1134B04F1A5
:1068B000200203EB8203294693F8C322029293F845
:1068C000C2220192B3F8C03200930D4A23462846F3
:1068D000FBF79EF905B0F0BD384605B0BDE8F040C5
:1068E000FDF7CCBA07490F232A46384605B0BDE864
:1068F000F040FDF7D7BB00BF58A7002018A4002028
:106900002CCE0608A2DF0608F0B5054685B008467D
:10691000FFF7BAF80B46044640B100231B491A465C
:10692000012005B0BDE8F040FBF7E2BE1849184F62
:106930006A46184646F039FF01AE88B1032C04D1EF
:106940002846FDF7D7FA05B0F0BDF9F783FE6A4691
:1069500046F8040B39460020013446F026FFECE7E8
:10696000032CEDD1DDE90146039F31463A46E0B202
:1069700034F02EFD18B92846FDF780FAE3E7054804
:106980003B4632462146FBF757F9DCE7D8A6002004
:1069900050D706083ECE0608F0B506468BB008462E
:1069A000FFF772F80D46044628B300233E491A4605
:1069B00001200BB0BDE8F040FBF738BF2D2903D014
:1069C000A1F13003092B49D8052C05DD30460BB069
:1069D000BDE8F040FDF78EBA2846F9F73BFE0AAB5A
:1069E000621C03EB440424F80C0C15F8013F303B07
:1069F000092BFAD9144629780029DFD1062CE5D1D4
:106A0000BDF81C20BDF91C30072ADFD8BDF91E5087
:106A1000A5F5FA7292B2B2F5FA6F18D8BDF92070E6
:106A2000A7F5FA7292B2B2F5FA6F10D8BDF922C08A
:106A300065450CDC67450ADBBDF924E00EF1640214
:106A400092B2C82A03D8BDF92640112C11DD17498E
:106A500030460BB0BDE8F040FDF7FAB9202902D16D
:106A600001352246C6E730460BB0BDE8F040FDF7E1
:106A700005BA0F4A0C2000FB032264B2A2F898501A
:106A8000A2F89A70A2F89CC082F89EE082F89F401B
:106A90000846CDE903E4CDE9017C064A0095FBF701
:106AA000B7F80BB0F0BD00BFACA4002058D7060863
:106AB00018A4002052CE06082DE9F04F074689B0F1
:106AC0000846FEF7E1FF8B46054640B100234D49DD
:106AD0001A46012009B0BDE8F04FFBF7CBBF4A4B87
:106AE000084693F8D4A693F8D59693F8BE87F9F79D
:106AF000B1FD092804467BDC062646430BF1010064
:106B00008DF81F50F8F747FF3E4D834638B1F9F72F
:106B1000A1FD0D2803D80123A8558DF81F30584634
:106B2000F8F739FF834660B1F9F794FD504508D86E
:106B3000062303FB045358709DF81F3001338DF872
:106B40001F305846F8F727FF824660B1F9F782FDFB
:106B5000484508D8062303FB045398709DF81F305E
:106B600001338DF81F305046F8F715FF814660B1AC
:106B7000F9F770FD804508D3062303FB0453D87052
:106B80009DF81F3001338DF81F30311D0DF11F02AC
:106B900029444846F9F762FD9DF81F30062B09D0BD
:106BA000AA1900233846AB51938009B0BDE8F04FD5
:106BB000FDF7A0B96343EA184FF4617650791921C3
:106BC00011FB00600590107911FB00610491D178F0
:106BD00003919178029152780192EB5C009300212D
:106BE0000A4A23460846FBF713F809B0BDE8F08FC0
:106BF000074909232A46384609B0BDE8F04FFDF79A
:106C000051BA00BFA0320020209300209CCE06087D
:106C1000A2DF06082DE9F74F05460846FEF734FFC8
:106C20000B46044618B9334A92F8B0732FB9284678
:106C300003B0BDE8F04FFDF721B92F49DFF8C89048
:106C4000DFF8C8A001AA184646F0AFFD264610B9E5
:106C500002F000FF08E056B9012201462846FEF77F
:106C600013F8421C04461AD103B0BDE8F08FF9F7BF
:106C7000F1FC2F28834636D80FB102F0DFFEBBF1BE
:106C8000060F13D01D49012309785FFA8BF2E0B299
:106C900002F072FC59464846FAF7CEFF0027164923
:106CA00001AA0020013646F080FDD0E7DAF8003076
:106CB0001B0114D5FF2C0ED0E1B22846FEF70EF8CA
:106CC000E8E72846FEF70AF8013798F80020F9B2FD
:106CD0008A42F6D8DEE7DFF824800027F5E7084887
:106CE000FAF7F6FFD6E707492F222846FDF7B0F856
:106CF000D5E700BF18A4002050D70608D011001017
:106D00008FDA06087EE206086DE206080C310020E4
:106D10002DE9F74307460846FEF7B6FE0B46044644
:106D200028B1384603B0BDE8F043FDF7E3B82F497A
:106D3000DFF8B89001AA184646F037FD264605460A
:106D4000A04665B92A4B3246D3F81801A1B240F0EB
:106D5000ABFF68BB27493846FDF77AF828E0B8F161
:106D6000000F06D0B8F1010F25D03846FDF7C2F864
:106D70001EE0284644F086FC1F4906460246284687
:106D8000F9F78CFB50B31D4932462846F9F786FBCC
:106D900030B31B4932462846F9F780FB10B3194936
:106DA00032462846F9F77AFBF0B13846FDF766F827
:106DB00003B0BDE8F083B31E5A425A412946384613
:106DC000FDF762FF421C0446F2D001AA49460020AA
:106DD00046F0EBFC08F101080546B2E74646F4E749
:106DE0000126F2E70226F0E70426EEE750D7060870
:106DF00018A40020AAE206089EE20608A1E20608FE
:106E0000A4E20608A7E206082DE9F74380460846F3
:106E1000FEF73AFE0B46054628B14046FDF76AF8F4
:106E200003B0BDE8F0832E49DFF8B49001AA1846FC
:106E300046F0BBFC2F4604462E467CB9022DECD111
:106E4000A7F57A73B3F57A7F21D926494FF4FA630F
:106E50004FF47A724046FDF725F9E1E74DB1012D77
:106E600010D001AA4946002046F09FFC0135044697
:106E7000E3E7012221464046FDF706FF431C064694
:106E8000EFD1CDE72046F9F7E5FB0746E9E7164BDA
:106E90001B68B8B25B689847FF2EBCEEC00A0CD1E5
:106EA000124BF8EE407A1A78114BA24213DC10EE26
:106EB000101A1048FAF7C0FEB2E70F4B0F48F8EE71
:106EC000407A03EB860310EE102A3146C3EDED7ACB
:106ED000FAF7B2FEA4E7E3EC017A0134E5E700BF7C
:106EE00050D70608B8E306084C170010D011001060
:106EF000CCA70020D5E2060818A40020C8E20608A6
:106F0000F8B507460846FEF7BFFDD0B1204BD3F8D1
:106F10009860013630460BF007FD34460546F0B95F
:106F20000134182CA8BF002420460BF0FDFC0546B8
:106F3000A8B9B442F4D138461649BDE8F840FCF788
:106F400087BF0846F9F786FB04460BF0EDFC0546C3
:106F500028B921461048BDE8F840FAF76DBE0C4B41
:106F6000C3F8984005F0FEFE0C482A462146FAF781
:106F700063FE172C09D80A4B0C2202FB043393F84A
:106F8000D006BDE8F84004F003BE0020F9E700BFDA
:106F9000FC050020E4E20608F8E206080EE3060815
:106FA0003CF8050838B5124D04460846FEF76CFD5E
:106FB00060B1104B104893F900104B1C0ABF0F4BE7
:106FC000C9B21978BDE83840FAF736BE0846F9F775
:106FD00041FB032804D8C0B2FAF74AFA2946E4E78D
:106FE00020460749BDE838400322FCF731BF00BF07
:106FF0007AE10608FC05002027E30608E0300020BF
:1070000037E30608F0B5032985B005460C46164659
:1070100014D80B4F3970FAF7F7FD0A492846FFF7E5
:10702000C1FF0949224601A8F9F742F901AB3246EE
:1070300008212846FCF78AFEFF233B7005B0F0BD0F
:10704000FC0500207AE1060827E3060838B5124D52
:1070500004460846FEF718FD60B1104B104893F93E
:1070600001104B1C0ABF0F4BC9B25978BDE838401C
:10707000FAF7E2BD0846F9F7EDFA032804D8C0B2E2
:1070800012F074FD2946E4E720460749BDE8384080
:107090000322FCF7DDBE00BF7AE10608FC050020F4
:1070A00023E30608E030002032E30608F0B50329A8
:1070B00085B005460C46164614D80B4F7970FAF782
:1070C000A3FD0A492846FFF7C1FF09492246684641
:1070D000F9F7EEF86B46324610212846FCF736FEEB
:1070E000FF237B7005B0F0BDFC0500207AE10608A7
:1070F00023E306082DE9F74F444BDFF82C911A786B
:107100005B7889F80130424B00911B7889F80020A8
:1071100005460BB902F074F83BF070FA00263D4CBE
:10712000B0460D233B4A0099734352F803A05046E2
:10713000F9F7D8F9002841D0B8F1000F01DDFAF7CE
:1071400063FD35485146FBF737FF002221462846AC
:10715000FCF770FEFAF758FD237903F01803082BAB
:1071600046D0102B49D02046FBF733FF294B0D2288
:1071700002FB0633B3F809003BF006FA8346D8B1A8
:107180002046F8F7ABFADBE9022107460244014446
:107190002046F8F73BFA78B9019051461F48FBF7B3
:1071A0000BFFDBF80810019A28461346CA1921463E
:1071B000FCF7E2FCFAF728FD08F10108013640F27D
:1071C0005D239E4204F10D04ABD10020F8F765FA6F
:1071D000FF2389F8003089F80130B8F1000F11D190
:1071E000009A0F49284603B0BDE8F04FFCF730BEC7
:1071F0000C492846FFF7D6FEB5E70A492846FFF7AF
:1072000025FFB0E703B0BDE8F08F00BFE0300020FD
:10721000209300201C0706085AD6060852E30608E9
:1072200024D706087AE10608FC0500202DE9F74F6F
:10723000804608460F4644F025FA044620B101284E
:1072400025D13B782A2B22D1A948AA4EAA4FFAF77A
:107250003FFD0025B1464FF00D0A04F001040AFB82
:1072600005F3384659F80310FBF7A6FE31462246CF
:107270004046FCF7DFFD0135FAF7C6FC40F25D231E
:107280009D4206F10D06EAD103B0BDE8F08F3D2125
:10729000384646F0BEFA002800F0238103469A469D
:1072A00013F8012D202AFAD0AAEB070A013005466F
:1072B00010F8013B202BFAD0DFF838B25FFA8AFAD7
:1072C0004FF000090D2303FB09F352465BF803104E
:1072D000009138460BEB0304F9F7E0F8064670BB63
:1072E0000099084644F0CEF9824528D1277907F065
:1072F000E001402900F0898012D871B366797F4A95
:1073000002EBC606002796F8E8220092BA463B46F2
:10731000009ABA4202D9BAF1000F62D02BB12DE027
:107320006029ECD0802900F0A48040467449FCF725
:107330008FFD204603B0BDE8F04FFBF74ABE09F1D0
:10734000010940F25D239945BCD16E493A46404659
:1073500003B0BDE8F04FFCF77BBD07F00703042B3B
:107360001CD10B460A222846F9F7D4F8D4F8053088
:1073700083420146D9D32046F8F7CAFA0D2303FB0E
:1073800009F961485BF80910FBF716FE0022214657
:10739000404603B0BDE8F04FFCF74CBD052B0DD1C6
:1073A00001230A222846F9F7B5F8D4F805308342BC
:1073B0000146BADB5B428342B7DCDCE72846F9F7DB
:1073C00049F917F0050F0BBFB4F80520B4F90520F3
:1073D000B4F80730B4F9073090420146A5DB984273
:1073E000EAE7D6F8E41251F8270060B12946019384
:1073F000F7F7A2FF019B30B9394620464FF0010A4A
:10740000F8F786FA5346013782E76379009307F06D
:107410000707013F009BB342B0DDAA4615F8013BC8
:10742000202BFAD02046F8F75FFA0546042F04D83F
:10743000DFE807F0030E0E141D005046F9F70AF9B5
:10744000A8552C21504646F0E4F90136451CE1E7E9
:107450005046F9F7FFF825F81600F2E700230A2254
:1074600000215046F9F756F845F82600E9E70123D0
:10747000F5E7284644F006F9E37994F805A0A779E2
:10748000DB0706460AD52046F8F72EFA03780146B0
:1074900023B13246284646F0E2F9E0B9DEB1B74200
:1074A00019D32046F8F720FA3A46002146F09AF917
:1074B000B2453FF663AF15493246284646F0CFF94C
:1074C00000283FF45BAF2046F8F70EFA3246294613
:1074D00046F030F952E70E493A464046FCF7B8FC10
:1074E00023E73946404603B0BDE8F04F02E600BF4F
:1074F00062E306081C0706085AD606083CF8050889
:10750000B0E3060824D70608A5E30608DBE706086B
:1075100075E3060870B5044608460E4644F0B2F816
:107520003146054602462046F8F7B8FF68B9635D64
:107530001846F8F79DFF00B933B901352C442046B1
:1075400001340378202BFAD070BD0020FCE708B589
:1075500004460948FAF750FBFAF732FB074BD3F819
:1075600018010DF0F5FF02F005FA012C01D141F0F0
:10757000E9FAF5F7A9F900BFBEE3060818A4002050
:1075800010B5044608460B46FEF77EFA28B90949AD
:1075900003221846F8F782FF28B90748FAF7F2FBEA
:1075A0000120FFF7D4FF20460449BDE81040FCF756
:1075B0004FBC00BFCAE30608CEE306088DDC060810
:1075C0002DE9F74F064601AA08462E49DFF8C48088
:1075D000DFF8C490DFF8ACA046F0E7F84FF0000BFE
:1075E00004465D46012714BBBBF1000F27D1264C92
:1075F000002D43D025482946FAF71EFB23780BB906
:1076000001F0FEFD3AF0FAFF002384F84D30FAF75E
:10761000ADFA15B12846F8F740F89FB13046FDF7AE
:107620003FFD78B1FAF70CF90020FFF790FFBBF1AE
:10763000000F0AD02046F9F70DF885B2C5B93046DB
:10764000FCF71CFC03B0BDE8F08F41462046F8F77C
:1076500049FF80B949462046F8F744FF0028EED09C
:107660005F4601AA5146002046F09FF80446BAE75B
:107670004FF0000BF5E74FF0010BF2E70448FAF783
:1076800081FBBFE750D7060820930020F9E30608E6
:107690001CE40608F0E30608D8E4060810B50C461A
:1076A000FDF7FEFC78B1084B01229A73FAF7C8F88F
:1076B0000648FAF767FB06492046F7F73DFE10B18A
:1076C0000020FFF744FF10BDE030002032E4060840
:1076D00058CD06082DE9F04F93B00E460290A04910
:1076E00030461746FFF716FF0546002840F0218177
:1076F0009C493046FFF70EFF0546002840F01B81ED
:1077000099493046FFF706FF0546002840F01581ED
:1077100096493046FFF7FEFE0546002840F00F81EF
:1077200093493046FFF7F6FE002805460ABF0124BC
:10773000082435467F4207F010078E4928463C430F
:10774000FFF7E8FE002800F0FC8044F020048A4B9C
:107750001B780BB901F054FD3AF050FF14F0090FFB
:1077600000F050838548FAF70DFB0020FCF722F863
:1077700014F48073059340F0EE808148FAF702FB21
:107780008048FAF7A5FA04F01803182B05D17E48B3
:10779000FAF7F8FA7D48FAF79BFA01230493FAF70F
:1077A00033FA7B497B48FAF747FA7B497B48FAF77B
:1077B00043FA04F48473082B07D179490298FAF745
:1077C0004AFA77490298FDF75BF814F080030793B3
:1077D0000ED1744B93F8D423002A734A03F57573C2
:1077E00006BF012113460021704A2046FAF710FA1D
:1077F0006F492046FBF75CFB6E492046FAF7E6FB33
:107800006D492046FAF7D7FA6C4BD3F800A06C4BC1
:1078100014F010061D6840F0A0806A48FAF7B2FA2A
:107820000396694B069399466AEA05034FF00008F0
:10783000099359F804BBBBF1000F21D0099B039AAF
:10784000012707FA08F73B400CBF01210021204621
:107850000893FAF7A3FA65EA0A033B4214BF012131
:1078600000215A4A03905B462046FAF753FC0899D8
:10787000564A00395B4618BF01212046FAF7C8F97D
:1078800008F10108B8F11D0FD3D165EA0A03DFF84A
:10789000549108934FF00008069B53F804BB0693DD
:1078A000BBF1000F24D0012707FA08F73D420AD0A8
:1078B0006AEA05033B424A465B4614BF01210021A8
:1078C0002046FAF727FC1AEA070F11D0089B039A03
:1078D0001F400CBF012100212046FAF75FFA391E34
:1078E00003905B464A4618BF01212046FAF790F9FB
:1078F00008F10108B8F11D0FCED12A4D344B354A9D
:1079000005F23C412046FAF799FC079B002B6BD00F
:10791000134B029822461821FCF718FA049B002BFF
:1079200000F0D4812C48FAF72DFA2C48FAF7D0F958
:10793000CCE10124FEE60224FCE60424FAE68124DC
:10794000F8E627492846FFF7E5FD00283FF4FFAE9B
:1079500044F48074FBE6002320E71A4B039360E7AE
:1079600058E406085FE4060867E406086DE40608C4
:1079700082DF060813E40608209300207BE4060853
:1079800083E406089BE40608A7E40608CFE406089B
:10799000E3D306088FD90608F2D30608ADD9060846
:1079A0007AE1060818A40020DBE70608DFE40608F1
:1079B000ECE40608F6E40608D3D006087438002084
:1079C000B836002039E4060858FE0508FCE406082D
:1079D00013E506084C980020D7E50608EDE50608F3
:1079E00076E4060808E50608DFF8C0A3DFF8C0B3B0
:1079F0009AF800209BF80030BC4F9A4214BF012136
:107A00000021BB4A20460CBF4FF001094FF000098E
:107A1000FAF7C4F99BF80030B64A07EB83038046B7
:107A2000D3F8A83549462046FAF774FB9AF8003097
:107A3000B04A07EB83074946D7F8A835AE4F204632
:107A4000FAF7E6F8D7ED007AAC4AF5EE407AF1EEB7
:107A500010FA0CBF012100212046FAF7D9F8A849F5
:107A600043463A462046FAF7D3FCA64B05F194026A
:107A700005F294412046FAF7D9FE26B195F9263051
:107A8000002B00F02981A048FAF77CF99F48FAF70B
:107A90001FF900239E4A9F4F9F4D02F59A61204691
:107AA000FAF76CFF9D4B9E4A019300923A68296851
:107AB0002046FBF7A7F940F202229A4B019300926D
:107AC000BA68A9682046FBF79DF9002E40F00681B0
:107AD0009548FAF757F93246944F9548DFF8D4C2E3
:107AE0000125002117F8013B10F8018B03F1480E26
:107AF000EE440EF8208C1CF801EB0EF14809E94425
:107B000009F8108C002D00F0EB80A3EB0E056B4202
:107B10006B41013108291D46E4D183F001010027A2
:107B200020468DF83070FAF739F9824A8DF84070A6
:107B30000EAB29462046FAF7EDFA7E4A0AAB2946F3
:107B40002046FAF765F87C4A7C4B02F536712046F0
:107B5000FAF73EFD7A4A7B4B02F536712046FAF77A
:107B60007FFD754A784B02F536712046FAF7C0FD65
:107B7000764B774A77492046FAF7E4FA764A774B0C
:107B800002F27C512046FAF7DFFB754A754B02F290
:107B90007C512046FAF7D8FC734B744A744920464E
:107BA000FAF7C8FF734B744A74492046FAF762FF2C
:107BB000002E40F097807248FAF7E4F8B346714D12
:107BC000DFF8F481A5F5FF67002639460222284632
:107BD00045F08CFE00285A4614BF012100212046A2
:107BE00095F800A00CBF4FF001094FF00009FAF71B
:107BF000D5F8BAF1020F834640F0E0807B784FF071
:107C0000190A40F2EE221AFB032301933B785E4AE5
:107C100018F803300093494633462046FAF77AFABB
:107C20006B7840F2EE221AFB032301932B78564A1D
:107C300018F803300093494633462046F9F7E8FF29
:107C40000136122E05F1020507F10207BDD1002110
:107C50004E4B02982246FCF779F8210740F1C68086
:107C60000025E9B2029822460135FFF7CBF9042D31
:107C7000F7D1474F474D3B782B70059B33B94648AA
:107C8000FAF780F845490298FFF78CF9FF232B702B
:107C90000026F1B2029822460136FFF707FA042EB9
:107CA000F7D17B786B70059B002B40F09C803C48A3
:107CB000FAF768F839490298FFF7C8F93948FAF72E
:107CC00061F83948F9F798FFFF236B70002013B073
:107CD000BDE8F04FF7F7E1BC0B4BDBE6124AFBE6E1
:107CE0002B4616E7DFF898B069E700BF3CF80508B7
:107CF00047E406081AE506086C31002023E506086B
:107D0000CC36002052D7060841E4060832E50608C2
:107D10003CA4002040320020883800203FE50608BF
:107D2000FFFF7F0046E506084DE406087CA9002019
:107D3000046B0608F9D60608D8A600204BDA060818
:107D400058A7002052E506084DE5060858E5060844
:107D500058990020A0AA00209CA500205CE50608F8
:107D6000C8A6002065E506086DE50608F499002020
:107D700054AC002076E50608A032002080370020B1
:107D800051E4060870AD002034E0060858E4060807
:107D90006C370020FC0500207AE506087AE1060829
:107DA0009DE50608C4E50608DAE406087C380020EC
:107DB0006431002018980020146D06083B781B4A97
:107DC00018F803300093494633462046FAF7A2F9E3
:107DD0002B78164A18F8033000934946334620465C
:107DE000F9F716FF2CE7FF236B7097E5104D02980B
:107DF00029782246FFF706F9697802982246FFF7AC
:107E000055F98BE5A20706D5094B02981978224649
:107E1000FFF7F8F85AE763077FF558AF044B02986D
:107E200059782246FFF742F950E700BF44E00608C0
:107E30006C370020224BB0F5FA6F1A680346A8BFD2
:107E40004FF4FA63B3F57A7FB8BF4FF47A73D20474
:107E500016D540F2DC52904215D007EE903A40F22F
:107E6000DB529042F8EE677A1FD8DFED166A9FED7D
:107E7000167A9FED160A77EEE67AA7EE870A704724
:107E8000B0F57A7F02D89FED120A704707EE903A5C
:107E9000DFED106A9FED107A9FED100AF8EE677A19
:107EA00077EEE67AA7EE870A7047DFED0D6A9FED61
:107EB0000D7A9FED0D0A77EEE67AA7EE870A7047F6
:107EC0000C31002000007A44D62000C000E082443B
:107ED0000000000000407A4466100040000040426C
:107EE00000A0BB44D620004000008344704700BF80
:107EF00000207047704700BF002070470120704786
:107F0000704700BF704700BF704700BF704700BF99
:107F10009FED010A704700BF00000000002070477D
:107F2000064B1B78834206D9054B00EB400003EB60
:107F3000C003586970470020704700BFD00500108B
:107F40000C050010034B00EB400003EBC003587C12
:107F5000704700BF0C050010024B1878003818BF9E
:107F600001207047D005001003681B6903B1184752
:107F7000704700BF70B5094C236873B105460026F1
:107F800006E099681A681E7321609047236823B140
:107F90005A68AA1A002A1846F3DA70BDC0B3002046
:107FA0000022FFF797BB0122FFF794BB2DE9F84FA2
:107FB00000261F4DDFF88090DFF880A007460C46B2
:107FC000B0462046FDF760FDD5F800B048B921461F
:107FD0005846F8F787FA20B968682146F8F782FA18
:107FE00080B15846F9F708FE696811B15046FAF7B2
:107FF000E3FFA96811B14846FAF7DEFFF9F704FE7E
:108000004FF0010801363A2E05F11005D9D120466E
:10801000FDF73AFD48B9B8F1000F06D122463846BF
:108020000449BDE8F84FFBF713BFBDE8F88F00BF68
:10803000D82506083BE6060835E606082FE60608BA
:10804000F8B5354C2368002B53D00A2801D00D28F1
:108050004DD1324D2B790BB1F9F7D6FD304E23219E
:10806000304645F0D6FB08B1801B20602368002213
:108070006BB902B12360F9F793FD2B79EBB1BDE841
:10808000F8402848F9F7B8BD01220B46F0E7591E21
:10809000705C2028F8D08AB90022234C204FF2547B
:1080A0003B26013E0CD13146204B9C4211D2E36865
:1080B000206898476B79002BDDD1F8BD2360EBE792
:1080C00021683846FFF726FA01460028ECD1103423
:1080D000E7E72B7923B116491648FBF733FDCAE7CA
:1080E0001548F9F789FD0E48F9F7F2FDC3E7FF2BB4
:1080F000E3D8A0F120025E2ADFD80BB92028DCD01B
:108100005A1C2260064AD054044B1B79002BD4D051
:10811000BDE8F840F9F7F4BF649C0020C0B300202C
:10812000649B002053CD0608D82506087829060848
:108130004FE606086BE6060871E6060808B5254B0B
:108140001B68DB040AD5B5EE400AF1EE10FA12D135
:108150009FED210A44F016FE80B208BDDFED1F7AC4
:10816000B4EEE70AF1EE10FA1CDA9FED1D0A44F0B6
:1081700009FE80B208BDDFED197AB4EEE70AF1EE30
:1081800010FAE5D49FED177AB4EEC70AF1EE10FAB3
:1081900014D870EE677A9FED147A9FED140AA7EE5B
:1081A000870AE4E770EE677A9FED117A9FED110A76
:1081B000A7EE870A44F0E6FD80B208BDDFED0E7A37
:1081C0009FED0E7A70EE677A9FED0D0AA7EE870A93
:1081D000CDE700BF0C3100200080BB4400004042CE
:1081E00000007A4400E0824466BEFFBE0060BB44EB
:1081F00038DFFF3E00407A440000834466BEFF3E05
:1082000000A0BB44F8B5CB4B1B6813F004052DED63
:10821000048B40F0DD809FEDC88AC84C13F020032A
:1082200005D094F8D43013F0020340F09F8094F806
:108230001521DFEDC38A94F8141112F0010240F009
:10824000AC80002940F08D80D4ED467A9FEDBD7A58
:10825000DFEDBD6A67EE877A94ED487AE8EE267A1C
:1082600038EE477AC4ED467A84ED477A63B194F8E4
:108270002821D4F8D830C4F8243101218A4284F866
:10828000161118BFC4F81C31B04B1E780D2E0BD13F
:10829000D4ED367A9FEDAE7AAE4B67EE877AFDEE7F
:1082A000E77A17EE902A9A809FEDA37AB0EE489A6B
:1082B0000025D4ED4E7AD4ED4F6A94ED4D8A37EE19
:1082C000677AE6EE877A37EEC87AC4ED4E7AA6EE84
:1082D000878A84ED4D8A84ED4C8A0DB184ED478AFE
:1082E00094ED507AD4ED527ADFED9B5AD4ED536A77
:1082F00094ED510A84ED508A38EE477AB0EE676A01
:1083000097EE256AE6EE867A37EEC07AC4ED527AA9
:10831000A6EE870A84ED510A84ED540A44F032FD3A
:1083200002B282EAE273A3EBE2739BB2092B40F242
:10833000DC80002AACBF0A380A3005B20D2EA4F842
:10834000545100F0BD80242E00F0D180382E05D18C
:10835000B0EE480A44F016FD7E4B9880BDEC048BCD
:10836000F8BD84F8162184F814216DE7D4ED397A2C
:10837000B4F8E830F8EEE77AC4ED367A002B40F036
:108380008280DFED6F8A94F8152194F8141112F0B1
:1083900001024FF001033FF454AF002962D0D4ED45
:1083A000489A6A4A94F81671167838EE699AA3B119
:1083B00017BB002D00F0A88094ED360A70EE487AC5
:1083C000012377EEA97A84F81631C4ED497A17E0D3
:1083D0005A4C012594ED328A20E70D2E65D0DFED51
:1083E000568AA7B9002D4AD094F82831002B44D1E1
:1083F000B0EE497A01255CE794ED360AD4ED497A6E
:1084000030EE670A0D2E84ED4C0A00F08A8094F855
:1084100028317BBB94ED4C7A002DEBD094F82931B8
:1084200077EE487A06EE903A77EEA97AF8EEE66AA9
:10843000F0EEE77A67EEA67ADFED486AF4EEE67AC8
:10844000F1EE10FAC4BF68EEA66AC6EEA78AF7EE90
:10845000007A77EEE87A67EE897AE8EE877AB0EE0E
:10846000677A26E7D4ED469A0122C4ED489A84F84B
:10847000142196E7022B02D00DB1012BB8D094ED58
:108480004C7A012515E707EE903ADFED336A9FED50
:10849000347AF8EEE77AC6EEA78AF4EEC78AF1EEF0
:1084A00010FA88BFF0EE478A6DE7DFED2E7A94ED83
:1084B0004C0A20EE270A44F065FC264B98808EE794
:1084C000DFED257A9FED270A224C68EEA77A29EE88
:1084D000000AFDEEE77A17EE903A238044F052FC52
:1084E000BDEC048B6080E580F8BD002526E7DFED5C
:1084F0001D7A94ED470A20EE270A44F043FCBDECB8
:10850000048B144B5880F8BD0D2EB8D1DFED157AD1
:1085100094ED4C0A20EE270A44F034FC0D4B988071
:10852000ADE7DFED107A20EE270A44F02BFC094B73
:1085300098806CE79C9C002000000000C0B30020E5
:108540009A99993ECDCC4C3FCDCC4C3E1622002082
:108550000AD7233C182200200000C84200401C46D5
:108560006666663FCDCCCC3D70B5234C2378012B9D
:1085700000D070BD214B1B68002BFAD0204D2B681A
:1085800028465B6898470028F3D01E4B1E4E1A6899
:10859000338892889A421ED31C4909680022496890
:1085A000EA622A6803FB01F12846D36898472B68E2
:1085B0009B6813B128469847D8B1154A338852684A
:1085C00001333380002AD4D01368928859690A4253
:1085D0000DD05A8370BD0E4B0E495B68097800229E
:1085E0002270002BC5D089079A881B68F1D41A83A2
:1085F00070BD40F079FCE0E7862B00202C200020A5
:1086000030200020802B0020842B0020782B00209D
:108610007C20002078200020C34BDB79022B40F027
:1086200021812DE9F047C14C2DED028BB4F8563174
:10863000B4F85821B4F85A519A4282B01ABF0127AF
:10864000A4F85831002715F4006500F0228194F851
:108650005C51002D00F00E82DFF8008394ED4C8A0F
:1086600098F80060B4F9D4A14A2E00F04E81492E4A
:1086700012D1B4F8681100231A4661F30F03B4F85D
:10868000061161F31F43B4F86A116AF30F0261F334
:108690001F42A749C1E90032DFF8C492B4F9D621DC
:1086A00099F81C30DFEDA36ADFEDA37AA3F105038F
:1086B000B3FA83F35B0984F86C31AAEB020307EE8B
:1086C000103AB8EEC77AB4EEE67AF1EE10FA67EE39
:1086D000277A00F20E819FED997A77EE877AF0EE95
:1086E000E78A4A2EA4F86A21C4ED5C7AC4ED618A57
:1086F00000F0D280002F6CD0D4ED767A94ED770A1A
:108700008F4A9FED907A1368C4F87431F8EE677A57
:10871000B4F80431C4ED587A30EE670A67EE876A20
:10872000C4ED777AD2ED017AB4F8E611C4ED596A56
:1087300020EE270A4C2E84ED5E0AA4F8683100F082
:108740004581E9B307EE903AF8EEE77A94F8FD3107
:10875000D4ED886A77EEC07AF1EE005AF0EEE77A4F
:1087600067EE877A07EE103AB8EEC77AF5EEC06A80
:1087700087EE876AF1EE10FA36EE257AC5EE877A33
:10878000C4ED717A40F39881DFED6F7A66EEA77AD7
:10879000B0EE007AF4EEC77AF1EE10FA88BFF0EE90
:1087A000477A042D0AD1B0EE0C7AB4EEC76AF1EE26
:1087B00010FA88BFB0EE476A76EE277AC4ED627A87
:1087C000482E00F052814A2E03D144F0DBFA584B78
:1087D0001880F1F7BFFD99F81C30052B40F0C280DE
:1087E00094F8D43013F0010200F0D680D4F80022BF
:1087F0005649821A8A4240F3F18203F00203002BA9
:1088000094F80821C4F8000214BF0023012384F85F
:10881000043218BF012194F9063208BF0021032A4F
:108820008CBF4FF0FF3201221344022B1A46A8BF1F
:10883000022222EAE272012B84F8062200F3D68299
:10884000002384F8053284F8CC11082D37D8DFE8EE
:1088500015F036017F02CC0194010D02F4012800CD
:108860002B007B013A4B03F1780102E00633994279
:108870000ED01A780A2AF9D19878DA789042FFF463
:10888000D0AE5A79002A7FF4CCAE06339942F0D1AB
:10889000704784F85C51DFE6254BA3F808A05A81A5
:1088A00028E738461BF030FC2A4BD4ED6D7A93ED67
:1088B000187AB4EEE77AF1EE10FA00F3E68098F851
:1088C00000304A2B28D0242B09D1DFED1B7A94ED00
:1088D000630A20EE270A44F055FA154B18801BF066
:1088E000C7FA384602B0BDEC028BBDE8F0471AF07B
:1088F000ADBFDFED196AB4EEE67AF1EE10FAC4BF4F
:108900009FED0E7A77EEC77AE9E6B0EE480A44F0BA
:1089100039FA074B9880BFE694ED650A44F032FAC5
:10892000034BD880DBE700BF4C990020C0B3002088
:10893000182200200000E1C4CDCCCC3D0000B4439F
:10894000980600200AD7233C3EC3AE393F420F00B1
:10895000589900205C1700100000E1441622002006
:10896000A09C0020002384F8CC31082DA7D801A3B7
:1089700053F825F0BF8A0108CD8D0108EB8B010863
:108980007B8B01086D8C01083B8C0108A3880108D2
:10899000A9880108498B010884F8CC21082D8ED8BC
:1089A00001A353F825F000BFBF8A0108D58D010847
:1089B000EB8B01087B8B01086D8C01083B8C010857
:1089C000A3880108A9880108498B0108FDEEC07A37
:1089D000D64817EE906A068100293FF4FAAE07EEFA
:1089E000903AF8EEE77A94F8FD31DFEDD16A77EE50
:1089F000C07A05EE903AF0EEE77A67EE877AF8EE05
:108A0000E55AB1EE005A87EEA56A94ED887A76EEC3
:108A1000054A66EE267AC5EE245AFDEEE77AB5EEF3
:108A2000C07A17EE903AF1EE10FAC4ED715A438114
:108A300040F3F581DFEDBF5A27EE257AF0EE007A9C
:108A4000B4EEE77AF1EE10FA88BFB0EE677A67EE1F
:108A5000267AFDEEE77A17EE903A1BB2042D838159
:108A600000F0E18184ED627AB3E644F08BF9AF4B1C
:108A70009880AEE60123284684F85C311AF0E6FEC1
:108A80001BF0F6F994F85C51E6E5AB4A136843F045
:108A90008053136094F81531D90709D594F81A2238
:108AA0001AB943F0020384F81531072014F02CF9A9
:108AB000002384F85C3102E7DFEDA07A71E694F8D8
:108AC0001531DD0704D49E4B1B7A002B00F0C981C1
:108AD000D4ED637AF4EEC87AF1EE10FAB8BFF0EE96
:108AE000487AC4ED637A002F3FF4E9AEB4F8E4317C
:108AF00094ED597AB4F8F82184ED658A06EE903A3F
:108B0000B6EE006A27EE067AF8EE666A94F8F3315C
:108B1000B4EEE67AF1EE10FA88BFB0EE667A012B79
:108B200084ED6A7A07EE102A00F0EC81B8EEC77A7D
:108B3000DFED7F6A022B27EE267A00F0D78177EEF1
:108B4000877AC4ED647ABAE67B4A136843F08053AF
:108B5000136094F81531DA0709D594F81A221AB976
:108B600043F0020384F81531012014F0CDF80023FE
:108B700084F8AC3184F85C31A1E6D4ED6C7AB7EEC0
:108B8000007AF4EEC77AF1EE10FA05D59FED6D7A12
:108B900077EE877AC4ED6C7AF3EE0E7AF4EEE78A1C
:108BA000F1EE10FA0DD5B4F8E03107EE903A042357
:108BB000F8EE677A84F85C310023C4ED687A84F8B3
:108BC000AC31B4F8E63194ED5E7A07EE903AF8EE07
:108BD000E77A5D4B84ED677AB4EEE77AF1EE10FA4E
:108BE0004CBF012200225A7269E694ED647A564B1A
:108BF000B4EEC87A1A7AF1EE10FACCBF0123002342
:108C0000934200F0F880B4F8EE31D4ED596A84ED67
:108C1000657A07EE903AF8EEE77A0023F4EEE76A19
:108C2000F1EE10FAC4F89831C4BF032384F85C3124
:108C3000D4F87831C4F89C3141E694F808329FEDBD
:108C40003C7A07EE903AF8EEE77A67EE877AB4EE70
:108C5000E78AF1EE10FA05D50622002384F85C219C
:108C600084F8AC3138461BF04FFA28E6364AD4ED8A
:108C70006C7AB7EE007AF4EEC77AF1EE10FA05D509
:108C80009FED307A77EE877AC4ED6C7AB4F8E631EE
:108C900094ED677A07EE903AF8EEE77A537AF4EEBD
:108CA000C77AF1EE10FACCBF012200229A4207D116
:108CB00077EEC77ADFED236AA7EEA67A84ED677AAE
:108CC000D4ED727A9FED216AF7EE006A76EEE76ADC
:108CD000B0EE007AE6EE867A37EE677AC4ED727A05
:108CE00084ED707A002F3FF4EAADB4F8E031D4EDB2
:108CF000595A94ED6A6A06EE903AF8EE666AB6EE54
:108D0000007A26EE877AF4EEC65A67EE277AF1EEFD
:108D100010FAC4ED686AC4ED697A3FF6D0AD052259
:108D2000002384F85C2184F8AC31C8E518220020C7
:108D30000000C8423EC3AE395C9B0020000000002A
:108D4000A89800200AD7233C980600200AD7A33B06
:108D500094ED597AF1EE047AB4EEE77AF1EE10FA76
:108D600000F18E80B4F8EE3107EE903AF8EEE77A33
:108D7000B4EEE77AF1EE10FA00F1968094ED647AA1
:108D8000D4F87821C4F89C21B4EEC78A4FF07E5203
:108D90000023F1EE10FA4FF00001C4F8C021C4F82E
:108DA000C4215F4AC4F8B031C4F8A431C4F8A0317A
:108DB000C4F8C831C4F898314CBF01230B46137274
:108DC000022384F8AC1184F85C3178E594F8D4304F
:108DD000D807BDD4072384F85D3170E594F80432D8
:108DE0003BB994F8051281F001012CE5012384F8C8
:108DF0000532002127E5C3B3B4F8F4319FED497A79
:108E000007EE903AF8EEE77A67EE877A94ED657AA6
:108E1000C4ED667A77EE277AC4ED657A08E79FEDB0
:108E2000427A00231AE6F0EE0C7AB4EEE76AF1EE2D
:108E300010FA98BFF0EE467A77EE877A0192C4ED89
:108E4000627AF1F787FA99F81C30019A052B49D11B
:108E500094F8D43013F001017FF4C8AC84F8CC113D
:108E600005E70023C4F88C3129E5B4F8F6319FED0D
:108E70002F7A07EE903AF8EEE77A67EE877AC5E741
:108E800094F80832DFED2A6A07EE903AF8EEE77AB6
:108E900067EEA67AB4EEE78AF1EE10FA7FF562AFDC
:108EA000082384F85C310AE5B4F8F831DFED205A84
:108EB0009FED206A06EE903AF8EEE66AB0EE487A48
:108EC000A6EEA57AF6EE006AB4EEC67A67EEA67A4A
:108ED000F1EE10FAB8BFB0EE467A84ED647AC4EDD4
:108EE0006A7A4DE7002384F8CC31C0E638EE078A71
:108EF000B4EEC78AF1EE10FAB8BFB0EE478A84ED3F
:108F0000648ADCE4B4F8E2319FED097A07EE903A26
:108F1000F8EEE77A67EE877AC4ED647ACFE400BFB3
:108F2000980600200AD7233C000000000AD723BC83
:108F30000000C84200007A442DE9F8438F4B1B68BB
:108F40005B0701D4BDE8F883DFF874828C4F98F892
:108F500000308C4EBD7AB268372B04BF8A4B1D801F
:108F60001378012B044607D0042D00F2FC80DFE8C3
:108F700005F08BAB96A0140092F90420834902EB14
:108F8000820201EBC202527E002AEDD08049814A62
:108F90000B7013704FF47A7770E0D6F8C0307E48CB
:108FA0009847002800F0A9807C49D6F8C430081DF5
:108FB0009847D6F8D090B9F1000F40F3AD8007EE96
:108FC000909A9FED770ADFED770AF8EEE77A27EEC1
:108FD000800A43F0FDFD74499FED747A744A087865
:108FE000F7EE007A77EEC07A67EE877A92ED007A34
:108FF000002800F09A8077EEC77AC6ED327A98F8AA
:109000000030372B17D107EE909A9FED6A0ADFF8F0
:109010007881F8EEE77A27EE800A43F0B3FED6F8BF
:10902000CC3096ED320AA8F80200A8F8043043F0DC
:10903000A9FEA8F8060096F8A430002B49D1052314
:10904000BB7298464FF47A77514B01221A7006EBA7
:109050008505F1F77FF9D5F82432001B984206EB1D
:10906000880388BFC5F82402D3F82432C6F83C32FE
:10907000002F3FF467AF0A2FB8BF0A274E4B1B687B
:109080001B681F61BDE8F883D6F8B03042489847A6
:1090900098B30123BB7298464FF47A77D4E7D6F899
:1090A000B8303D4898470323BB729846B6F8A8707D
:1090B000CAE7D6F8BC3038489847F0B10423BB72F1
:1090C00098464FF47A77BFE7D6F8B43032489847DD
:1090D00098B10223BB72F1F73DF906EB8505001B41
:1090E000D5F82432834212D2C5F82402D6F82C32A5
:1090F000C6F83C324FF47A77BDE7BB7A254A0121A6
:10910000022B1170E7D098464FF47A779CE7D6F897
:109110002C32C6F83C32EDE7234B1B78002B7FF452
:109120006EAF0023C6F8C83069E7DFF898C0234B5C
:10913000B3F800E0BCF8003001339BB277EE877AD9
:109140009E45C2ED007AACF80030EAD807EE103A3E
:10915000B8EEC77A0123C7EE876AACF800000B703F
:10916000C2ED006ADDE7D6F8AC300B489847002323
:10917000BB729846B6F8A67066E700BF9C9C0020BC
:1091800098060020C0B3002018220020CC1900202F
:109190009018001058170010C8B300208CB400209D
:1091A00008942537B1DC423E80320020D048874AFF
:1091B0007C3200200AD7233C8C1800108232002019
:1091C000162200208432002038B50546F8F7F8FC56
:1091D000094B18680CF0BCF9F8F7E2FC074B0024C7
:1091E0005C711C711EF0DCFC25B12046BDE83840E6
:1091F000FEF7ADB938BD00BF30A50020C0B30020D8
:1092000038B5074C074DAC4203D3074B01221A7007
:1092100038BDD4E90210A28844F08CFA1C34F2E77D
:1092200050ED060810F60608209300202B4B82B064
:109230009A790190002A39D093F82420DFED286A2A
:10924000D979284B07EE902AF8EEE77A264A86EE7F
:10925000A77AA1F10201B1FA81F1127849091972D4
:1092600083ED017A02B321499FED216AB1F84A12D8
:109270009DED017A07EE901AF8EE677AB8EE477A1C
:1092800067EE867AF7EE006A67EE877A0C3377EE40
:10929000A66A002187EEA67A03EBC20219600833A2
:1092A00003ED017A9A42F9D102B07047114A12686F
:1092B0001001F9D593F82420DFED096ADB7907EE78
:1092C000902AF8EEE77A991E86EEA77A054A4B4275
:1092D0004B41137282ED017AE6E700BF8022002045
:1092E0005555554090180010CC050010C0B3002013
:1092F00027D4D2360C31002038B5094D2B7963B113
:1093000000242B685B6B20460BB1984708B90020FE
:1093100038BD2B7901349C42F3D3012038BD00BF06
:109320004C1700100B4BDA7A12B90B4B9879704737
:10933000094A906800B970470849096840F6B83C86
:10934000091A614503DD00219079D9727047002028
:10935000F1E700BF980600204C170010C01900204C
:109360002DE9F84FDFF808821F46531ED8F8005049
:1093700091460646142B00F2AC80DFE803F0565607
:10938000565656AA0B0B0B0BAA0B0B0BAAAAAAAA92
:10939000AA0B0B004FF47A7B4FF00A0A012F4AD038
:1093A000002F40D16D4A6E4B14781878631C03F07F
:1093B0000303834237D06B4D137004EB440305EB7A
:1093C000C3034FF47A7283F80CA09A604FEA440802
:1093D000B1B1182303FB04530C3309E0FF2E07F14E
:1093E00001070CBF4A460022B94203F8012F07D0FB
:1093F000BE42F3D101374A46B94203F8012FF7D1F3
:10940000FFF77AFF002800F09780574A08EB040323
:10941000DB00D268E9180120E85402F51C530F3331
:10942000B3FBF2F34B60BDE8F88F012FDFF844B1D6
:109430004FF0010AB4D14D4A537C012B03D0022BCB
:1094400000F08280002798F80400E0B1444B1C78BB
:10945000444B18220C2112FB04121A44002309E089
:10946000FF2E03F101030CBF49460021834202F89D
:10947000011F08D0D9B28E42F2D10133494683424E
:1094800002F8011FF6D142F22830F1F7D5FA3FF089
:10949000FBFA0FB9EB6998472B6A03B1984798F824
:1094A0000430DBB1002420460AE0FF2E0FD0204616
:1094B0009847013498F80430E4B29C4220460DD21B
:1094C000EB6B9847A642AB6A4FF00001EDD14946DD
:1094D000EDE74FF47A7B4FF0010A5FE7AB6903B128
:1094E0009847EB6A98474FB90AF1FF3A1AF0FF0A1A
:1094F0000ED03FF0C9FAEB699847CDE7EB690AF166
:10950000FF3A98471AF0FF0A02D03FF0BDFAC3E7CE
:109510005846F1F791FA98F80420002A83D0104BAE
:1095200010481C780D21182313FB04131844002144
:10953000BDE8F84F44F056B908EB0403DB00EA1825
:10954000E8545060BDE8F88F9779002F3FF47BAF67
:109550009778083F18BF012775E700BF4D1A002014
:109560004E1A0020501A0020980600208022002069
:109570004C170010A08601002DE9F041134C24780F
:109580000CB9BDE8F08180460F4616461D46CBB1AA
:10959000012BF6D10E4B987980F001000028F0D015
:1095A0002F2EEED80B4B0C4A1B781278013303F0A8
:1095B00003039342E5D02B46324639464046BDE888
:1095C000F041CDE6FFF7AEFEE8E700BFC8A70020F8
:1095D0004C1700104D1A00204E1A002010B5437B86
:1095E00082680446581C6073D154627B237B93428B
:1095F00006D82AB12368D4E9010198470023637390
:1096000010BD00BF427B42B110B503680446D0E9EB
:10961000010198470023637310BD704730B504689B
:109620002578012D83B00BD0022D02D0002003B08D
:1096300030BD236A002BF9D137F02AFA0120F6E772
:1096400094F904408E46944601798DF807C00DF1D7
:109650000703724620463EF069FD0028E7D0204609
:10966000F2F716FE03B030BD30B5056895F800E09E
:10967000BEF1010F95B004468C4643D0BEF1020FF7
:1096800002D0002015B030BD19462B6A002BF8D14E
:10969000CDE90A210DF10F0204920122CDE9053234
:1096A000CDE908336CF07F018DF81C308DF8302047
:1096B0008DF844200D931093129300220023CDE9DE
:1096C0000E238DF80F10EFF3118C102383F3128803
:1096D00003681B6A002B31D0069B04A802461BB10D
:1096E000D3691432002BFBD12B6AEBB1996839B9DD
:1096F0009A4219D01968A9B15B6899680029F7D016
:109700001433F3E795F90450017900922846624634
:10971000F2F7ECFD0028B5D0284615B0BDE8304082
:10972000F2F7B6BDC3E900405FFA8CFC8CF31188F8
:109730002268136A002BFCD10120A3E704AB2B6243
:109740005FFA8CFC8CF31188F1F74AFCF0E700BF5C
:1097500030B5056895F800E0BEF1010F95B00446FC
:109760008C4642D0BEF1020F02D0002015B030BDB1
:1097700019462B6A002BF8D1CDE90A210DF10F0211
:1097800004920122CDE90532CDE908336CF07F0166
:109790008DF81C308DF830208DF844200D931093F7
:1097A000129300220023CDE90E238DF80F10EFF362
:1097B000118C102383F3128803681B6A53B3069B32
:1097C00004A802461BB1D3691432002BFBD12B6ACB
:1097D000B3B1996839B99A4212D0196871B15B680E
:1097E00099680029F7D01433F3E795F9040021793B
:1097F00000926246F2F77AFD15B030BDC3E9004031
:109800005FFA8CFC8CF311882268136A002BFCD160
:109810000120ABE704AB2B625FFA8CFC8CF3118860
:10982000F1F7DEFBF0E700BF10B5036804469B6864
:109830009847FF230122A373627310BD036810B51C
:1098400004461B689847236801219B682046984777
:10985000E37B0133E37310BD2DE9F041069F04461D
:1098600038460D461646984641F00CFF2844A07233
:10987000E672387850B10697294625682046AC69CB
:1098800043463246A446BDE8F0416047BDE8F0815A
:1098900003689B6A184700BF03685B6D03B11847F4
:1098A000704700BF0368DB6C03B11847704700BF07
:1098B0000B46002110B5C17342749A6C03600446D4
:1098C000017302B19047236801219B6820469847A5
:1098D0002368FF21A173DB6C012262731BB1204658
:1098E000BDE81040184710BD01380F280BD8074BB2
:1098F00000EBC00003EB800393F91C0018B9197743
:109900005A77012070470020704700BFC002002036
:10991000074A00235168814202F1240203F1010346
:1099200003D0102BF6D100207047D8B2704700BF8B
:10993000C002002010B40D4B0D4C1B780122824058
:10994000134054F8200051B1003B18BF012318B157
:10995000818802683BB111835DF8044B7047B3FA0C
:1099600083F35B09F3E75183F6E700BF782000201B
:109970007C20002010B50A4C23681B6B9847094BCC
:10998000094A997840F2DC500023A360A4F805301E
:10999000032998BF1046BDE81040F1F74DB800BF4D
:1099A0004C17001080220020FCA6070070B51B4B4E
:1099B0005B79012B06460D4618D1194B1B68ABB1DC
:1099C000184B0846B3F94C42FCF75EF898B92846A4
:1099D000F6F740FE00F54373B3F5C36F04460AD9AA
:1099E00030461149BDE87040FAF732BABDE8704020
:1099F0000E48F8F7C7B90E48F8F7C4F90D48F8F75C
:109A0000FBF8F8F7DDF80C4B18680BF0A1FDFFF739
:109A1000B1FF2046BDE87040F5F764BB342200205A
:109A20002C200020C0B30020ABE606087EE6060826
:109A3000C3E60608BEE3060830A5002010B5044CB6
:109A400023681B6998470023A371A36010BD00BF62
:109A50004C17001010B5074C63791BB12368DB6805
:109A6000984700B910BD044B01221B68A271A36086
:109A700010BD00BF4C170010C01900202DE9F041A7
